:100000000C949E170C94D7170C94D7170C94D717F1
:100010000C94B6430C94B6430C94B6430C94B6437C
:100020000C94D7170C94D7170C94D7170C94D71798
:100030000C94D7170C94712B0C94D7170C94D717DA
:100040000C94D7170C94BD270C94B6D10C94D717E9
:100050000C94098F0C94FF8E0C94D7170C94D7171F
:100060000C94D7170C94D7170C94D7170C94D71758
:100070000C94D7170C94D7170C94D7170C94D71748
:100080000C9472830C94D7170C94D7174E414E4999
:100090004E495459494E46CDCCCC3D0AD7233C1746
:1000A000B7D13877CC2B329595E6241FB14F0A0093
:1000B0000020410000C84200401C4620BCBE4CCA83
:1000C0001B0E5AAEC59D7400407A10F35A00A07200
:1000D0004E18090010A5D4E80000E8764817000083
:1000E000E40B54020000CA9A3B000000E1F5050051
:1000F0000080969800000040420F000000A086019A
:10010000000000102700000000E803000000006469
:1001100000000000000A00000000000100000000D4
:10012000002C76D888DC674F0823DFC1DFAE59E1A9
:10013000B1B796E5E3E453C63AE651997696E8E618
:10014000C28426EB898C9B62ED407C6FFCEFBC9CEB
:100150009F40F2BAA56FA5F490055A2AF75C936BFD
:100160006CF9676DC11BFCE0E40D47FEF520E6B5B8
:1001700000D0ED902E0300943577050080841E0892
:100180000000204E0A000000C80C333333330F98B0
:100190006E12831141EF8D2114893BE65516CFFE77
:1001A000E6DB18D1844B381BF77C1D901DA4BBE403
:1001B00024203284725E228100C9F124ECA1E53D45
:1001C000275045544700504C41005072696E7420CE
:1001D00041626F72746564004D3235005061757311
:1001E000696E672E2E2E004D323400454550524F19
:1001F0004D2056657273696F6E204572726F720082
:10020000454550524F4D20496E64657820457272C5
:100210006F7200454550524F4D2043524320457266
:10022000726F72003F0049676E6F726500526573AE
:10023000657400496E697469616C697A6520454529
:1002400050524F4D0000FE0003FF8007C7C007015A
:10025000E00000E00000F00000700400700E00708C
:100260001F00703F80F00E00E00F01E007C7C003E1
:10027000FF8000FE0000FE0003FF8007C7C00F01E3
:10028000E00E00E03F80F01F00700E007004007070
:100290000000700000F00000E00701E007C7C003A5
:1002A000FF8000FE000E000E000E000E000E000E7D
:1002B000000E000E007FC03F801F000E00040004EF
:1002C000000E001F003F807FC00E000E000E000ECB
:1002D000000E000E000E000E00FFFFFF7F80FFC02B
:1002E000FFC0FFC07F807F80FFC0FFC0FFC03F0016
:1002F0001E000C0050726F6265205A204F666673B4
:1003000065740020082046616374002008204D6158
:1003100078002008204D696E004F6666004F6E0021
:100320004175746F74656D700045207374657073EA
:100330002F6D6D005A2053746570732F6D6D0059C9
:100340002053746570732F6D6D0058205374657061
:10035000732F6D6D00416476616E63656420536533
:100360007474696E67730054656D7065726174753D
:1003700072650053746570732F6D6D00436F6E6608
:10038000696775726174696F6E003F004E657874BD
:1003900020436F726E657200446F6E65004E657823
:1003A0007400486F6D696E672058595A0053746F16
:1003B00072652053657474696E6773004C6F616475
:1003C0002053657474696E677300426564205472CB
:1003D000616D6D696E670050726F6265205A204FC3
:1003E0006666736574004661646520486569676880
:1003F00074004F6666004F6E00426564204C65765F
:10040000656C696E67004C6576656C2042656400BA
:100410004732394E00473239004175746F20486FBA
:100420006D65004D6F74696F6E0053572D4D6F648D
:10043000650053746F77004465706C6F7900536585
:100440006C662D5465737400526573657400436F58
:100450006E66696775726174696F6E005265737458
:100460006F72652044656661756C7473004C6F61D2
:10047000642053657474696E67730053746F72659A
:100480002053657474696E677300424C546F7563D2
:10049000680050726F6265205A204F6666736574FB
:1004A00000416476616E6365642053657474696E9F
:1004B0006773004D61696E003F004261636B0053DA
:1004C000746F70004D323200417474616368204D66
:1004D00065646961004D3231005072696E74206646
:1004E000726F6D204D656469610052656C65617362
:1004F00065204D6564696100436F6E66696775725A
:100500006174696F6E0054656D70657261747572A7
:1005100065004D6F74696F6E00526573756D65206F
:100520005072696E740054756E650053746F70205C
:100530005072696E74005061757365205072696EF7
:100540007400496E666F2053637265656E000A4DD4
:100550003234004D3233202573003F0053746172F2
:1005600074205072696E740043616E63656C005054
:1005700072696E740043616E6E6F7420656E74658F
:1005800072207375626469723A200002202E2E0078
:100590000152656672657368004D61696E002100E5
:1005A000486F74656E6420746F6F20636F6C6400B5
:1005B0004261636B0050726F63656564004D6F74D8
:1005C000696F6E0044697361626C65205374657075
:1005D00070657273004D383400426564204C657656
:1005E000656C696E67004175746F20486F6D6500BA
:1005F000473238004D61696E0050726568656174FC
:10060000202420426564005072656865617420246E
:1006100020456E640054656D706572617475726515
:1006200000C601C101436F6F6C646F776E0050723A
:10063000656865617420240046616E2053706565AD
:100640006400426564004E6F7A7A6C65004D6169A2
:100650006E0050726F6265205A204F666673657433
:1006600000466C6F770046616E20537065656400CC
:10067000426564004E6F7A7A6C65005370656564FC
:10068000004D61696E00486F6D696E672046616953
:100690006C6564006F70656E00545249474745525F
:1006A0004544003A20007A5F6D696E00795F6D699C
:1006B0006E00785F6D696E005265706F7274696E5E
:1006C0006720656E6473746F7020737461747573E2
:1006D0000A0020746F6F206C6F6E672065787472EB
:1006E0007573696F6E2070726576656E7465640AE5
:1006F0000020636F6C6420657874727573696F6E27
:100700002070726576656E7465640A00486F6D6569
:100710002025732573257320466972737400576111
:10072000726E696E673A20486F6D696E6720427518
:100730006D702044697669736F72203C20310A0025
:10074000020204000040C10000E0C0000000000000
:100750000068430000634300007A430000A04000AB
:1007600000A04000000040FFFDFCFAF8F6F4F2F0B3
:10077000EEECEAE9E7E5E3E1E0DEDCDAD9D7D5D46F
:10078000D2D0CFCDCBCAC8C7C5C3C2C0BFBDBCBA0B
:10079000B9B7B6B4B3B2B0AFADACAAA9A8A6A5A478
:1007A000A2A1A09E9D9C9A99989795949392908FC0
:1007B0008E8D8B8A8988878684838281807F7E7DE7
:1007C0007B7A797877767574737271706F6E6D6CF1
:1007D0006B6A696867666564636261605F5E5D5CE1
:1007E0005B5A5958585756555453525150504F4EC2
:1007F0004D4C4B4A4A49484746464544434242418C
:10080000403F3E3E3D3C3B3B3A3938383736353544
:10081000343332323130302F2E2E2D2C2B2B2A29EF
:100820002928272726252524232322212120201F8C
:100830001E1E1D1C1C1B1B1A19191818171616151D
:100840001514131312121111100F0F0E0E0D0D0CA3
:100850000C0B0A0A0909080807070606050504041F
:10086000030302020100000000000100000001007B
:10087000008000555555000000400033333300AA76
:10088000AA2A004992240000002000C7711C009988
:10089000991900D1451700555515003BB113002497
:1008A00049120011111100000010000F0F0F00E39A
:1008B000380E0043790D00CCCC0C00C3300C00E89E
:1008C000A20B0064210B00AAAA0A00703D0A009D39
:1008D000D80900427B090092240900DCD308008873
:1008E0008808001042080000000800F0C1070087D7
:1008F00087070075500700711C07003EEB0600A13A
:10090000BC06006990060066660600703E0600613F
:1009100018060017F4050074D105005BB00500B29D
:10092000900500627205005555050078390500B83C
:100930001E0500050505004EEC040087D40400A147
:10094000BD040090A7040049920400C17D0400EE9C
:10095000690400C7560400444404005C32040008E3
:1009600021040041100400000004003FF00300F8DF
:10097000E0030026D20300C3C30300CCB503003A52
:10098000A803000A9B0300388E0300C08103009F68
:10099000750300D0690300505E03001D530300344B
:1009A000480300913D030033330300162903003848
:1009B0001F030097150300300C0300030303000B13
:1009C000FA020049F10200BAE802005CE002002DE0
:1009D000D802002DD0020059C80200B0C002003178
:1009E000B90200DAB10200AAAA0200A0A30200BC68
:1009F0009C0200FA9502005C8F0200DF88020082F0
:100A0000820200457C020027760200277002004324
:100A10006A02007C640200D05E02003F590200C8F6
:100A200053020000005C4300005C4300007A430076
:100A30000040C10000E0C00000000053657474690C
:100A40006E67732053746F726564000000FA430090
:100A500000FA430000A0400000C8410000A042008E
:100A600000A0420000C8430080C043F4010000F42D
:100A7000010000640000008813000024F4D430500A
:100A8000C38E20C2A24017828B7011127A910D8101
:100A90006CD90AA861E108C7586607615143061E70
:100AA0004B5D05C145A7041A411104093D98037126
:100AB0003931034036DB0265339102D43054028071
:100AC0002E1D02632CEE01752AC501B028A001106D
:100AD0002781018F2564012B244B01E0223401ACD6
:100AE000211F018D200D01801FFC00841EED009749
:100AF0001DDF00B81CD200E61BC600201BBC006432
:100B00001AB200B219A8000A19A0006A189900D1F7
:100B100017910040178B00B516840031167E00B384
:100B20001579003A157300C7146F0058146A00EE67
:100B30001366008813630025135E00C7125B006C08
:100B400012570015125400C111510070114F0021AD
:100B5000114B00D61049008D10470046104400028A
:100B6000104200C00F4000800F3E00420F3C0006C4
:100B70000F3B00CB0E3800930E37005C0E3500277C
:100B80000E3400F30D3200C10D3100900D300060C5
:100B90000D2E00320D2D00050D2C00D90C2B00AEB2
:100BA0000C2900850C29005C0C2700350C27000E51
:100BB0000C2600E80B2400C40B2400A00B23007DAE
:100BC0000B23005A0B2100390B2100180B2000F8D1
:100BD0000A1F00D90A1E00BB0A1E009D0A1D0080C4
:100BE0000A1D00630A1C00470A1B002C0A1B001187
:100BF0000A1A00F7091A00DD091900C4091900AB27
:100C0000091900920917007B091800630917004CA5
:100C100009160036091600200916000A091500F504
:100C2000081500E0081400CC081400B8081400A44B
:100C3000081400900813007D0812006B0813005878
:100C4000081200460812003408110023081100128F
:100C500008110001081100F0071000E0071000D093
:100C6000071000C0071000B0070F00A10710009187
:100C7000070E0083070F0074070F0065070E00576B
:100C8000070E0049070E003B070D002E070E00203F
:100C9000070D0013070D0006070D00F9060C00ED07
:100CA000060D00E0060C00D4060C00C8060C00BCC3
:100CB000060C00B0060C00A4060B0099060C008D73
:100CC000060B0082060B0077060B006C060B00611A
:100CD000060A0057060B004C060A0042060A0038B6
:100CE000060A002E060A0024060A001A060A001048
:100CF00006090007060A00FD050900F4050900EBD6
:100D0000050900E2050900D9050900D0050900C759
:100D1000050900BE050900B5050800AD050800A5D8
:100D20000509009C050800940508008C050800844E
:100D30000508007C050800740508006C05070065BF
:100D40000508005D050700560508004E0507004729
:100D50000507004005080038050700310507002A8F
:100D6000050700230507001C050600160507000FF0
:100D70000507000805060002050700FB040600F54C
:100D8000040700EE040600E8040600E2040700DBA6
:100D9000040600D5040600CF040600C9040600C3FB
:100DA000040600BD040600B7040600B1040500AC4B
:100DB000040600A6040600A00405009B0406009596
:100DC000040500900406008A0405008504050080DF
:100DD0000406007A04050075040500700405006B24
:100DE00004050066040500610405005C0405005765
:100DF000040500520405004D0405004804050043A5
:100E00000405003E0404003A0405003504050030E2
:100E10000404002C04050027040400230405001E1C
:100E20000404001A04040016040500110404000D53
:100E3000040400090405000404040000040400FC88
:100E4000030400F8030400F4030400F0030400ECBE
:100E5000030400E8030400E4030400E0030400DCEE
:100E6000030400D8030400D4030400D0030400CC1E
:100E7000030400C8030300C503030024F404D920BD
:100E80001BC40C5C0E9804C4095F0265077101F471
:100E900005F900FB04B30048048700C1036900584A
:100EA00003550003034500BE023A0084023100539B
:100EB000022A002902250004022000E4011C00C8C7
:100EC000011900AF0117009801140084011300718B
:100ED0000110006101100051010E0043010D0036A8
:100EE000010B002B010B0020010B00150109000C68
:100EF00001090003010800FB000800F3000800EBF3
:100F0000000700E4000600DE000600D8000600D25C
:100F1000000600CC000500C7000500C2000500BDAA
:100F2000000400B9000400B5000400B1000400ADE5
:100F3000000400A9000400A5000300A20003009F14
:100F40000004009B0003009800030095000200933A
:100F5000000300900003008D0002008B0003008856
:100F60000002008600020084000300810002007F6E
:100F70000002007D0002007B000200790002007781
:100F8000000100760002007400020072000100718E
:100F90000002006F0002006D0001006C0002006A98
:100FA00000010069000200670001006600010065A1
:100FB00000010064000200620001006100010060A5
:100FC0000001005F0002005D0001005C0001005BA9
:100FD0000001005A000100590001005800010057AB
:100FE00000010056000100550001005400010053AB
:100FF00000000053000100520001005100010050A8
:101000000001004F0001004E0000004E0001004DA5
:101010000001004C0001004B0000004B0001004AA1
:10102000000100490001004800000048000100479D
:101030000001004600000046000100450000004598
:101040000001004400010043000000430001004291
:10105000000000420001004100000041000100408A
:101060000001003F0000003F0001003E0000003E84
:101070000001003D0000003D0001003C0000003C7C
:101080000000003C0001003B0000003B0001003A72
:101090000000003A0001003900000039000100386A
:1010A0000000003800000038000100370000003761
:1010B0000001003600000036000000360001003557
:1010C000000000350000003500010034000000344D
:1010D0000000003400010033000000330000003342
:1010E0000001003200000032000000320001003137
:1010F000000000310000003100010030000000302D
:10110000000000300001002F0000002F0000002F21
:101110000000002F0001002E0000002E0000002E15
:101120000001002D0000002D0000002D0000002D0A
:101130000001002C0000002C0000002C0000002CFE
:101140000001002B0000002B0000002B0000002BF2
:101150000001002A0000002A0000002A0000002AE6
:1011600000010029000000290000002900000029DA
:1011700000000029000100280000002800000028CD
:1011800000000028000000280001002700000027C0
:1011900000000027000000270000002700010026B3
:1011A00000000026000000260000002600000026A7
:1011B000000100250000002500000025000000259A
:1011C000000000250000002500010024000000248C
:1011D000000000240000002400000024000100237F
:1011E0000000002300000023000000230000002373
:1011F0000000002300000023000100220000002264
:101200000000002200000022000000220000002256
:101210000001002100000021000000210000002149
:10122000000000210000002100000021000100203A
:10123000000000200000002000000020000000202E
:101240000000002000000020000000200001001F1E
:101250000000001F0000001F0000001F0000001F12
:101260000000001F0000001F0001001E0000001E03
:101270000000001E0000001E000000393000003396
:1012800025000087190000B00F0000DB080000BD3A
:10129000040000740200003F01000020436F756EDF
:1012A0007420583A0042656400453100450062658B
:1012B00064002C2073797374656D2073746F707083
:1012C000656421204865617465725F49443A200075
:1012D0004572723A204D415854454D50004D415889
:1012E00054454D50207472696767657265640048A3
:1012F000656174696E67204661696C656400486564
:101300006174696E67206661696C6564004572721C
:101310003A204D494E54454D50004D494E54454D8F
:10132000502074726967676572656400544845525D
:101330004D414C2052554E415741590054686572F9
:101340006D616C2052756E6177617900202F0020ED
:1013500042403A0020403A007C3C3E5E2B3D3F2F0D
:101360005B5D3B2C2A225C00434F4D4D554E49435B
:101370004154494F4E0044525952554E0045525225
:101380004F525300494E464F004543484F00535477
:101390004F505045442E20005072696E7465722083
:1013A00073746F707065642064756520746F206558
:1013B00072726F72732E204669782074686520659A
:1013C00072726F7220616E6420757365204D3939B9
:1013D0003920746F20726573746172742E202854E2
:1013E000656D7065726174757265206973207265D0
:1013F0007365742E2053657420697420616674656A
:10140000722072657374617274696E67290A004E86
:101410006F20436865636B73756D2077697468200E
:101420006C696E65206E756D6265722C204C6173FF
:1014300074204C696E653A20004E6F2043686563E6
:101440006B73756D2077697468206C696E65206EAA
:10145000756D6265722C204C617374204C696E65E9
:101460003A2000636865636B73756D206D69736DF9
:10147000617463682C204C617374204C696E653A0A
:1014800020004C696E65204E756D6265722069732F
:10149000206E6F74204C617374204C696E65204E11
:1014A000756D6265722B312C204C617374204C6910
:1014B0006E653A20004D3131300053657269616CC0
:1014C00020737461747573206D69736D61746368E2
:1014D0000A0053442072656164206572726F720A5B
:1014E000002121204B494C4C2063617573656420B9
:1014F000627920746F6F206D75636820696E616317
:10150000746976652074696D65202D20637572722B
:10151000656E7420636F6D6D616E643A20004D6579
:1015200064696120496E73657274656400627573E5
:10153000793A2070617573656420666F7220696EF8
:101540007075740A00627573793A207061757365FD
:101550006420666F7220757365720A006275737914
:101560003A2070726F63657373696E670A00506C1E
:1015700065617365205265736574005052494E541D
:1015800045522048414C5445440025533A202553A8
:10159000004B494C4C45442E20005072696E7465D6
:1015A000722068616C7465642E206B696C6C2829EC
:1015B0002063616C6C6564210A0053544F505045A0
:1015C000442E20005072696E7465722073746F70BF
:1015D0007065642064756520746F206572726F7227
:1015E000732E2046697820746865206572726F7268
:1015F00020616E6420757365204D39393920746F10
:1016000020726573746172742E202854656D706544
:101610007261747572652069732072657365742ECA
:101620002053657420697420616674657220726548
:101630007374617274696E67290A006563686F3A32
:10164000004572726F723A004F4646004F4E00429C
:10165000696C696E656172204C6576656C696E6750
:1016600020477269643A0A0021212053544F5020C8
:1016700063616C6C65642062656361757365206F7E
:101680006620424C546F756368206572726F7220D9
:101690002D20726573746172742077697468204DAF
:1016A0003939390A0021212053544F502063616C8D
:1016B0006C65642062656361757365206F662042A6
:1016C0004C546F756368206572726F72202D2072A2
:1016D0006573746172742077697468204D39393983
:1016E0000A004F46460A00466164652048656967FE
:1016F00068742000426564204C6576656C696E678D
:1017000020004661696C656420746F20656E6162BB
:101710006C6520426564204C6576656C696E670A6D
:1017200000496E76616C6964206D6573682E0A00ED
:1017300050726F62696E6720506F696E7400255336
:101740002025692F2569002E0A002F0050726F6234
:10175000696E67206D65736820706F696E74200014
:10176000202844525952554E29004732392041759C
:10177000746F20426564204C6576656C696E670005
:101780003F20284C2C522C462C4229206F75742067
:101790006F6620626F756E64732E0A003F285629AB
:1017A0006572626F7365206C6576656C20696D701B
:1017B0006C61757369626C652028302D34292E0A9E
:1017C00000426164205A2076616C75650A004E6F94
:1017D0002062696C696E65617220677269640A00D3
:1017E0004732384C300020204D3230312058004DE7
:1017F000617820416363656C65726174696F6E2006
:1018000028756E6974732F7332290020204D323091
:10181000332058004D617820666565647261746597
:10182000732028756E6974732F732900205200206D
:10183000204D323034205000416363656C65726125
:1018400074696F6E2028756E6974732F7332292046
:1018500028503C7072696E742D616363656C3E2024
:10186000523C726574726163742D616363656C3E92
:1018700020543C74726176656C2D616363656C3EC7
:101880002900204A0020540020530020204D3230EF
:1018900035204200416476616E6365642028423CD5
:1018A0006D696E5F7365676D656E745F74696D6594
:1018B0005F75733E20533C6D696E5F66656564724B
:1018C0006174653E20543C6D696E5F74726176652B
:1018D0006C5F66656564726174653E204A3C6A753A
:1018E0006E635F6465763E29002044002049002035
:1018F000204D333031205000486F74656E642050A5
:1019000049440020440020490020204D3330342039
:10191000500042656420504944002E0A00206E6F3A
:10192000742064697361626C65642E20536861720F
:101930006564207769746800203B204C6576656C8F
:10194000696E67200020204D3432302053004175ED
:10195000746F20426564204C6576656C696E670023
:1019600020460020420020480020204D3134352000
:1019700053004D6174657269616C206865617475AE
:101980007020706172616D657465727300204A0029
:101990002020473239205720490020204D3134394A
:1019A0002043203B20556E69747320696E20436587
:1019B0006C736975730A0054656D70657261747536
:1019C000726520556E697473002020473231203BC8
:1019D000004C696E65617220556E69747300204910
:1019E0006E76616C696420657874727564657220C6
:1019F00000536C6565702E2E2E005A2050726F6257
:101A0000652050617374204265640A005A20507248
:101A10006F626520506173742042656400205A3AF9
:101A2000200020593A200042656420583A20004D99
:101A300065736820706F696E74206F7574206F66AF
:101A40002072616E67650A00436C69636B20746F76
:101A500020526573756D652E2E2E00616C736F209C
:101A6000656E61626C6564290A004E6F204D6F7669
:101A7000652E004E6F206D656469610A00456E64D5
:101A80002066696C65206C6973740A004265676939
:101A90006E2066696C65206C6973740A00286E6F2D
:101AA0002066696C6529004E6F7420534420707263
:101AB000696E74696E670A005344207072696E74AF
:101AC000696E672062797465200043757272656E75
:101AD000742066696C653A20002E0A0044656C65C6
:101AE00074696F6E206661696C65642C2046696C50
:101AF000653A200046696C652064656C65746564B0
:101B00003A002569730025696D20256973002569F0
:101B1000682025696D202569730025696420256981
:101B2000682025696D20256973002569792025695C
:101B300064202569682025696D202569730050722D
:101B4000696E742074696D653A20006F6B006F6672
:101B50006600891384137D13761368134445425538
:101B6000473A004D3131322053687574646F776E97
:101B7000004D3131332053004D656761205A657245
:101B80006F204F46462E00434F4E4649475F45580B
:101B9000504F5254004D4541545041434B00434F28
:101BA0004F4C45525F54454D504552415455524556
:101BB000004348414D4245525F54454D50455241C6
:101BC0005455524500424142595354455050494E94
:101BD000470041524353004D4F54494F4E5F4D4FC4
:101BE00044455300544845524D414C5F50524F5468
:101BF000454354494F4E00455854454E4445445F73
:101C00004D3230004C4F4E475F46494C454E414D9A
:101C100045004155544F5245504F52545F53445F15
:101C20005354415455530053445F5752495445004F
:101C30005245504541540053444341524400505290
:101C40004F4D50545F535550504F525400484F53CE
:101C5000545F414354494F4E5F434F4D4D414E44B5
:101C60005300454D455247454E43595F50415253ED
:101C7000455200434153455F4C494748545F4252E7
:101C8000494748544E45535300544F47474C455FCE
:101C90004C494748545300534F4654574152455FAF
:101CA000504F574552004255494C445F50455243AE
:101CB000454E54004C4556454C494E475F444154AF
:101CC00041005A5F50524F42450052554E4F5554B5
:101CD000004155544F4C4556454C005052494E54C6
:101CE0005F4A4F420050524F4752455353004155AF
:101CF000544F5245504F52545F54454D500041553A
:101D0000544F5245504F52545F504F5300564F4C12
:101D1000554D455452494300454550524F4D0042A0
:101D2000494E4152595F46494C455F5452414E53CA
:101D30004645520053455249414C5F584F4E5F58FB
:101D40004F4646004649524D574152455F4E414D20
:101D5000453A4D61726C696E20322E302E392E3329
:101D60002D6B616431202844656320323720323086
:101D700032312031333A34393A34332920534F55F4
:101D80005243455F434F44455F55524C3A6769742F
:101D90006875622E636F6D2F6B61642F4D61726C7D
:101DA000696E2050524F544F434F4C5F564552532B
:101DB000494F4E3A312E30204D414348494E455F00
:101DC000545950453A4D656761205A65726F2045F8
:101DD000585452554445525F434F554E543A312062
:101DE000555549443A64626663636435352D6562CE
:101DF00062612D343631352D616264372D313936CB
:101E00006161343338663330340A002F2F004D318E
:101E1000343520533C696E6465783E206F757420BC
:101E20006F662072616E67652028302D31290A00A7
:101E30003F4A206F7574206F662072616E6765205F
:101E400028302E303120746F20302E33290A0020A4
:101E5000580020204D61783A2000200020204D6954
:101E60006E3A2000203B200020204D32313120539B
:101E70000046523A0020466C6F773A2000206F757A
:101E800074206F662072616E67650A005365727612
:101E90006F20003A200020536572766F2000507248
:101EA0006F6265204F6666736574205A0050726FCA
:101EB0006265204F6666736574205A00646973001A
:101EC000656E0043290A0061626C656420286D69B3
:101ED0006E2074656D702000436F6C6420657874AB
:101EE00072756465732061726520004D3432312053
:101EF000696E636F727265637420706172616D6583
:101F00007465722075736167650A004D657368209A
:101F1000706F696E74206F7574206F662072616EC9
:101F200067650A00454550524F4D204F4B0A002926
:101F30000A0020746F20003F5A206F7574206F666E
:101F40002072616E6765202800290A0020746F20C6
:101F5000003F59206F7574206F662072616E67654F
:101F600020282D00290A0020746F20003F58206F80
:101F70007574206F662072616E676520282D004D94
:101F8000383400446F6E65207072696E74696E67D4
:101F90002066696C650A004D3737004D33310049C2
:101FA0006E76616C69642065787472756465720A16
:101FB000004361703A0020286D6D2900203B00200D
:101FC000204D3835312058005A2D50726F626520EF
:101FD0004F666673657400436F6F6C696E672E2E73
:101FE0002E0048656174696E672E2E2E00453120E3
:101FF00025530020573A0020573A00426564204399
:102000006F6F6C696E672E2E2E00426564204865E6
:102010006174696E672E2E2E0023646566696E6595
:102020002044454641554C545F00626564004B6452
:1020300020004B6920004B7020005049442041751E
:10204000746F74756E652066696E69736865642166
:102050002050757420746865206C617374204B7017
:102060002C204B6920616E64204B6420636F6E737B
:1020700074616E74732066726F6D2062656C6F7729
:1020800020696E746F20436F6E6669677572617444
:10209000696F6E2E680A00504944204175746F7450
:1020A000756E65206661696C6564212074696D6573
:1020B0006F75740A00504944204175746F74756ED1
:1020C00065206661696C6564212054656D70657278
:1020D000617475726520746F6F20686967680A00A3
:1020E000504944204379636C65730025532025696A
:1020F0002F256900204B643A2000204B693A2000CC
:10210000204B703A200020436C6173736963205048
:102110004944200A00204E6F206F76657273686F05
:102120006F740A002054753A2000204B753A200045
:10213000206D61783A2000206D696E3A200020649D
:102140003A200020626961733A2000576169742067
:10215000666F7220686561742075702E2E2E005097
:102160004944204175746F74756E65207374617293
:10217000740A00504944204175746F74756E65206F
:102180006661696C6564212054656D706572617467
:1021900075726520746F6F20686967680A0050491E
:1021A00044204175746F74756E6500504944204138
:1021B00075746F74756E65206661696C6564212045
:1021C000426164206865617465722069640A004533
:1021D00072723A207574663820666F6E74206E6F66
:1021E0007420696E697469616C697A65642E004552
:1021F00072723A207574663820666F6E74206E6F46
:102200007420696E697469616C697A65642E004531
:1022100072723A207574663820666F6E74206E6F25
:102220007420696E697469616C697A65642E004214
:10223000656400456E636C6F737572650025687523
:102240003A25303268750025303268753A253032CB
:102250006875002530326875272530326875002092
:1022600020202020202000202020200065727200E5
:102270001FE020102010201010201020201020100F
:1022800030300840048003001FE03FF03FF03FF093
:102290001FE01FE03FF03FF03FF00FC0078003005A
:1022A0003FFFF038007030FC3020FC102078102008
:1022B00030102C00D02E31D02F7BD02F7BD02E3160
:1022C000D02C00D020301020781020FC1030FC30B2
:1022D0003800703FFFF03FFFF03800703186302348
:1022E00087102787902F87D02F03D0203010207899
:1022F000102078102030102F03D02F87D027879000
:102300002387103186303800703FFFF01FFFF81F21
:10231000FFF80410400208200208200410400820A2
:10232000801041001041000820800410400000008F
:102330001FFFF81FFFF8001DC43F0000000C8619A6
:102340008000000D0E198000000F0B198000000D99
:102350009F198000000DD3998000001CFBFF000036
:10236000000000000000000000000000F380001FDB
:1023700080007700001980005B1CF6131DAE5B35F2
:10238000AB0635FB5B3DA70CBD9B4B30EB19B19BFE
:10239000E39D8E9F9D8E0001E00000000001200063
:1023A00000000001E0000000000C0F00FE07022505
:1023B00003BB017FFE08FE08FE050808060000407A
:1023C000F0C88888987810050808060000C0F888CA
:1023D00088888888F80505050600012030F8302037
:1023E0000508080600002070F820202020E00509DC
:1023F000090600FF2070A8A8B88888702007050586
:10240000070001D86C366CD80509090600FFF8A84A
:102410008888888888A8F8050A0A0600FE20505097
:10242000505088A8A8887003030306000340A0400A
:10243000FFFFFFFFFFFFFFFFFFFFFFFFFFFFFFFFAC
:10244000FFFFFFFFFFFF0000000605FF0107070673
:10245000020080808080800080030303060105A0C5
:10246000A0A005060606000050F85050F8500509D7
:10247000090600FF2070A8A07028A8702005070793
:10248000060000C8C81020409898050707060000FD
:1024900040A0A040A8906801030306020580808048
:1024A0000309090601FF204040808080404020034E
:1024B00009090601FF804040202020404080050798
:1024C0000706000020A8702070A82005050506005A
:1024D000012020F820200203030601FFC0408005F0
:1024E0000101060003F8020202060100C0C0050750
:1024F000070600000810102040408005070706006E
:1025000000708898A8C8887003070706010040C0BB
:1025100040404040E0050707060000708808102092
:1025200040F8050707060000F80810300888700515
:10253000070706000010305090F810100507070636
:102540000000F880F00808887005070706000030D2
:102550004080F0888870050707060000F808101012
:102560002020200507070600007088887088887082
:1025700005070706000070888878081060020505C6
:10258000060100C0C000C0C00206060601FFC0C0B0
:1025900000C0408003050506010120408040200561
:1025A0000303060002F800F8030505060101804058
:1025B00020408005070706000070881020200020BA
:1025C0000507070600007088B8A8B88070050707DF
:1025D000060000708888F8888888050707060000CC
:1025E000F04848704848F0050707060000708880EA
:1025F00080808870050707060000F0484848484872
:10260000F0050707060000F88080F08080F80507D5
:1026100007060000F88080F080808005070706002C
:1026200000708880809888700507070600008888F9
:1026300088F8888888030707060100E0404040408A
:1026400040E00507070600003810101010906005E4
:1026500007070600008890A0C0A09088050707061D
:102660000000808080808080F805070706000088D1
:10267000D8A8888888880507070600008888C8A821
:102680009888880507070600007088888888887001
:10269000050707060000F08888F08080800507079E
:1026A00006000070888888A8906805070706000063
:1026B000F08888F0A09088050707060000708880E1
:1026C00070088870050707060000F82020202020E9
:1026D0002005070706000088888888888870050715
:1026E00007060000888888885050200507070600E4
:1026F0000088888888A8A8500507070600008888F1
:102700005020508888050707060000888850202040
:102710002020050707060000F80810204080F80375
:1027200009090601FFE080808080808080E0050745
:102730000706000080404020101008030909060128
:10274000FFE020202020202020E0050303060005D4
:102750002050880501010600FEF803030306010569
:102760008040200505050600007008788878050778
:10277000070600008080F0888888F00505050600BF
:1027800000708080887005070706000008087888B8
:102790008888780505050600007088F080700507B8
:1027A00007060000304840E04040400507070600AB
:1027B000FE7088888878087005070706000080800A
:1027C000F0888888880307070601004000C0404061
:1027D00040E00409090601FE1000301010101090AE
:1027E0006005070706000080808890E09088030756
:1027F00007060100C04040404040E00505050600D6
:1028000000D0A8A8A8A8050505060000B0C88888BB
:10281000880505050600007088888870050707068A
:1028200000FEF0888888F080800507070600FE78A3
:10283000888888780808050505060000B0C88080EB
:102840008005050506000078807008F0050707067A
:1028500000002020F820202018050505060000882B
:102860008888986805050506000088888850200536
:1028700005050600008888A8A85005050506000083
:1028800088502050880507070600FE888888502059
:102890004080050505060000F8102040F8030909EE
:1028A0000601FF20404040804040402001090906C9
:1028B00002FF80808080808080808003090906017B
:1028C000FF80404040204040408005030306000256
:1028D00048A890FF43616E6E6F74206F70656E2024
:1028E00073756264697220005344206361726420CE
:1028F0006F6B0A006F70656E526F6F74206661694E
:102900006C65640A00766F6C756D652E696E69740E
:10291000206661696C65640A004E6F205344206331
:102920006172640A002E0A006F70656E206661692C
:102930006C65642C2046696C653A200046696C65BC
:102940002073656C65637465640A002053697A6559
:102950003A200046696C65206F70656E65643A20A8
:1029600000454E4420535542524F5554494E450A56
:10297000002220706F73002220706172656E743ABD
:102980002200535542524F5554494E452043414C25
:102990004C207461726765743A22005375626361FA
:1029A0006C6C204F766572666C6F77004578636556
:1029B00065646564206D617820535542524F5554CB
:1029C000494E452064657074683A006672657368A4
:1029D00000646F696E67002066696C653A20004E7E
:1029E0006F77200057726974696E6720746F206674
:1029F000696C653A20006D61726C696E66772E6F46
:102A0000726700322E302E392E332D6B6164310007
:102A10001FFFFFFFFFFFFF600000000001FF4000FD
:102A200000000000FF8000000000007F83CF000056
:102A30000C303F87FF80000C301F867980000C002F
:102A40000F8C30C7838C30E78C30CFC7CC31F38C00
:102A500030DCECEC33B98C30D86C6C33198C30D062
:102A60006C0C33198C30D86C0C33198C30DC6C0E38
:102A70003B198C30CF7C079F198C30C77C038F1992
:102A800040000000000002600000000000061FFF80
:102A9000FFFFFFFFF870012C0190012701B0012218
:102AA00001C0011D01F00118011002130130020ED6
:102AB000016002090190020401C002FF000003FA54
:102AC000004003F5008003F000D003EB002004E693
:102AD000007004E100E004DC004005D700C005D22E
:102AE000004006CD00D006C8008007C3003008BEF5
:102AF00000F008B900C009B400B00AAF00B00BAADA
:102B000000D00CA500000EA000500F9B00C0109636
:102B1000005012910000148C00C0158700B017827D
:102B200000B0197D00D01B7800001E730040206E9D
:102B30000090226900F024640040275F0090295A29
:102B400000E02B5500102E500020304B0010324674
:102B500000E033410090353C0010373700703832C8
:102B600000A0392D00B03A2800A03B2300603C1E95
:102B700000103D1900903D1400103E0F00703E0AF9
:102B800000C03E0500003F0000403FFBFF803FF6D5
:102B9000FFC03FF1FF2020506C616E6E6572427580
:102BA0006666657242797465733A200020467265E4
:102BB00065204D656D6F72793A200020436F6D700E
:102BC000696C65643A2044656320323720323032C4
:102BD000310A00204C61737420557064617465641F
:102BE0003A20323032312D30392D3033207C2041A3
:102BF0007574686F723A20286B61642C20416E797D
:102C00006375626963204D656761205A65726F2044
:102C100041424C20313256290A004D61726C696E76
:102C200020322E302E392E332D6B6164310A002074
:102C3000536F6674776172652052657365740A001C
:102C4000205761746368646F672052657365740A06
:102C5000002042726F776E206F7574205265736525
:102C6000740A002045787465726E616C2052657339
:102C700065740A00506F77657255700A007374614D
:102C800072740A004732385859004D3130303100E3
:102C90006572726F722077726974696E6720746FE3
:102CA0002066696C650A00446F6E65207361766901
:102CB0006E672066696C652E0A004D323900456EDC
:102CC0006473746F7073002553202563202563207F
:102CD000256320256300205A3A0020593A002058E5
:102CE0003A00656E6473746F7073206869743A207B
:102CF00000000000010200090A00000000040308AF
:102D000007000000000000000000000000000000BC
:102D100000004D6F76652025736D6D004D6F7665F3
:102D200020302E316D6D004D6F766520316D6D0058
:102D30004D6F76652031306D6D004D6F76652041A9
:102D4000786973004D6F7665204578747275646597
:102D500072004D6F7665205A004D6F7665205900E0
:102D60004D6F76652058005072696E742066726FE0
:102D70006D204D6564696100FFFFFF205A3A200015
:102D800020593A200042656420583A20004D65677A
:102D900061205A65726F2052656164792E0050720D
:102DA000696E74696E672E2E2E005072696E7420E3
:102DB00050617573656400204500205A0020590059
:102DC00020204D393220580053746570732070658F
:102DD0007220756E6974003B2000220A00556E6BEC
:102DE0006E6F776E20636F6D6D616E643A202200A6
:102DF0006F6B00DB0FC93F45BCDA3F8FB30240FC6D
:102E0000F0274056946140FE4B9B4084A5D840E09B
:102E1000231841346A5641E859974164DBD5416E25
:102E2000271742B4B75542CE1A9742C8AED542B51D
:102E3000885A43D40684BFA65FA7BF7443E0BF107F
:102E4000B11AC01C2C58C0E8F697C0B849D6C04E7D
:102E50004E17C124D355C1802497C1A0B5D5C11246
:102E60001A17C244AE55C2781797C26CACD5C26768
:102E7000885AC320746F6F206C6F6E6720657874FA
:102E8000727573696F6E2070726576656E746564B5
:102E90000A0020636F6C6420657874727573696FC3
:102EA0006E2070726576656E7465640A006F6B0AD9
:102EB00000526573656E643A200020453A00205A3E
:102EC0003A0020593A00583A000000220025002814
:102ED000002B0000002100240027002A000202022B
:102EE00002020202020404040404040404030303AF
:102EF00003030303030101010101010101010204B4
:102F000008102040800102040810204080010204C3
:102F10000810204080804020100804020145727291
:102F20006F722077726974696E6720746F204545EF
:102F300050524F4D210A00005ADE75E511241FBE84
:102F4000CFEFD0E4DEBFCDBF84B78093961514BE1B
:102F50000FB6F894A8958091600088618093600016
:102F6000109260000FBE12E0A0E0B1E0E8E1F7EEE1
:102F700001E00BBF02C007900D92A239B107D9F74B
:102F800025E1A2E9B2E001C01D92A639B207E1F73E
:102F900017E1CDE9D7E104C02197FE010E94DAF0E4
:102FA000CC39D107C9F70E9429DF0C9480F30C9427
:102FB0000000A0E1B0E0EFEDF7E10C9403F18C012B
:102FC000DC01ED91FC910280F381E02DBE016F5F89
:102FD0007F4F0995882309F45DC08981807C91F534
:102FE0006F81637070E0762F6627770F770F888583
:102FF000B4E08B9FC0011124682B792B89858295C1
:10300000869586958370682B6F5F7F4F90E080E098
:103010002A852370220F3B8537FB332730F9232B7A
:103020003E813F70230F3327331F2750310904C0DF
:10303000660F771F881F991F2A95D2F76096E4E0E4
:103040000C941FF1803419F568856695669570E0DB
:1030500090E080E0CB01772766272A85622B0985DF
:1030600010E0102F0027012E000C220B330B602BD9
:10307000712B822B932B6F5F7F4F8F4F9F4F4AE0B7
:10308000660F771F881F991F4A95D1F7D7CF8BE01E
:10309000F801848360E070E0CB01D0CF0895FC019B
:1030A000828108954F925F926F927F928F929F924A
:1030B000AF92BF92CF92DF92EF92FF92CF93DF93C6
:1030C000CDB7DEB728970FB6F894DEBF0FBECDBFE1
:1030D00060913C0770913D076115710511F1809178
:1030E000380790913907A0913A07B0913B0789833F
:1030F0009A83AB83BC83072E000C880B990B0E942C
:1031000015EA29813A814B815C810E942CF14B01A7
:103110005C0120E030E040E251EC0E940FEA87FFC2
:1031200007C081E080933201C12CD12C760113C0FD
:1031300020E030E040E251E4C501B4010E9490F289
:10314000181604F581E080933201C12CD12C9FE741
:10315000E92E93E4F92EC701B60128960FB6F8942C
:10316000DEBF0FBECDBFDF91CF91FF90EF90DF901C
:10317000CF90BF90AF909F908F907F906F905F9017
:103180004F9008958091430790914407A09145077F
:10319000B09146078D839E83AF83B88780913201BB
:1031A000882391F01092960410929704109298043C
:1031B0001092990410929204109293041092940425
:1031C0001092950410923201209196043091970448
:1031D0004091980450919904C501B4010E942DF1C9
:1031E0002B013C0120E030E0A9010E9490F2C12CAB
:1031F000D12C760187FD14C02D813E814F815885E9
:1032000060E070E08FE793E40E94A4F16B017C0121
:10321000A30192010E940FEA181614F473016201CF
:10322000C0929604D0929704E0929804F092990488
:1032300020913F073091400740914107509142074C
:10324000C501B4010E9474EA4B015C0180928A04BA
:1032500090928B04A0928C04B0928D04A7019601E9
:103260006D817E818F8198850E9474EA6B017C015B
:10327000C0928E04D0928F04E0929004F092910458
:103280004090920450909304609094047090950440
:1032900029813A814B815C81609186047091870419
:1032A00080918804909189040E942CF12091470715
:1032B000309148074091490750914A070E9474EAAB
:1032C000A30192010E942CF120ED3CEC4CE45DE363
:1032D0000E9474EAA30192010E942DF19B01AC01AE
:1032E0002093920430939304409394045093950454
:1032F00089819A81AB81BC818093860490938704F5
:10330000A0938804B0938904C501B4010E942DF1F3
:10331000A70196010E942DF16B017C0120E030E0B5
:103320004FE753E40E940FEA181634F4C12CD12C55
:103330008FE7E82E83E4F82E20E030E0A901C701F2
:10334000B6010E9490F287FF06CFEECE609138075B
:103350007091390780913A0790913B070895FC01DD
:1033600090E1A5E7B4E001900D929A95E1F70895F8
:10337000EF92FF920F931F93E0928E03F0928F03D0
:103380000093900310939103B62F172F022FF32E63
:10339000242F582FB09392031093930350939403C8
:1033A0006FEFFF27B01B1F09520B30F4509510959B
:1033B000B195160B560B66276093AB04A6E0BA9F37
:1033C00000929F04712DEE271A9F700DE11D5A9FE8
:1033D000E00D7093A004E093A104AFE0BA9F0092C7
:1033E000A304712DEE271A9F700DE11D5A9FE00D69
:1033F0007093A404E093A504AAE0BA9F0092A704E6
:10340000712DEE271A9F700DE11D5A9FE00D7093EC
:10341000A804E093A9041F910F91FF90EF900895E5
:10342000A5E0B0E0E6E1FAE10C94FCF06F3671053E
:103430008105910578F4FB01EE0FFF1FEE0FFF1FD2
:10344000E959F74F65917591859194912596EBE037
:103450000C9418F1F62EE72E282FE7E6F7E0002768
:10346000BB275F2D8E2D922F992341F4982F852F06
:10347000B85F992319F4982F8827B85F903138F4F2
:1034800082959295582F5F70807F952BBC5F90340A
:1034900028F4880F991F880F991FBE5F903818F481
:1034A000880F991FB395880F991FE90FF01F54914A
:1034B00081E09927B85079F1C0F0B0FF02C0550FF4
:1034C000881FB1FF04C0550F881F550F881FB2FF1A
:1034D00006C082955295152F1F70507F812BB3FF28
:1034E0001AC0982F852F552716C0B195B0FF02C07E
:1034F00085955795B1FF04C0859557958595579546
:10350000B2FF05C08295507F5295582B8F70B3FF44
:1035100002C0582F8827BB247727AA27B2E0F59E40
:10352000B0187109A00BB00BE59E7019A109B00B82
:10353000259FA019B109F89E7019A109B00BE89E4A
:10354000A019B109289FB019F99EA019B109E99EE7
:10355000B0195B9DA12C99244427662733278B9DA6
:10356000A00C911C401F601F301F9B9D900C411DA3
:10357000601F301F579FA00C911C401F601F301F01
:10358000879F900C411D601F301F979F400D611D4C
:10359000301F5A9F900C411D601F301F8A9F400DA5
:1035A000611D301F9A9F600D311D5B9F400D611D95
:1035B000301F8B9F600D311D9B9F300DB1E0AA27FE
:1035C0007727BB24F49EB0187109A00BB00BE49EC2
:1035D0007019A109B00B249FA019B109F69E7019AA
:1035E000A109B00BE69EA019B109269FB019F39E60
:1035F000A019B109E39EB019BF187E09A20B20F0F3
:10360000B1E04B0F601F301F1124762F642F90E024
:10361000832F1CCFFC017081472F50E0062E02C083
:10362000559547950A94E2F740FF14C040910D0468
:1036300050E0062E02C0559547950A94E2F740FFE8
:1036400009C021E030E001C0220F6A95EAF7209519
:103650002723208308958F929F92AF92BF92CF929B
:10366000DF92EF92FF92FC01C080D180E280F38074
:1036700020E030E048EC52E4C701B6010E9474EA51
:103680004B015C0120E030E0A901C701B6010E94B6
:103690000FEA20E030E040EA50E487FF04C020E079
:1036A00030E040EA50ECC501B4010E942DF12DEC50
:1036B0003CEC4CEC5DE30E9474EA0E940CF29B012E
:1036C0008BE237FF05C022273327261B370B8DE2FD
:1036D00080939C02C90168EE73E00E94C7F0CB01A1
:1036E000EAE0F0E0BF010E94C7F0805D80939D0298
:1036F000C90164E670E00E94C7F0CB01BF010E94DF
:10370000C7F0805D80939E02C901BF010E94C7F08F
:103710009C01CB01BF010E94C7F0805D80939F0296
:103720008EE28093A002205D2093A1028CE992E0BA
:10373000FF90EF90DF90CF90BF90AF909F908F90D1
:1037400008954F925F926F927F928F929F92AF9265
:10375000BF92CF92DF92EF92FF92FC01C080D180A6
:10376000E280F38020E030E04AE754E4C701B6018C
:103770000E9474EA4B015C0120E030E040E251EC31
:10378000C701B6010E940FEA181654F420E030E099
:1037900048EC52E4C701B6010E9490F287FD8AC04E
:1037A00020E030E0A901C701B6010E940FEA87FFBF
:1037B00072C060E070E080EA90ECA50194010E9484
:1037C0002DF12DEC3CEC4CEC5DE30E9474EA0E9480
:1037D0000CF26B017C01F7FC63C020E137E240E0B2
:1037E00050E00E945FF0CA01B9012AE030E040E0F9
:1037F00050E00E945FF0605D60939C02C701B601DB
:1038000028EE33E040E050E00E945FF09AE0892E1D
:10381000912CA12CB12CCA01B901A50194010E94DF
:103820005FF0605D60939D02C701B60124E630E061
:1038300040E050E00E945FF0CA01B901A501940187
:103840000E945FF0605D60939E028EE280939F0213
:10385000C701B601A50194010E945FF06B01CA0186
:10386000B901A50194010E945FF0605D6093A00220
:10387000F0E3CF0EC092A1028CE992E0FF90EF90AE
:10388000DF90CF90BF90AF909F908F907F906F9080
:103890005F904F90089560E070E080EA90E48DCFF3
:1038A000F094E094D094C094C11CD11CE11CF11C94
:1038B0006DE2A2CF20E030E0A901C701B6010E946D
:1038C0000FEA87FF6BC060E070E080EA90ECA50132
:1038D00094010E942DF12DEC3CEC4CEC5DE30E9438
:1038E00074EA0E940CF24B015C0120E030E0A90177
:1038F000C701B6010E940FEA87FD0BC020E030E04F
:1039000040E251E4C701B6010E9490F260E287FDF7
:1039100013C0B7FC48C0C501B40128EE33E040E055
:1039200050E00E945FF0CA01B9012AE030E040E0B7
:1039300050E00E945FF0605D60939D02C501B4019C
:1039400024E630E040E050E00E945FF08AE0482E3C
:10395000512C612C712CCA01B901A30192010E9462
:103960005FF0605D60939E028EE280939F02C501CE
:10397000B401A30192010E945FF06B01CA01B90179
:10398000A30192010E945FF0605D6093A00280E35A
:10399000C80EC092A1028DE992E070CF60E070E0A5
:1039A00080EA90E494CFB094A09490948094811C89
:1039B000911CA11CB11C6DE2BFCF282F81E32436DE
:1039C00009F080E280939E0290E22A3040F03AE0D3
:1039D000822F632F0E949AF00E949AF0905D90933C
:1039E0009F02822F6AE00E949AF0905D9093A0025D
:1039F00085E28093A1028EE992E0089560912C0106
:103A000070912D01072E000C880B990B0E9415EA6E
:103A10002AE037ED43E25CE30E9474EA60936F01B1
:103A20007093700180937101909372010895CF9308
:103A3000DF93EC01CB01BA010E9415EA23E333E3E3
:103A400043E250E40E9474EA20E030E040E05FE3AB
:103A50000E942DF10E9411F26883DF91CF910895A9
:103A60000E9415EA23E333E343E250E40E9474EA40
:103A700020E030E040E05FE30E942DF10E9411F26F
:103A800024E6629FC001112481589F4F6FEF70E0C0
:103A90000E94C7F0862F91CF80917C07811104C0CE
:103AA000809130078093AF0708958091DB148823BD
:103AB000C1F081508093DB14E1E0F3E1882351F001
:103AC0008150990B2BE1289FF001299FF00D1124C3
:103AD000E353FC4E8BE1A6EEB2E101900D928A9584
:103AE000E1F72091DB14211105C08091E514806479
:103AF0008093E51481E090E0A0E0B0E0211103C0E4
:103B000080E090E0DC018093720790937307A093AC
:103B10007407B093750710926D0781E080936F076B
:103B200083E080936A010895CF93DF93EC01CB018A
:103B3000BA010E9415EA688379838A839B83DF91A7
:103B4000CF910895CF93DF93EC01CB01BA010E948E
:103B500015EA2DEC3CEC4CEC5DE30E9474EA6883C2
:103B600079838A839B83DF91CF910895CF93DF93ED
:103B7000EC01CB01BA010E9415EA2AE037ED43E2DD
:103B80005CE30E9474EA688379838A839B83DF9174
:103B9000CF910895CF92DF92EF92FF92CF93DF9370
:103BA00000D000D0CDB7DEB70E9415EA2AE037ED8D
:103BB00043E25CE30E9474EA6B017C0120E030E0A8
:103BC000A9010E940FEA2DEB37E346E055E387FF9A
:103BD00004C02DEB37E346E055EBC701B6010E9468
:103BE0002DF169837A838B839C83CE010196A9DDB5
:103BF0000F900F900F900F90DF91CF91FF90EF906B
:103C0000DF90CF900895CF93DF93EC01CB01BA0101
:103C10000E9415EA0E940CF279836883DF91CF91AC
:103C200008958F929F92AF92BF92CF92DF92EF92C0
:103C3000FF92FC01C080D180E280F38020E030E080
:103C4000A901C701B6010E940FEA87FD99C06DEB7B
:103C500077E386E095E3A70196010E942DF19F7717
:103C600020E030E048EC52E40E9474EA20E030E0CA
:103C700040EA50E40E942DF12DEC3CEC4CEC5DE36D
:103C80000E9474EA0E940CF26B017C0180E2809336
:103C90009B0260E2F0E1CF16F7E2DF06E104F104F7
:103CA0008CF0C701B60120E137E240E050E00E940D
:103CB0005FF0CA01B9012AE030E040E050E00E9424
:103CC0005FF0605D60939C0260E288EEC81683E05E
:103CD000D806E104F1048CF0C701B60128EE33E008
:103CE00040E050E00E945FF0CA01B9012AE030E0F4
:103CF00040E050E00E945FF0605D60939D0260E2F2
:103D0000E4E6CE16D104E104F1048CF0C701B6015B
:103D100024E630E040E050E00E945FF0CA01B901C3
:103D20002AE030E040E050E00E945FF0605D609388
:103D30009E028AE0882E912CA12CB12CC701B601DD
:103D4000A50194010E945FF06B01CA01B901A501B0
:103D500094010E945FF0605D60939F028EE2809309
:103D6000A002F0E3CF0EC092A1028BE992E0FF9097
:103D7000EF90DF90CF90BF90AF909F908F9008957D
:103D80006DEB77E386E095EB66CFA4E0B0E0EBEC7B
:103D9000FEE10C9405F10E9415EA2DEC3CEC4CEC94
:103DA0005DE30E9474EA69837A838B839C83CE01EE
:103DB000019637DF2496E2E00C9421F1CF93DF9354
:103DC000EC018D810E943F8F60E08B810E941DD0AD
:103DD000DF91CF910895CF92DF92EF92FF920F93F0
:103DE0001F93CF938C01C62F69017A01E7DF0E94F0
:103DF00096D18C2F80640E94338F8F2D0E94338F39
:103E00008E2D0E94338F8D2D0E94338F8C2D0E941A
:103E1000338F87E8C11101C085E90E94338FCC3010
:103E200011F40E94388FC0E00E94388FF801868319
:103E300087FF04C0CF3F11F0CF5FF6CFCF911F9126
:103E40000F91FF90EF90DF90CF90089561E0FC011B
:103E500083810E941DD08FEF0C94338F0F931F939B
:103E6000CF938C01ABDF0E9496D1C82F882369F0D5
:103E70008DEF0E94338F0E9496D1C82FC801E6DFD4
:103E80008C2FCF911F910F91089582E1F8018483C7
:103E9000F5CFB0E0A0E0EFE4FFE10C94FBF0EC0123
:103EA0006A017B014801590120E030E0A90167E384
:103EB00092DFA501980167E1CE018DDF81111DC060
:103EC0008F81833039F089E0CC0CDD1CEE1CFF1CA7
:103ED0008A95D1F7A701960169E1CE017CDF11E057
:103EE000882319F010E087E08C83CE01AFDF812FAB
:103EF000CDB7DEB7ECE00C9417F189E08C8310E0CD
:103F0000F4CFCF93DF93EC016EBDFA01CA019E5F3F
:103F10000DB407FEFDCF20812EBD0DB407FEFDCFF1
:103F200021812EBD3296E817F90791F70DB407FEEF
:103F3000FDCF8FEF0E94338F8FEF0E94338F0E944F
:103F4000388F8E838F71853041F083E18C83CE0171
:103F50007DDF80E0DF91CF91089581E0FBCF0F936B
:103F60001F93CF93DF93EC018B0128DF0E9496D142
:103F700081110BC085E18C8310E0CE0167DF812FBA
:103F8000DF91CF911F910F910895A8016CEFCE01A1
:103F9000B8DF182F882371F3F0CF0F931F93CF93BF
:103FA000DF93EC0189018F81833039F089E0440F80
:103FB000551F661F771F8A95D1F79A01AB0168E1FB
:103FC000CE0109DF811127C0A8016EEFCE0199DF74
:103FD000182F8823A9F00E9496D1182F8823C1F0AA
:103FE00020E030E0A9016DE0CE01F5DE882321F06C
:103FF00086E18C8310E004C00E94388F8111F8CFD5
:10400000CE0124DF812FDF91CF911F910F91089571
:1040100087E18C83F5CF86E0ECCF1F93CF93DF93BE
:10402000EC01CCDE20E030E0A9016CE0CE01D3DE73
:1040300011E0882319F010E083E08C83CE0106DFC5
:10404000812FDF91CF911F9108951F93CF93DF931D
:10405000EC018F81833039F089E0440F551F661FD2
:10406000771F8A95D1F79A01AB0162E1CE01B3DEE9
:1040700011E0882319F010E085E08C83CE01E6DEA4
:10408000812FDF91CF911F9108958F929F92AF92D0
:10409000BF92EF92FF920F931F93CF93DF938C0108
:1040A000EB017A010E9402D14B015C012CE2820EED
:1040B00021E0921EA11CB11C0E94388FF80186835A
:1040C0008F3F69F40E9402D1681979098A099B0916
:1040D00097FDF2CF81E1F8018483C0E021C08E3FDB
:1040E00069F5F1E0EF1AF1088FEF8EBDFE012FEFB9
:1040F0000DB407FEFDCF8EB581932EBDCF018C1B75
:104100009D0B8E159F05A0F30DB407FEFDCF8EB558
:10411000CE0DDF1D88830E94388F0E94388FC1E04A
:10412000C80194DE8C2FDF91CF911F910F91FF90EA
:10413000EF90BF90AF909F908F9008958FE0CBCF7E
:104140000F931F93CF93DF93EC018B0137DE40E099
:1041500052E0B801CE0199DFDF91CF911F910F910D
:1041600008950F931F93CF93DF93EC0189018F8103
:10417000833039F089E0440F551F661F771F8A95F9
:10418000D1F79A01AB0161E1CE0125DE882351F020
:1041900084E08C83CE015ADE80E0DF91CF911F91C5
:1041A0000F91089540E052E0B801CE016EDFF5CFE7
:1041B000B0E0A0E0EEEDF0E20C94FBF0EC01162F85
:1041C0001F821C824B830E9402D16B017C0120ED77
:1041D000C20E27E0D21EE11CF11CA89561E08B8184
:1041E0000E941DD08B810E94EBB5249A2C9A279AAD
:1041F0002698259A81E00E943F8F85E08D830E945A
:104200003F8F0AE08FEF0E94338F0150D9F7A895B6
:1042100020E030E0A90160E0CE01DDDD8E83813059
:1042200079F00E9402D16C197D098E099F0997FDD2
:10423000EFCF81E08C83CE0109DE1A8280E065C079
:10424000A8952AEA31E040E050E068E0CE01C3DD05
:10425000853031F581E08F83A8958F81812C912C59
:104260005401823029F4812C912CA12C80E4B82EA9
:1042700020E030E0A90167E3CE01ADDDA5019401A6
:1042800069E2CE01A8DD8E838823F1F00E9402D17D
:104290006C197D098E099F0997FDEACF8AE0CACF84
:1042A00004E00E94388F8E830150D9F78A3A11F4C6
:1042B00082E0D1CF0E9402D16C197D098E099F093D
:1042C00097FDBFCF82E0B6CF8F818230B9F420E076
:1042D00030E0A9016AE3CE017EDD882311F088E099
:1042E000A9CF0E94388F807C803C11F483E08F83BB
:1042F0000E94388F0E94388F0E94388FCE01A6DD31
:1043000081E08A83173030F41D83CDB7DEB7ECE04F
:104310000C9417F188E18C8391CF0F931F93CF9367
:10432000DF93EC018B0120E030E0A90169E053DD6F
:10433000882351F080E18C83CE0188DD80E0DF911D
:10434000CF911F910F91089540E150E0B801CE0147
:104350009CDEF5CFCF93C82FCB010E94528483EA15
:1043600096E00E94528484E996E0CC2311F089E91A
:1043700096E00E9452848AE00E943184CF91089591
:10438000EF92FF920F931F93CF937B018A01C2E4B8
:104390008F3F09F0C4E580E20E9431848C2F0E9497
:1043A00031848AE30E943184F701608171818281C6
:1043B000938142E00E940AB68CE493E10E94528409
:1043C000F801608171818281938142E00E940AB686
:1043D00062E070E080E090E00E9479D0CF911F9180
:1043E0000F91FF90EF9008950C940ED140918C03A3
:1043F00021E042276CE070E00C94BFB540918C0343
:1044000021E0422764E070E00C94BFB540918C033A
:1044100021E0422761E070E00C94BFB540918C032D
:1044200021E0422761E070E00C94BFB540918C031D
:1044300021E0422768E070E00C94BFB540918C0306
:1044400021E042276CE070E00C94BFB541E061E0F0
:1044500070E00C94BFB540918C0321E042270C948E
:10446000BFB56CE070E00C94ACD061E070E00C94EF
:10447000ACD061E070E00C94ACD06CE070E00C94D7
:10448000ACD064E070E00C94ACD09091B30281E0C9
:1044900089270C94CA7961E080E397E00C94567AFE
:1044A00020E030E0A901BC0185E791E00C94D9C679
:1044B00080E090E0A0E8B0E480937D0190937E01DD
:1044C000A0937F01B09380018AE192E0E9DF80E070
:1044D00090E0A0EFB1E48093750190937601A093F2
:1044E0007701B09378018093790190937A01A0933A
:1044F0007B01B0937C01E091EA03EE0FFF0BE650E5
:10450000FE4F808191818330910539F1843091058E
:10451000C9F1029761F480E090E0AEE3B3E48093E8
:10452000750190937601A0937701B093780182E0B2
:1045300092E0B6DF10927D0110927E0110927F0111
:10454000109280018AE192E0ABDF8091EA038F5FF5
:104550008430ECF48093EA03089580E090E0AEE3C9
:10456000B3E48093750190937601A0937701B093A3
:1045700078018093790190937A01A0937B01B093A5
:104580007C01D5CF80E090E0AEE3B3E4F2CF1092AF
:10459000EA030895A4E0B0E0E0EDF2E20C9405F146
:1045A00084EF91E0A0E0B0E089839A83AB83BC8381
:1045B000BE016F5F7F4F88E70E94F9822496E2E098
:1045C0000C9421F1B0E0A0E0E8EEF2E20C9405F1E9
:1045D00020E24F8158856E818D810E94D0CBE2E030
:1045E0000C9421F180913007909131070C9443D1C4
:1045F000609130078FEF0C944DD180913007682F78
:104600000C944DD16FEF809130070C944DD164E143
:1046100073E582E00C94DECD68E173E581E00C94F3
:10462000DECD6CE173E580E00C94DECD60E273E5F5
:1046300083E00C94DECD10926D070C942DD74FE3E0
:1046400050E064EC74E08EEE96E00C9466F380919A
:10465000671390916813891B8F7011F40C94AA7BD7
:1046600081E0089580916A01882341F06091E2031E
:104670007091E30341E081E00C9470CB08950F93B7
:104680001F93CF93DF93FC012381222331F080E03D
:10469000DF91CF911F910F9108958B01EC01FB01E8
:1046A0008789803139F582E08B831D8A1E8A1F8AB3
:1046B000188E808D918DB0E0A0E025E0880F991FC5
:1046C000AA1FBB1F2A95D1F7898B9A8BAB8BBC8B0A
:1046D0001A8F098F81E08983188619861A861B86AE
:1046E0001C821D821E821F82188A1C861D861E86C1
:1046F0001F86CECF803259F683E08B83428D538D57
:10470000648D758D4D8B5E8B6F8B788F9E012F5EC8
:104710003F4FC8010E948BD88111DACFB8CFCF9319
:10472000DF93EC010E94F4D81B82DF91CF910895B2
:10473000CF93DF93EC01462F41706C857D858E858C
:104740009F850E949DD5882351F0888920E2829F11
:10475000C001112483569F4EDF91CF91089590E0C0
:1047600080E0FACFCF93DF93EB01FC01238121118D
:1047700004C080E0DF91CF9108952250223028F4C8
:104780008FE28883198281E0F5CF60E0D1DF009766
:1047900081F3DC0160E080E09EE22D91203299F00F
:1047A000883031F49E01260F311DF90190836F5F2F
:1047B0009E01260F311DAD0141505109FA01408182
:1047C000F90140836F5F8F5F8B3039F7FE01E60F91
:1047D000F11D1082D8CFACE0B0E0E1EFF3E20C9431
:1047E000F6F05C01DC0159968D909C90F401818576
:1047F0009285A385B4859C01AD012F5F3F4F4F4F3C
:104800005F4F29873A874B875C87D50114964D9077
:104810005D906D907C901797411451046104710470
:1048200009F459C0BFEF4B1A5B0A6B0A7B0A312CA3
:10483000730162011D821E821F821886F401818528
:104840009285A385B4852D813E814F815885281797
:1048500039074A075B0708F056C089859A85AB85FA
:10486000BC858C159D05AE05BF0550F482E0C82EB1
:10487000D12CE12CF12C92E0492E512C612C712C81
:104880009E012F5F3F4FB701A601C4010E940FD8C0
:104890008823C9F189819A81AB81BC81892B8A2BBC
:1048A0008B2B01F1260137019FEF491A590A690A3A
:1048B000790A2D813E814F8158852F5F3F4F4F4FA1
:1048C0005F4F2D833E834F8358873FEFC31AD30A30
:1048D000E30AF30AB3CF40805180628073803324AF
:1048E0003394A6CFC414D504E604F70411F70FEFF0
:1048F0001FEF2FEF3FE0B701A601C4010E9495D73B
:10490000782E811106C0712C872D2C96E1E10C9434
:1049100012F1F50144815581668177814115510578
:104920006105710539F097018601C4010E9495D790
:10493000882349F3D5011496CD92DD92ED92FC9235
:104940001797332051F0D701C6010196A11DB11D63
:10495000F40180839183A283B383F50185899689CD
:10496000A789B08D892B8A2B8B2B71F6C58AD68AA5
:10497000E78AF08E818180688183C6CF40E050E075
:10498000BA010C943DD94F925F926F927F92AF9291
:10499000BF92CF92DF92EF92FF920F931F93CF932C
:1049A000DF931F92CDB7DEB78C017B015A01C22E77
:1049B000DB0159968D919C91F801928F818FCB01EB
:1049C000DDDF712CF70180859185A285B385418952
:1049D00052896389748984179507A607B70708F079
:1049E00052C055E0B695A795979587955A95D1F7FA
:1049F000F82FFF70DF2ED70113968C91823010F4C0
:104A000080E0DAC041E050E0BE016F5F7F4FC70138
:104A10000E9438DA0197A1F7F70180859185A28578
:104A2000B3854F96A11DB11D80879187A287B3875B
:104A3000F0E2DF9EB001112463567F4E61157105CF
:104A4000F9F2DB018C91882341F0853E09F04BC0DF
:104A5000772029F077247394B5CF71100EC0809120
:104A60009D1290919E12A0919F12B091A012F801F8
:104A700084879587A687B787D08ADB018C918111BF
:104A8000E9CF772473948C2D8274823409F0B8CFE7
:104A9000772009F4A1C0F801D08861E0C80148DEA0
:104AA000009709F4ADCF20E2DC011D922A95E9F7C9
:104AB0002BE0F501DC0101900D922A95E1F721E24E
:104AC00038E2FC01318B208B40E058E05787468765
:104AD000338B228B318F208F578B468B0E9454D57E
:104AE000811109C08DCF4BE050E0C5010E9416F343
:104AF000892B09F067CFF0E2DF9ED00111249D01E0
:104B000023563F4EF9018385817121F08C2D8271EE
:104B100009F000C1F801818D928D40919D12509154
:104B20009E1260919F127091A012448755876687EC
:104B30007787D08AFD01E356FF4E44885588712C53
:104B4000612C320155244424D80155964D925D9232
:104B50006D927C925897428D538D70E060E04429AD
:104B600055296629772955964D935D936D937C93CE
:104B70005897D9011B962C91287109F0BDC0848DDE
:104B8000958DA68DB78DF801818B928BA38BB48BFD
:104B900081E083838C2D8F70F801818314821582CC
:104BA00016821782108611861286138681E0C4FE53
:104BB00003C0C8010E94C2D90F90DF91CF911F910D
:104BC0000F91FF90EF90DF90CF90BF90AF907F90CC
:104BD0006F905F904F900895D70113968C91139723
:104BE000823009F40DCF51968D919D910D90BC911D
:104BF000A02D803E9F4FAF41B10508F001CFC70106
:104C0000EADD882309F4FCCE0E9454D5882309F4F8
:104C1000F7CED7015996ED91FC915A9714964D9085
:104C20005D906D907C901797B2E04B1A5108610827
:104C30007108858504C0440C551C661C771C8A9538
:104C4000D2F786859785A089B189480E591E6A1EBC
:104C50007B1E81E08093A11240929D1250929E1281
:104C600060929F127092A012EDE9F0E180E092E074
:104C7000DF019C011D9221503040E1F7DD24D394E7
:104C8000D7015996ED91FC918481D816C0F480919A
:104C9000A2129091A312DC01ED91FC910288F3899C
:104CA000E02D2DE930E1B301A2014D0D511D611D33
:104CB000711D0995882309F4A3CED394E1CF2585EE
:104CC00080E092E0A0E0B0E004C0880F991FAA1F26
:104CD000BB1F2A95D2F7F7014189528963897489EC
:104CE000840F951FA61FB71F818B928BA38BB48B4C
:104CF0008DE990E1D12CD7CE203161F498012F5E5F
:104D00003F4F0E948BD8882329F084E0D801139666
:104D10008C9340CFD80113961C9272CEFC01238154
:104D20002111FDCC0895A1E4B0E0E9E9F6E20C948C
:104D3000F5F04C015B017A01222E19821C821C8E37
:104D40001F8E6115710569F410E0CE014C96E6DF07
:104D5000CE010196E3DF812FCF5BDF4FE2E10C94C0
:104D600011F1FC0183818111EFCFFA0180818F3233
:104D700051F18B01CE0101966C012C0180E2382E9D
:104D8000360122963FAE229721963FAE21973FAE45
:104D90003EAE3DAE3CAE3BAE3AAE39AE38AE3FAACB
:104DA000970190E047E0D9018D91882309F446C02E
:104DB0008F3209F443C08E3201F54A3029F298E06F
:104DC0004AE09D01F0CFFB0183818250823098F050
:104DD000618D728DCE014C9652DC882309F4B4CFDC
:104DE0008E01045E1F4FC7017C010196F7012081EF
:104DF0002F32D1F3BFCF8B01F6CFE8E5F3E1249159
:104E0000222321F031968213FACF9ECF491708F45E
:104E10009BCF813208F498CF8F3709F495CF3FE9C3
:104E2000380F3A3108F420EEE7E3F0E0EC0FFD1F15
:104E3000E90FF11D820F80839F5FC3CF8FA980325E
:104E400009F482CF7901F90180812F5F3F4F8F32C2
:104E5000C9F38823C1F021E0AE01495C5F4FB8017E
:104E6000C60191DD882309F46FCF0A151B0511F0E7
:104E7000C80155DCCE014C964C145D0409F0C30109
:104E800086016C017ECF222DAE01495C5F4FB801D7
:104E9000C40179DD182F59CFEF92FF921F93CF9362
:104EA000DF93CDB7DEB728970FB6F894DEBF0FBEFD
:104EB000CDBF182F82EBE82E82E1F82EF701608536
:104EC0007185072E000C880B990B0E9415EA6D83E3
:104ED0007E838F839887F70184819581A681B7812E
:104EE00089839A83AB83BC83AE014B5F5F4FBE0166
:104EF0006F5F7F4F80E044DA94E3E92E97E0F92E6C
:104F0000F70160857185072E000C880B990B0E94B4
:104F100015EA6D837E838F839887F701848195815D
:104F2000A681B78189839A83AB83BC83AE014B5F33
:104F30005F4FBE016F5F7F4F8FEF22DA87E118026C
:104F4000F0011124EE54FD4E628570E084E593E19A
:104F50000E94AF8DF701628570E08FE493E10E94BB
:104F6000AF8D28960FB6F894DEBF0FBECDBFDF9190
:104F7000CF911F91FF90EF9008950F930FB70F936C
:104F800000916E000B7F00936E0078940F930BB727
:104F90000F930CB70F921F922F933F934F935F93F2
:104FA0006F937F938F939F93AF93BF93EF93FF93F1
:104FB00011240E94EC65FF91EF91BF91AF919F91F9
:104FC0008F917F916F915F914F913F912F911F90A2
:104FD0000F900CBF0F910BBF0F910460F8940093DA
:104FE0006E000F910FBF0F911895CF93DF93109222
:104FF0009C03C2EBD2E1198618860E940ED11A8654
:105000005D98C4E3D7E0198618860E94326A1A8632
:105010005C98DF91CF910895B0E0A0E0E2E1F8E282
:105020000C94FBF0B0E4A0E06A2F70E0AB014B0FF2
:10503000511D55954795411111C0E7E9FAE2659177
:105040007491072E000C880B990B0E9415EACDB7BE
:10505000DEB7ECE00C9417F1B42FE8CFA41711F0F1
:10506000B41303C0E3E9FBE2EACF9A01215031090E
:10507000220F331F220F331FF901EB56F54DE59038
:10508000F490F901E756F54DC591D4918E159F0521
:105090001CF3A42FC817D9070CF4C6CFF901E956A1
:1050A000F54D05911491F901E556F54DC590D49053
:1050B000BC016E197F09072E000C880B990B0E940A
:1050C00015EA4B015C01B601601B710B072E000C49
:1050D000880B990B0E9415EA9B01AC01C501B40134
:1050E0000E9474EA4B015C01BE016E197F09072E14
:1050F000000C880B990B0E9415EA9B01AC01C501BD
:10510000B4010E94A4F16B017C01B801012E000CD6
:10511000880B990B0E9415EA9B01AC01C701B601EF
:105120000E942DF194CFEF92FF920F931F93CF9394
:10513000DF93C82F7B018A0180912F07833090F085
:105140000E94BF8AC7010E94528482EB92E10E94B2
:105150005284CF3F79F58EEA92E10E9452848AE030
:105160000E94318442DFA8958091850481113EC060
:1051700081E08093850482E080932F0736DFD5E1BC
:10518000D150149A49F169E170E080E090E00E940A
:1051900079D0A895149868E270E080E090E00E94D1
:1051A00079D0A89568E270E080E090E00E9479D024
:1051B000A895E6CFC7FDD3CF8CEA92E10E94528436
:1051C0006C2F0C2E000C770B880B990B0E94C0B330
:1051D0008AE00E943184C3CF65EA72E1CF3F11F0CB
:1051E00069EA72E140E0C8010E94618ECDB7DEB786
:1051F000E6E00C941DF1B0E0A0E0E1E0F9E20C94EF
:10520000F7F0EC016B014A01B22EFA0140805180A7
:1052100062807380A30192016D817E818F81988568
:105220000E940FEA8823A1F04D825E826F82788609
:10523000AA24A39420E030E0A901F40160817181E7
:10524000828193810E9490F218160CF0A12CAC82FE
:105250008C818230A1F0833009F44FC08130D1F5C8
:105260002D813E814F815885F60160817181828157
:1052700093810E940FEA87FD2DC082E08C83B701E5
:105280000F2C000C880B990B0E9415EA9B01AC01B6
:105290006D817E818F8198850E942CF19B01AC01EC
:1052A000F60160817181828193810E9490F287FD75
:1052B00016C00E9402D16B017C019801A8EEB3E0F8
:1052C0000E948BF0C60ED71EE81EF91EC882D98236
:1052D000EA82FB82CDB7DEB7E0E10C9413F10E94C5
:1052E00002D1088119812A813B81601B710B820BDD
:1052F000930B97FDEFCF83E08C834CE253E16CE39B
:1053000073E18B2D10DFE6CF40ED52E16DED72E1E0
:105310000ACFCF93DF93A8958091B4129091B512E4
:105320000E9438B56093B6127093B7128093B8128A
:105330009093B91280913607909137076DDE609394
:1053400038077093390780933A0790933B07C091D1
:10535000B412D091B5128091630190916401C81785
:10536000D90714F480E0D0DF8091BA129091BB127B
:10537000181619066CF480916101909162018C17E6
:105380009D0734F44DE053E16AE173E180E0CBDE48
:1053900020913607309137078091E5069091E60617
:1053A0002817390714F48FEFAFDF80913C079091F5
:1053B0003D07181619068CF42091360730913707EF
:1053C00080915F01909160018217930734F44DE062
:1053D00053E16AE173E18FEFA6DEDF91CF9108958B
:1053E000A4E0B0E0E6EFF9E20C94FBF080912F0727
:1053F000811106C0A8952496ECE00C9417F128C101
:1054000080919A048111F7CF81E080939A04809172
:105410009D03811107C010929A042496ECE00C942D
:1054200017F116C176DF10929D030E9402D14B0145
:105430005C010E94DBB36B017C016091670170919C
:105440006801072E000C880B990B0E9415EA9B013E
:10545000AC01C701B6010E9490F218160CF4E7C027
:105460006091BA127091BB12072E000C880B990B39
:105470000E9415EA69837A838B839C8334E0E32E50
:10548000F12C08E210E020E0AE014F5F5F4F66EBC9
:1054900072E18CE193E1AFDEC090B612D090B7120A
:1054A000E090B812F090B9126091650170916601B8
:1054B000072E000C880B990B0E9415EA9B01AC018A
:1054C000C701B6010E9490F21816CCF460916701F2
:1054D00070916801072E000C880B990B0E9415EA49
:1054E0009B01AC01C701B6010E940FEA87FF07C00C
:1054F0000E94E4B30E940CF27595679501C060E0CC
:105500006093BC128091AE129091AF12A091B01234
:10551000B091B1120097A105B105C1F0A5019401A8
:10552000281B390B4A0B5B0BDA01C901B7FD0EC012
:105530000E94DBB30E940CF22091AC123091AD12AC
:10554000621773070CF47DC00E940ED10E94A61949
:1055500020E030E04AEF52E40E9490F218160CF47A
:1055600063C08091980390919903A0919A03B091A0
:105570009B030097A105B105A1F0881A990AAA0A10
:10558000BB0AB7FC0EC00E94A6190E940CF2209123
:10559000960330919703621773070CF44BC00E9477
:1055A000326A60913C0770913D07072E000C880B12
:1055B000990B0E9415EA69837A838B839C8392E01E
:1055C000E92EF12C04E110E02FEFAE014F5F5F4FA9
:1055D00068E377E085E293E10EDE809038079090F3
:1055E0003907A0903A07B0903B0720E030E040EA4E
:1055F00050E4C501B4010E9490F287FD11C020E083
:1056000030E04AEF52E4C501B4010E940FEA1816D7
:105610003CF00E9452180E940CF27595679501C0EB
:1056200060E060933E07F7CE8FEF6EDE9ACF80E0AA
:105630006BDE16CF4FEE52E16EEF72E18FEF73DD4E
:10564000B0CF4FEE52E16EEF72E180E06CDD7ECFC5
:10565000CF92DF92EF92FF92CF93DF93EC01C8805D
:10566000D980EA80FB808BE992E10E945284C701D5
:10567000B6010E941776CC80DD80EE80FF8082EC40
:105680009EE20E945284C701B6010E941776C88428
:10569000D984EA84FB848EEB9EE20E945284C70187
:1056A000B6010E9417768AE00E943184DF91CF9183
:1056B000FF90EF90DF90CF900895BC012091660499
:1056C00030916704409166045091670424173507B0
:1056D00031F481E02617370709F080E008959A0138
:1056E000F1CF0F930FB70F9300916E000F930B7FC5
:1056F00000936E0000916F000D7F00936F000F9379
:105700000BB70F930CB70F921F922F933F934F93AA
:105710005F936F937F938F939F93AF93BF93EF9319
:10572000FF931124E1D4FF91EF91BF91AF919F912D
:105730008F917F916F915F914F913F912F911F902A
:105740000F900CBF0F910BBF0F910260F894009364
:105750006F000F9100936E000F910FBF0F9118957E
:1057600000C000C08091E90680FF1FC0459A8FEFFE
:1057700080931F048091E90681FF1AC0479A8FEF3A
:10578000809320048091E90682FF15C02A988FEF4C
:10579000809321048091E90683FF10C028988FEF41
:1057A0008093220400C000C00895459881E0E0CFB6
:1057B000479881E0E5CF2A9A81E0EACF289A81E0F4
:1057C000EFCF80918D03982F977F90938D03982F23
:1057D000937081E011F080E008955E9A08955E98DC
:1057E00080918D03886080938D030895E82FF0E009
:1057F00021E030E0082E02C0220F331F0A94E2F7A6
:105800002095309590918D03922390938D03EA50CB
:10581000FE4F2081922321E019F020E0822F08958D
:10582000813079F038F08230C9F7159A90917F076E
:105830009B7F04C05E9A90917F079E7F90937F0725
:10584000EDCF5E9A90917F079D7FF8CF80E0CEDF0D
:1058500081E0CCDF82E0CADFB4CF813079F070F034
:10586000823071F021E030E001C0220F8A95EAF722
:1058700080918D03822B80938D0308955E98F2CFE3
:105880001598F0CFB0E0A0E0E8E4FCE20C94FDF065
:10589000C1E7DDE007E917E081E8A82E8DE0B82E2A
:1058A000C12CD12C7601C3946991799189919991F8
:1058B0000E9413EA288939894A895B890E9474EA1F
:1058C0000E9411F2F80161937193819391938F017A
:1058D000C616D706E806F90610F46B017C01AC1673
:1058E000BD0611F76FEF7FEFCB01A70196010E9474
:1058F0003DF02093A7073093A8074093A907509342
:10590000AA07CDB7DEB7EAE00C9419F10F931F9305
:10591000CF93DF9305E81DE0C0EBD7E0F8012191BC
:105920003191419151918F0160E070E080E89FE3F7
:105930000E94A4F16993799389939993F7E0C03C0D
:10594000DF0761F70E94FCC69DDFDF91CF911F91B9
:105950000F910895DBCFDACFD9CFD8CF90916713CD
:1059600080916813981306C08091B90D9091BA0D7B
:10597000892B21F080E00E94508FF0CF0895909104
:10598000671380916813981307C08091B90D9091A7
:10599000BA0D892B09F45ACF80E00E94508FEFCFC7
:1059A000CF92DF92EF92FF92CF93DF932091B302D9
:1059B000222319F1EC0108960E947B776B017C0190
:1059C00020E030E0A9010E940FEA20E030E0A901C8
:1059D000882349F0CE010E94F377A70196010E9427
:1059E00074EA9B01AC01688579858A859B850E9454
:1059F0002CF1688779878A879B87DF91CF91FF9009
:105A0000EF90DF90CF900895CF92DF92EF92FF92C8
:105A1000CF93DF932091B302222319F1EC01089672
:105A20000E947B776B017C0120E030E0A9010E949D
:105A30000FEA20E030E0A901882349F0CE010E945E
:105A4000F377A70196010E9474EA9B01AC01688577
:105A500079858A859B850E942DF1688779878A8759
:105A60009B87DF91CF91FF90EF90DF90CF900895CB
:105A7000AEE1B0E0EEE3FDE20C94F7F09E8F8D8F87
:105A80005B018A01FC01EA5BFF4F20813181428189
:105A90005381298B3A8B4B8B5C8BCA01B9010E94D5
:105AA00013EA6B017C01D5012D913D914D915C91E3
:105AB0000E9474EA0E9491F12B013C01F8012081BF
:105AC000318142815381C701B6010E9474EA0E946C
:105AD00091F14B015C01C301B2010E9411F26D8B87
:105AE0007E8B8F8B988F683771058105910540F407
:105AF00028E730E040E050E02D8B3E8B4F8B588FF5
:105B0000C501B4010E9411F2698F7A8F8B8F9C8F2F
:105B1000683771058105910540F488E790E0A0E0C1
:105B2000B0E0898F9A8FAB8FBC8FED8DFE8DEE5AD2
:105B3000FF4F208131814281538129873A874B87EA
:105B40005C87CA01B9010E9415EA2B013C016D89ED
:105B50007E898F89988D0E9413EA6D837E838F835F
:105B6000988720E030E0A901C301B2010E940FEA4A
:105B7000882309F4BBC1A7019601C701B6010E94A1
:105B800074EA4B015C012D813E814F815885CA0129
:105B9000B9010E9474EA9B01AC01C501B4010E94E5
:105BA0002CF14B015C01A3019201C301B2010E94DF
:105BB0002DF19B01AC01C501B4010E94A4F10E942A
:105BC00091F10E9411F269837A838B839C836985AA
:105BD0007A858B859C8590958095709561957F4F92
:105BE0008F4F9F4F0E9415EA4B015C01698D7A8DA2
:105BF0008B8D9C8D0E9413EA69877A878B879C879F
:105C000020E030E0A901C501B4010E940FEA882319
:105C100009F470C129853A854B855C85CA01B901B3
:105C20000E9474EA6D877E878F87988BA701960103
:105C3000C701B6010E9474EA9B01AC016D857E85A7
:105C40008F8598890E942CF16B017C01A50194013C
:105C5000C501B4010E942DF19B01AC01C701B60141
:105C60000E94A4F10E943DF2AD8DBE8D95962D91BE
:105C70003D914D915C9198972D873E874F87588B2A
:105C800069017A0129813A814B815C81C21AD30A68
:105C9000E40AF50A0E9411F2C61AD70AE80AF90ABC
:105CA000F7FE8CC02D813E814F815885CA01B90114
:105CB0000E9474EA6B017C0120E030E0A901C3017D
:105CC000B2010E940FEA882309F418C16D857E8510
:105CD0008F8598890E9413EA9B01AC010E942DF1E7
:105CE000A30192010E9474EA4B015C0129853A8567
:105CF0004B855C85CA01B9010E9474EA9B01AC0125
:105D0000C501B4010E942DF1A70196010E942CF15A
:105D10004B015C0120E030E040E850E4C301B201F7
:105D20000E9474EA9B01AC01C501B4010E94A4F178
:105D30000E9491F14B015C0120E030E0A9010E943A
:105D400090F287FF03C0812C912C5401C501B4014E
:105D50000E9411F269837A838B839C832D853E8513
:105D60004F855889261737074807590720F4298394
:105D70003A834B835C8369817A818B819C810E9409
:105D800013EA4B015C01A3019201C301B2010E941D
:105D90002DF19B01AC01C501B4010E9474EAA70179
:105DA00096010E942DF10E94C9F20E9411F2698BA6
:105DB0007A8B8B8B9C8BC12CD12C760169897A894B
:105DC0008B899C892D893E894F89588D621B730B65
:105DD000840B950B0E9413EAA30192010E94A4F187
:105DE00020E034E244EF59E40E9474EA0E9411F288
:105DF0004B015C0169897A898B899C89298D3A8D4F
:105E00004B8D5C8D621B730B840B950B0E9413EA08
:105E1000A30192010E94A4F120E034E244EF59E48E
:105E20000E9474EA0E9411F26D837E838F839887AB
:105E3000C501B4010E94101A2B013C016D817E81C5
:105E40008F8198850E94101A29813A814B815C814B
:105E5000AD8DBE8D99962D933D934D935C939C97FC
:105E600089019A010C0D1D1D2E1D3F1DFD0105A769
:105E700016A727A730ABE65BFF4F2D893E894F89D8
:105E8000588D2083318342835383D5968D929D9282
:105E9000AD92BC92D8972D813E814F815885D9967D
:105EA0002D933D934D935C93DC973D9740825182B7
:105EB000628273823496608371838283938329899B
:105EC0003A894B895C89D1962D933D934D935C9390
:105ED000D4973D96298D3A8D4B8D5C8D20833183EF
:105EE000428353836E96E0E10C9413F160E070E01E
:105EF000CB0165CE60E070E0CB01B4CE60E070E035
:105F0000CB0116CF90916F0081E091FD02C080E03F
:105F1000089590916F009D7F90936F000895EFE634
:105F2000F0E08081826080830895CF93C82FEADFFC
:105F300094E0C99F90011124F901E759FB4F2B58B8
:105F40003B4FD9014D915D916D917C91408351837F
:105F50006283738391E0909368048111E0DFCF91B5
:105F60000895CF93DF938091E806811105C0809159
:105F7000EA06882309F44EC08091FA03329B4DC093
:105F800081608093FA038091FA03339B48C082605A
:105F90008093FA038091FA03349B43C0846080931A
:105FA000FA03C0915904C0FF0FC08091E90680FF39
:105FB0000BC08091FA0380FF07C080912E0781609B
:105FC00080932E0780E0B1DFC1FF0FC08091E9060A
:105FD00081FF0BC08091FA0381FF07C080912E07DB
:105FE000826080932E0781E0A0DFC2FF13C0809102
:105FF000E90682FF0FC08091EA06882359F080915C
:10600000FA0382FF07C080912E07846080932E07D9
:1060100082E08BDFDF91CF9108958E7FB2CF8D7FAD
:10602000B7CF8B7FBCCF6EDF1092AB071092AC075F
:106030001092AD071092AE07811171CF08950F93A2
:106040001F938091671390916813891B8F7009F4D7
:1060500049C090916413992361F0833040F48FEF2D
:10606000890F29F08093641390E080E038C010928B
:106070006413809168132BE5829FC0011124805422
:10608000984FFC01208120FDEFCF4091AB0750914C
:10609000AC076091AD077091AE07E95AFF4F0081E0
:1060A000118122813381401B510B620B730B409392
:1060B000AB075093AC076093AD077093AE07209188
:1060C00068132F5F2F702093651330916813209110
:1060D0006613321304C020916513209366131F9139
:1060E0000F910895A0DFC0CFA3E1B0E0EAE7F0E3AD
:1060F0000C94F5F08FEF9FEF9093890080938800C8
:106100002AE02983312C212C78948091620490918B
:106110006304A0916404B0916504892B8A2B8B2BB6
:1061200009F0C2C1809168048823D1F0809166048F
:106130009091670410926804892B91F01092670483
:10614000109266041092590490916713809168131D
:10615000981731F0809168138F5F8F708093681368
:106160008091660490916704892B09F49DC1409148
:106170005E0450915F0460916004709161048091AD
:106180005A0490915B04A0915C04B0915D0400916D
:10619000500410E030E020E0841B950BA60BB70BF9
:1061A000081719072A073B0710F4D901C8018A8B81
:1061B000840F951FA61FB71F80935E0490935F0402
:1061C000A0936004B0936104E1E0C0902704D090F4
:1061D0002804E0902904F0902A04809137049091DB
:1061E0003804A0913904B0913A04C80ED91EEA1EB1
:1061F000FB1EC0923704D0923804E0923904F0922A
:106200003A04F7FC33C040911F04042E000C550BD8
:10621000660B770B8091750490917604A0917704BA
:10622000B0917804840F951FA61FB71F8093750443
:1062300090937604A0937704B0937804809123041C
:1062400090912404A0912504B0912604B701A601E1
:10625000481B590B6A0B7B0BDB01CA018093370487
:1062600090933804A0933904B0933A0400912B041E
:1062700010912C0420912D0430912E0480913B0428
:1062800090913C04A0913D04B0913E04080F191F69
:106290002A1F3B1F00933B0410933C0420933D04B2
:1062A00030933E0437FD33C040912004042E000C8F
:1062B000550B660B770B8091790490917A04A0912D
:1062C0007B04B0917C04840F951FA61FB71F809399
:1062D000790490937A04A0937B04B0937C0480911A
:1062E000230490912404A0912504B0912604280150
:1062F0003901481A590A6A0A7B0AD301C2018093FC
:106300003B0490933C04A0933D04B0933E04409121
:106310002F045091300460913104709132048091C7
:106320003F0490914004A0914104B0914204480F71
:10633000591F6A1F7B1F40933F0450934004609392
:1063400041047093420477FD33C080902104082CEF
:10635000000C9908AA08BB0880917D0490917E04E6
:10636000A0917F04B0918004880D991DAA1DBB1DCA
:1063700080937D0490937E04A0937F04B093800467
:106380008091230490912404A0912504B0912604C7
:106390003A014B01681A790A8A0A9B0AD401C3019F
:1063A00080933F0490934004A0934104B09342042F
:1063B0008090330490903404A0903504B09036045B
:1063C0008091430490914404A0914504B091460407
:1063D000880D991DAA1DBB1D80934304909344040E
:1063E000A0934504B0934604B7FD33C04090220407
:1063F000042C000C55086608770880908104909062
:106400008204A0908304B0908404840C951CA61C84
:10641000B71C8092810490928204A0928304B0926F
:1064200084048090230490902404A0902504B090CC
:1064300026042C013D01481859086A087B085301BD
:1064400042018092430490924404A0924504B09289
:106450004604E11104C0E0918400F0918500F7FE4C
:106460005F9A37FF469A77FF2B9AB7FF299AE091F8
:106470008400F0918500E0918400F0918500F7FEA2
:106480005F9837FF469877FF2B98B7FF29985A886F
:10649000552021F080918400909185002A89215017
:1064A0002A8BE0E0211191CE8091620490916304E7
:1064B000A0916404B0916504892B8A2B8B2B09F081
:1064C000B0C640906604509067045B8A4A8A4114C3
:1064D000510409F402C780915E0490915F04A09179
:1064E0006004B091610440915A0450915B04609142
:1064F0005C0470915D0484179507A607B70708F43C
:1065000049C0109267041092660410925904909149
:10651000671380916813981709F4DFC68091681398
:106520008F5F8F7080936813A0EDCA2EA7E0DA2EDC
:10653000E12CF12C8091660490916704892B09F07D
:1065400068C67DDD9093670480936604892B09F407
:1065500060C640906604509067045B8A4A8AD20104
:106560008C9183FF08C5C20145960E94AF19109215
:1065700067041092660410925904909167138091F9
:1065800068139817F1F2809168138F5F8F70809372
:106590006813D7CF40915504509156046091570429
:1065A00070915804481759076A077B0708F40FC20F
:1065B00040915104509152046091530470915404DD
:1065C000EA89FB8985A996A9A7A9B0AD48175907FB
:1065D0006A077B0708F0D0C14115510561057105B7
:1065E00009F066C08090920390909303A09094036A
:1065F000B09095038BE792E1A1E0FC010591159124
:1066000025913491081519052A053B0558F4B694CF
:10661000A79497948794AA0F0496E7E9F2E1E81704
:10662000F90759F7A0935004F0E28F169104A104E2
:10663000B10428F4E0E28E2E912CA12CB12C20E2A2
:10664000821A9108A108B108811438E09306A104C8
:10665000B10408F49AC1A4E09A9EC001112485589F
:10666000914FFC01329625913491B82DEE27B39FBE
:106670008001B29F010D1E1F06940E1F1E1F1124C4
:1066800030E020E0FC01C590D490F12CE12CC01A40
:10669000D10AE20AF30A4C0D5D1D6E1D7F1D409369
:1066A000510450935204609353047093540442CFA6
:1066B00010E00A81942F852E862FBC81AD81FE814A
:1066C000EF81388529854B80E0918E03E99FA12DCC
:1066D000FF2730918F03399FA00DF11D109090037B
:1066E000199EF00DE89DA00DF11D389DF00DE89F5D
:1066F000F00D4A2EBF2F4A9EE12D332722274F9EB1
:10670000E00D311D211FBA9FE00D311D211FBF9FDC
:10671000300D211D432EB22F4A9E012D33272227F3
:106720004F9E000D311D211FBA9F000D311D211FED
:10673000BF9F300D211D432EB22FEE279091920363
:1067400080909303809194030090AB04012A09F494
:1067500083C03091A704349DE119910B810A810B0C
:106760002091A804249DE0199109810A810B0091D0
:10677000A904049D90198108810B3B9FE0199109A0
:10678000810A810B2B9F90198108810B0B9F801828
:1067900081094A9E012D332722274F9E000D311D6E
:1067A000211FBA9F000D311D211FBF9F300D211DDC
:1067B000432EB22F3091A304349DE10D911F811E11
:1067C000811F2091A404249DE00D911D811E811F35
:1067D0000091A504049D900D811C811F3B9FE00D3D
:1067E000911D811E811F2B9F900D811C811F0B9F6E
:1067F000800C811D4A9E012D332722274F9E000DBC
:10680000311D211FBA9F000D311D211FBF9F300D6B
:10681000211D432EB22F30919F04349DE119910B1D
:10682000810A810B2091A004249DE0199109810A1D
:10683000810B0091A104049D90198108810B3B9F5D
:10684000E0199109810A810B2B9F90198108810B16
:106850000B9F8018810982C03091A704349DE10DFF
:10686000911F811E811F2091A804249DE00D911D80
:10687000811E811F0091A904049D900D811C811F20
:106880003B9FE00D911D811E811F2B9F900D811C50
:10689000811F0B9F800C811D4A9E012D33272227CB
:1068A0004F9E000D311D211FBA9F000D311D211F6C
:1068B000BF9F300D211D432EB22F3091A304349D74
:1068C000E119910B810A810B2091A404249DE01908
:1068D0009109810A810B0091A504049D90198108FA
:1068E000810B3B9FE0199109810A810B2B9F901925
:1068F0008108810B0B9F801881094A9E012D332747
:1069000022274F9E000D311D211FBA9F000D311D02
:10691000211FBF9F300D211D432EB22F30919F04A8
:10692000349DE10D911F811E811F2091A004249DA3
:10693000E00D911D811E811F0091A104049D900D09
:10694000811C811F3B9FE00D911D811E811F2B9F8C
:10695000900D811C811F0B9F800C811D11244B8287
:106960000A83BC83AD83FE83EF8338872987982C05
:10697000892EB12CA82E3ECEAA89BB89D1968D90A6
:106980009D90AD90BC90D49735CED501C401B695FD
:10699000A795979587958C7F8558954FFC01C59055
:1069A000D490FC01329625913491E82DE7708E2E1B
:1069B000E29FC001E39F900D112433E096958795E7
:1069C0003A95E1F7C81AD90AF12CE12C64CE40912E
:1069D0004C0450914D0460914E0470914F0448173F
:1069E00059076A077B0708F030C2809047049090EF
:1069F0004804A0904904B0904A0480914B04EA896D
:106A0000FB8981117CC0EF5BFF4FE080F180028148
:106A10001381EA89FB89E25BFF4F2081318142814A
:106A20005381AA89BB89D1966D917D918D919C915D
:106A3000D4970E94B819B1E0B0934B04EA89FB895E
:106A400041A952A963A974A98BE792E1A1E0FC01D5
:106A500005911591259134910417150726073707DD
:106A600058F47695679557954795AA0F0496E7E9E8
:106A7000F2E1E817F90759F7A093500440325105A5
:106A80006105710520F440E250E060E070E04052A2
:106A90005109610971094115F8E05F076105710548
:106AA00008F4B3C124E0529FC00111248558914FCE
:106AB000FC01329625913491AA27439FF001429F11
:106AC000E10DFA1F0694EA1FFA1F1124AF0170E0CE
:106AD00060E0FC01C590D490F12CE12CC41AD50AD9
:106AE000E60AF70A8C0C9D1CAE1CBF1C8092470462
:106AF00090924804A0924904B0924A041BCD81AD03
:106B000092ADA3ADB4AD88169906AA06BB0608F0EF
:106B100072C181149104A104B10449F4409192031B
:106B20005091930360919403709195038DCFA0E0F1
:106B3000BA85982D492D8A2DFB85EC857D856E853E
:106B40005F853889298950918E03599F712D662759
:106B500030918F03399F700D611D10909003199E25
:106B6000600D549F700D611D349F600D589F600D26
:106B7000F72FE62FF79F512D33272227F69F500D31
:106B8000311D2A1FE79F500D311D2A1FE69F300D32
:106B9000211DF32FE22FF79FB12D33272227F69FD8
:106BA000B00D311D2A1FE79FB00D311D2A1FE69F32
:106BB000300D211DF32FE22F552790919203409124
:106BC0009303809194030090AB040A2A09F483C0D4
:106BD0003091A7043F9F51199A0B4A0B8A0B2091C1
:106BE000A8042F9F501991094A0B8A0BB091A90450
:106BF000BF9F901941098A0B3E9F501991094A0B7A
:106C00008A0B2E9F901941098A0BBE9F401981095A
:106C1000F79FB12D33272227F69FB00D311D2A1F74
:106C2000E79FB00D311D2A1FE69F300D211DF32F68
:106C3000E22F3091A3043F9F510D9A1F4A1F8A1FD4
:106C40002091A4042F9F500D911D4A1F8A1FB091BF
:106C5000A504BF9F900D411D8A1F3E9F500D911DA1
:106C60004A1F8A1F2E9F900D411D8A1FBE9F400DF7
:106C7000811DF79FB12D33272227F69FB00D311DBF
:106C80002A1FE79FB00D311D2A1FE69F300D211DE1
:106C9000F32FE22F30919F043F9F51199A0B4A0B1B
:106CA0008A0B2091A0042F9F501991094A0B8A0B3F
:106CB000B091A104BF9F901941098A0B3E9F5019C2
:106CC00091094A0B8A0B2E9F901941098A0BBE9F8E
:106CD0004019810982C03091A7043F9F510D9A1F2E
:106CE0004A1F8A1F2091A8042F9F500D911D4A1FF3
:106CF0008A1FB091A904BF9F900D411D8A1F3E9F1E
:106D0000500D911D4A1F8A1F2E9F900D411D8A1FF5
:106D1000BE9F400D811DF79FB12D33272227F69F7F
:106D2000B00D311D2A1FE79FB00D311D2A1FE69FB0
:106D3000300D211DF32FE22F3091A3043F9F5119F5
:106D40009A0B4A0B8A0B2091A4042F9F501991098A
:106D50004A0B8A0BB091A504BF9F901941098A0B79
:106D60003E9F501991094A0B8A0B2E9F9019410999
:106D70008A0BBE9F40198109F79FB12D3327222727
:106D8000F69FB00D311D2A1FE79FB00D311D2A1F40
:106D9000E69F300D211DF32FE22F30919F043F9F7E
:106DA000510D9A1F4A1F8A1F2091A0042F9F500D3A
:106DB000911D4A1F8A1FB091A104BF9F900D411DD4
:106DC0008A1F3E9F500D911D4A1F8A1F2E9F900DB6
:106DD000411D8A1FBE9F400D811D1124BA87FB876C
:106DE000EC877D876E875F87388B298B542F492FDF
:106DF00070E0682F29CE2A893B89225B3F4FD90159
:106E00004D915D916D917C911FCEDB01CA01B695CC
:106E1000A795979587958C7F8558954FFC01C590D0
:106E2000D490FC013296259134914770429FC00165
:106E3000439F900D1124A3E096958795AA95E1F7BD
:106E4000C81AD90AF12CE12C4DCE80912E019091D7
:106E50002F01A0913001B0913101B7FF61C0EA89E3
:106E6000FB89EA5BFF4FC080D180E280F3808BE733
:106E700092E121E0FC0145915591659174914C1589
:106E80005D056E057F0558F4F694E794D794C79492
:106E9000220F049647E952E14817590759F7209302
:106EA000500450E2C516D104E104F10428F470E264
:106EB000C72ED12CE12CF12C60E2C61AD108E108D2
:106EC000F108C11478E0D706E104F10408F431C0F8
:106ED000A4E0DA9EC00111248558914FFC0132963E
:106EE00025913491BC2D6627B39FA001B29F410D1F
:106EF000561F0694461F561F112470E060E0FC01E7
:106F000085919491B0E0A0E0841B950BA60BB70B84
:106F100080932E0190932F01A0933001B093310103
:106F2000C0902E01D0902F01E0903001F0903101FF
:106F300001CBD701C601B695A795979587958C7F0C
:106F40008558954FFC0125913491FC01329645916D
:106F50005491EC2DE770E49FC001E59F900D112442
:106F600063E0969587956A95E1F7281B390BC9016F
:106F7000B0E0A0E0CDCFEA89FB8985889688A78814
:106F8000B08C81E081149104A104B10409F480E083
:106F9000AA89BB895996CD90DD90ED90FC905C97C5
:106FA000C114D104E104F10409F08260EA89FB898B
:106FB000458D568D678D70A141155105610571058F
:106FC00009F0846080935904109247041092480499
:106FD0001092490410924A041092510410925204E3
:106FE0001092530410925404EA89FB8985A196A15A
:106FF000A7A1B0A580935A0490935B04A0935C046E
:10700000B0935D04442455243201481A590A6A0A8F
:107010007B0A40923704509238046092390470928F
:107020003A0440923B0450923C0460923D047092BA
:107030003E0440923F04509240046092410470929A
:10704000420441A052A063A074A0440C551C661CCD
:10705000771C880C991CAA1CBB1C80922704909258
:107060002804A0922904B0922A04CC0CDD1CEE1C4A
:10707000FF1CC0922B04D0922C04E0922D04F092BD
:107080002E04440F551F661F771F40932F04509303
:107090003004609331047093320440923304509270
:1070A00034046092350470923604880F991FAA1F29
:1070B000BB1F8093230490932404A0932504B093D2
:1070C000260410925E0410925F04109260041092E5
:1070D000610481A592A5A3A5B4A5809355049093BE
:1070E0005604A0935704B093580485A596A5A7A568
:1070F000B0A980934C0490934D04A0934E04B09398
:107100004F04EB5BFF4F80819091E906891721F0D6
:107110008093E9060E94B02B0E94B12F44244A9428
:10712000542C320140922E0150922F016092300176
:1071300070923101EA89FB89FD96E080F18002813D
:107140001381AA89BB89D1962D913D914D915C9176
:10715000D4976D01BAE4CB0ED11CF6016081718128
:10716000828193810E94B81910924B04D6014D91EF
:107170005D916D917C918BE792E1A1E0FC0105911D
:10718000159125913491041715072607370758F4F0
:107190007695679557954795AA0F0496E7E9F2E12A
:1071A000E817F90759F7A0935004403251056105DB
:1071B000710520F440E250E060E070E04052510977
:1071C000610971094115F8E05F076105710508F46F
:1071D00062C024E0529FC00111248558914FFC01E8
:1071E000329625913491AA27439FF001429FE10DE9
:1071F000FA1F0694EA1FFA1F1124AF0170E060E045
:10720000FC01C590D490F12CE12CC41AD50AE60AF1
:10721000F70AC0926204D0926304E0926404F09290
:1072200065048091620490916304A0916404B0911C
:107230006504AC01BD01009731E0A307B10520F062
:107240004FEF5FEF60E070E0841B950BA60BB70B70
:107250008093620490936304A0936404B0936504E4
:10726000F89480918400909185004096A981A15066
:10727000A983AA2381F1240E351E2816390610F49D
:107280000C94843030928900209288007894639620
:10729000E2E10C9411F1DB01CA01B695A79597952F
:1072A00087958C7F8558954FFC01C590D490FC0143
:1072B0003296259134914770429FC001439F900DB3
:1072C000112433E0969587953A95E1F7C81AD90AC3
:1072D000F12CE12C9ECF1C01D5CF80EDC82E87E08C
:1072E000D82EE12CF12C2DC9CF93DF938091671319
:1072F00090916813891B80958F7019F40E94508FAC
:10730000F5CF809167138F5F8F70A09167139BE516
:10731000A99FD0011124FD01E054F84FEF0119920B
:107320009A95E9F798E09083AB52B84F90E1E9E67F
:10733000F3E101900D929A95E1F7209167139091F6
:107340006813291303C094E6909364138093671322
:107350000E948F2FDF91CF910895FC012081318110
:10736000428153816091910D7091920D8091930DA6
:107370009091940D0E9474EA0E9495F260937513A7
:10738000709376138093771390937813909167138B
:1073900080916813981709F0A7CF0E94AE2C0E9425
:1073A000822F4091751350917613609177137091ED
:1073B0007813409381045093820460938304709304
:1073C000840481110C948F2F08954F925F926F92D5
:1073D0007F928F929F92AF92BF92CF92DF92EF9265
:1073E000FF92CF93DF93EC012091910D3091920D9C
:1073F0004091930D5091940D6C857D858E859F8570
:107400000E9474EA0E9495F26B017C0120918D0D1F
:1074100030918E0D40918F0D5091900D688579853A
:107420008A859B850E9474EA0E9495F24B015C015B
:107430002091890D30918A0D40918B0D50918C0DCA
:107440006C817D818E819F810E9474EA0E9495F2F9
:107450002B013C012091850D3091860D4091870DC7
:107460005091880D688179818A819B810E9474EA9C
:107470000E9495F26093691370936A1380936B1363
:1074800090936C1340926D1350926E1360926F1331
:10749000709270138092711390927213A092731372
:1074A000B0927413C0927513D0927613E092771352
:1074B000F09278139091671380916813981781F078
:1074C00013DFDF91CF91FF90EF90DF90CF90BF90CF
:1074D000AF909F908F907F906F905F904F900895A6
:1074E0000E94AE2C0E94822FC82F89E693E10E9451
:1074F000AF19CC2331F30E948F2FE3CFCF92DF92CD
:10750000EF92FF92CF93DF93C82F0E94822F94E0D7
:10751000C99FE0011124FE01EB58FB4FC080D180D0
:10752000E280F38081110E948F2FC055D84FC70190
:10753000B6010E9415EA288139814A815B810E9447
:1075400074EADF91CF91FF90EF90DF90CF90089594
:107550008F929F92AF92BF92CF92DF92EF92FF9263
:107560001F93CF93DF93CDB7DEB760970FB6F89434
:10757000DEBF0FBECDBF182F80E0C0DF4B015C0126
:107580008092FB039092FC03A092FD03B092FE0355
:1075900081E0B4DF6B017C01C092FF03D092000454
:1075A000E0920104F092020482E0A8DF60930304F9
:1075B0007093040480930504909306041D861E8630
:1075C0001F86188A89829A82AB82BC82CD82DE8233
:1075D000EF82F88669877A878B879C8783E08EDFC6
:1075E0006D877E878F87988BCE0101960E94D02C65
:1075F0001E3FD9F480E1FE013196A5E7B1E001908C
:107600000D928A95E1F760960FB6F894DEBF0FBE33
:10761000CDBFDF91CF911F91FF90EF90DF90CF9082
:10762000BF90AF909F908F90089584E0189FF001D5
:107630001124DF01AB58BE4F81E090E08C0F9D1FFD
:10764000E80FF91F40815181628173814D935D93F1
:107650006D937C931397D7CFCF92DF92EF92FF92E7
:10766000CF93DF93C82F0E94822F94E0C99FE0013F
:107670001124FE01E759FB4FC080D180E280F380E6
:1076800081110E948F2FC055D84FC701B6010E94AB
:1076900015EA288139814A815B810E9474EADF9171
:1076A000CF91FF90EF90DF90CF900895A1E0B0E0F0
:1076B000ECE5FBE30C9405F1898360E0CE010196D3
:1076C0000E940A1B61E0CE0101960E940A1B62E043
:1076D000CE0101960E940A1B89812196E2E00C945A
:1076E00021F1A2E1B0E0E7E7FBE30C9401F1DEDF7A
:1076F0008823C1F1EDB6FEB641E952E082FF02C037
:1077000048E852E021E932E081FF02C02AE832E095
:1077100080FD25C081E992E05F934F933F932F93C3
:107720009F938F938CE097E09F938F938E010F5FD1
:107730001F4F1F930F930E94A8E90E94C28AC8019D
:107740000E944384C8010E9465C50FB6F894DEBF4D
:107750000FBECDBF81E06296E6E00C941DF18CE88F
:1077600092E0DACF80E0F7CFA0E2B0E0EAEBFBE313
:107770000C94F5F080911201882309F4BEC0809129
:107780000D04082F10E080FF3CC0C0901401D09081
:107790001501E0901601F09017012091A30230919D
:1077A000A4024091A5025091A602C701B6010E9411
:1077B00090F2181644F4C092A302D092A402E09270
:1077C000A502F092A602C0902001D0902101E09085
:1077D0002201F09023012091A3023091A402409154
:1077E000A5025091A602C701B6010E940FEA87FFC9
:1077F00008C0C092A302D092A402E092A502F09227
:10780000A60201FF3CC0C0901801D0901901E09081
:107810001A01F0901B012091A7023091A80240911B
:10782000A9025091AA02C701B6010E9490F218164F
:1078300044F4C092A702D092A802E092A902F0926A
:10784000AA02C0902401D0902501E0902601F0907A
:1078500027012091A7023091A8024091A9025091DE
:10786000AA02C701B6010E940FEA87FF08C0C092B2
:10787000A702D092A802E092A902F092AA0202FF07
:107880003CC0C0901C01D0901D01E0901E01F09002
:107890001F012091AB023091AC024091AD0250919A
:1078A000AE02C701B6010E9490F2181644F4C092CD
:1078B000AB02D092AC02E092AD02F092AE02C09068
:1078C0002801D0902901E0902A01F0902B0120910D
:1078D000AB023091AC024091AD025091AE02C701B3
:1078E000B6010E940FEA87FF08C0C092AB02D09297
:1078F000AC02E092AD02F092AE028091700D83FD79
:1079000061C02091810130918201409183015091A9
:1079100084016091AF027091B0028091B1029091A8
:10792000B2020E940FEA882309F44CC00E94B8B644
:10793000182F882331F00E94C28A81EF96E00E94BE
:1079400052842091810130918201409183015091B4
:1079500084016091AF027091B0028091B102909168
:10796000B2020E942CF19F7720916F01309170013B
:1079700040917101509172010E9474EA20E030E060
:1079800046E154E40E9490F21816D4F40E94C28A90
:1079900082ED96E00E9452848091AF029091B002F5
:1079A000A091B102B091B2028093810190938201C3
:1079B000A0938301B09384018FEA92E0CEDC02C0F1
:1079C0001111EACF2AE037ED43E25CE360910C014C
:1079D00070910D0180910E0190910F010E9474EA47
:1079E0006B017C016091100170911101072E000C58
:1079F000880B990B0E9415EA9B01AC01C701B601E7
:107A00000E9474EA698B7A8B8B8B9C8B8091B3027A
:107A1000882309F18090B4029090B502A090B6023C
:107A2000B090B702C090AB02D090AC02E090AD0233
:107A3000F090AE0220E030E0A901C501B4010E943F
:107A40000FEA8823F9F0A7019601C501B4010E944D
:107A500090F21816BCF020E030E0A901BE016F5E84
:107A60007F4F83EA92E00E94D9C680E1E3EAF2E028
:107A7000A5E7B1E001900D928A95E1F7A096E2E1C9
:107A80000C9411F1209175013091760140917701AC
:107A9000509178016091A3027091A4028091A50297
:107AA0009091A6020E942CF14B015C01209179017A
:107AB00030917A0140917B0150917C016091A70245
:107AC0007091A8028091A9029091AA020E942CF1C3
:107AD0006D8B7E8B8F8B988F20917D0130917E01F5
:107AE00040917F0150918001C701B6010E942CF1A5
:107AF0006D8F7E8F8F8F98A32091810130918201AD
:107B000040918301509184016091AF027091B00265
:107B10008091B1029091B2020E942CF1698F7A8F0C
:107B20008B8F9C8F20E030E0A901C501B4010E9439
:107B30000FEA81110CC020E030E0A9016D897E8937
:107B40008F89988D0E940FEA882309F484CFA501BC
:107B50009401C501B4010E9474EA6B017C012D8976
:107B60003E894F89588DCA01B9010E9474EA9B0170
:107B7000AC01C701B6010E942DF16B017C012D8D76
:107B80003E8D4F8D58A1CA01B9010E9474EA9B0134
:107B9000AC01C701B6010E942DF16B017C01298D5A
:107BA0003A8D4B8D5C8DCA01B9010E9474EA9B012C
:107BB000AC01C701B6010E942DF16B017C010E944E
:107BC000C9F22B013C012CEC3CEB4CE85BE2C70119
:107BD000B6010E940FEA87FF06C0498C5A8C6B8C55
:107BE0007C8CE89477F82DEB37E346E855E3C30146
:107BF000B2010E940FEA87FD38CF2DEC3CEC4CE43B
:107C00005EE3C301B2010E9474EA0E9411F21B01FB
:107C1000672B19F422242394312CB10190E080E0E9
:107C20000E9413EA9B01AC0160E070E080E89FE3F2
:107C30000E94A4F16B017C01AC019B01C301B20164
:107C40000E9474EA2B013C01A7019601C501B40111
:107C50000E9474EA4B015C01A70196016D897E893F
:107C60008F89988D0E9474EA6D8B7E8B8F8B988F95
:107C7000A70196016D8D7E8D8F8D98A10E9474EA6B
:107C80006D8F7E8F8F8F98A3A7019601698D7A8D56
:107C90008B8D9C8D0E9474EA698F7A8F8B8F9C8F5D
:107CA00080E1E5E7F1E08E010F5F1F4FD801019001
:107CB0000D928A95E1F70E9402D16B017C0128ECBC
:107CC000C20ED11CE11CF11C81E0281A310809F414
:107CD00054C00E9402D19B01AC012C193D094E09F0
:107CE0005F0957FD4DC06B017C0128ECC20ED11C11
:107CF000E11CF11C80E00E94508FA5019401698174
:107D00007A818B819C810E942DF169837A838B8398
:107D10009C832D893E894F89588D6D817E818F810D
:107D200098850E942DF16D837E838F8398872D8D9A
:107D30003E8D4F8D58A169857A858B859C850E94E3
:107D40002DF169877A878B879C87298D3A8D4B8D9A
:107D50005C8D6D857E858F8598890E942DF16D875C
:107D60007E878F87988BA3019201BE016F5E7F4F44
:107D7000C8010E94D9C68111A7CFA30192016ECE7E
:107D80000E94F029BACF8091090490910A04A09131
:107D90000B04B0910C0480930C0190930D01A093FF
:107DA0000E01B0930F018091070490910804909305
:107DB000110180931001089580910C0190910D01A3
:107DC000A0910E01B0910F018093090490930A04D1
:107DD000A0930B04B0930C048091100190911101B9
:107DE000909308048093070484E690E09093110137
:107DF000809310010895ACE0B0E0E1E0FFE30C9463
:107E0000F7F02B013C0129873A874B875C874701B4
:107E10005801D601CD90DD90ED90FC9020E030E04F
:107E2000A901C701B6010E940FEA811171C08091BA
:107E30006B0190916C01A0916D01B0916E018983ED
:107E40009A83AB83BC8320E030E0A901C701B6016F
:107E50000E940FEA811106C0C12CD12C80E8E82EC7
:107E600080E4F82ECD82DE82EF82F886A5019401AF
:107E700060917D0170917E0180917F0190918001E0
:107E80000E940FEA87FF0CC080927D0190927E01D4
:107E9000A0927F01B0928001CE0105960E945022EF
:107EA000409275015092760160927701709278014C
:107EB00089859A85AB85BC858093790190937A01F9
:107EC000A0937B01B0937C01CE0101960E945022C9
:107ED000A501940160917D0170917E0180917F01E7
:107EE000909180010E9490F2181664F480927D01B6
:107EF00090927E01A0927F01B0928001CE01059602
:107F00000E9450220E94AE2C2C96E0E10C9413F1BA
:107F1000D701C60194CFCF92DF92EF92FF920F93D9
:107F20001F936B01FC01E080F18002811381E5E782
:107F3000F1E02481358146815781608171818281A0
:107F4000938159DF1F910F91FF90EF90DF90CF90B9
:107F500008950C94FCC60F931F93CF93DF93EC010D
:107F60008B010E941A8E882331F081E0DF91CF913E
:107F70001F910F910895B801CE01CDDF80912E079A
:107F8000C82FC47082FD0AC010922E0782E0E0DA8A
:107F9000E0DF81E0CC2351F380E0E8CF0E94D98D6F
:107FA000882391F3E2CFCF930E94822FC82F809134
:107FB000681380936713809366138093651384E638
:107FC000809364130E94133080ED93E09093BA0D78
:107FD0008093B90DC1110E948F2F81E080936804B6
:107FE0000E94AE2C8EEFB4DAB4DFCF910895ACE0EE
:107FF000B0E0EDEFFFE30C9405F10E9477B60E942C
:10800000822F9CE0E5E7F4E0DE01119601900D92ED
:108010009A95E1F781110E948F2FCE0101960E945F
:10802000282B2C96E2E00C9421F1B0E0A0E0EBE1EB
:10803000F0E40C94F7F04090750150907601609058
:108040007701709078018090790190907A01A090EA
:108050007B01B0907C01C0907D01D0907E01E090CA
:108060007F01F09080010E94422C60912C01709160
:108070002D01072E000C880B990B0E9415EA2AE0AF
:1080800037ED43E25CE30E9474EA60936F01709302
:108090007001809371019093720104E111E0D0E0CE
:1080A000C0E0CE01815D954F0E947577F801619324
:1080B0007193819391938F01CE018D5D954F0E94B5
:1080C0007577F80160877187828793872496CC3013
:1080D000D10539F760E08BE194E00E94567A0E9466
:1080E000237B0E94862CA3019201609175017091FF
:1080F000760180917701909178010E940FEA8111B9
:108100001BC0A50194016091790170917A01809161
:108110007B0190917C010E940FEA81110DC020919A
:108120007D0130917E0140917F0150918001C70116
:10813000B6010E940FEA81115ADFCDB7DEB7E0E148
:108140000C9413F1A4E0B0E0E8EAF0E40C9405F13B
:1081500084EF91E0A0E0B0E089839A83AB83BC8395
:10816000BE016F5F7F4F8CE30E94F98288EB96E03F
:108170000E94528486B162EB76E082FB882780F908
:108180000E94AA2186B16CEA76E083FB882780F9F9
:108190000E94AA2186B166EA76E0829581700E94EB
:1081A000AA21349907C00E942D832496E2E00C9402
:1081B00021F106C00E9416832496E2E00C9421F17E
:1081C0008091E806811103C08091EA0681110C9428
:1081D000B12F0895ACE0B0E0E0EFF0E40C9405F1CD
:1081E000A1E7BDE090E080E0FC01E559F54F459145
:1081F0005591659174914D935D936D937D93FC01C1
:10820000E55AF54F459155916591749150964D936E
:108210005D936D937C935397FC01E55BF54F45911E
:1082200055916591749190964D935D936D937C9368
:108230009397049680319105B9F680E29EE4A0E020
:10824000B0E08093810D9093820DA093830DB09345
:10825000840D80E090E0AAEFB3E48093A50D9093A5
:10826000A60DA093A70DB093A80D8093A90D909390
:10827000AA0DA093AB0DB093AC0D8093AD0D909370
:10828000AE0DA093AF0DB093B00D1092B10D109242
:10829000B20D1092B30D1092B40D1092B50D109254
:1082A000B60D1092B70D1092B80D8AE097EDA3EAC3
:1082B000BDE38093930790939407A0939507B093A1
:1082C000960780E090E0A0E2B1E480931B049093D5
:1082D0001C04A0931D04B0931E040E940C7A8CE031
:1082E000E5E8F1E0DE01119601900D928A95E1F743
:1082F00089819A81AB81BC818093561390935713E7
:10830000A0935813B09359138D819E81AF81B88586
:1083100080935A1390935B13A0935C13B0935D13F7
:1083200089859A85AB85BC8580935E1390935F1396
:10833000A0936013B09361138EEB90E090934C0781
:1083400080934B078CE390E090934E0780934D070A
:108350001092500710924F0786EE90E090935207CC
:108360008093510786E490E09093540780935307DD
:1083700010925607109255078FE892ECADE8B1E4E1
:108380008093BD129093BE12A093BF12B093C012FF
:108390008CE998EFA5E4BEE38093C1129093C212DA
:1083A000A093C312B093C41281E49CEBABECB3E492
:1083B0008093C5129093C612A093C712B093C812AF
:1083C00080E090E0AFEAB3E480933F0790934007EA
:1083D000A0934107B093420785E996E2A5E2B1E494
:1083E0008093430790934407A0934507B0934607B3
:1083F00080EA9CE6ACE2B5E4809347079093480797
:10840000A0934907B0934A071092E8061092E70636
:10841000D7DE0BDE2C96E2E00C9421F1A4E0B0E074
:10842000E4E1F2E40C94F6F09091EA06981709F46E
:1084300055C0382E80E090E0A0E2B1E489839A83B1
:10844000AB83BC83C0905E13D0905F13E090601349
:10845000F090611320E030E0A901C701B6010E944D
:108460000FEA87FF0CC0A701960160E070E080E290
:1084700091E40E942CF169837A838B839C83CE01E3
:1084800001960E948DC740907501509076016090D2
:108490007701709078018090790190907A01A09096
:1084A0007B01B0907C013320F1F00E941A8E19827A
:1084B0001A821B821C82E0907D01F0907E01009167
:1084C0007F0110918001CE0101966C01A5019401FC
:1084D000C301B20190DC3092EA0672DE80E024969D
:1084E000E1E10C9412F10E94D98DE1CFB0E0A0E05F
:1084F000ECE7F2E40C94F7F0C82FE82EF12CF7012A
:10850000E858F24DD491823071F481E087DF811117
:1085100005C00E941A8E882309F4E2C0CDB7DEB7E9
:10852000E0E10C9413F16D2FDD0F770B880B990BA5
:108530000E9415EA2B013C01C701880F991F880F83
:10854000991F855A984F0E9475774B015C01A301D2
:108550009201C501B4010E9474EA4B015C016701FC
:10856000CC0CDD1CCC0CDD1CC601815B984F0E943D
:108570007577A30192010E9474EA20E030E040EC9C
:108580005FE30E9474EAAB01BC0100E010E09801D7
:108590008C2F0E94C3CAC23009F0CCC00E94D98D72
:1085A00020E030E0A901C501B4010E940FEA882350
:1085B00029F100E010E020E830E4B501A401705892
:1085C0008C2F0E94C3CAC23009F467C0A501940170
:1085D000C501B4010E942DF14B015C01C23009F0CC
:1085E00062C000E010E020E030E4B501A4018C2F6F
:1085F0000E94C3CAC23011F40E94D98D81E090E07C
:108600000C2E01C0880F0A94EAF790917F07982BEF
:1086100090937F0790910D04892B80930D04C601E0
:108620008D5B984F0E947577F601EB58FE4F608383
:10863000718382839383C230D1F420915E13309191
:108640005F13409160135091611360917D017091AF
:108650007E0180917F01909180010E942CF16093B6
:108660007D0170937E0180937F019093800171DC86
:10867000F601ED55FD4FD601AB58BE4F8D919D9142
:108680000D90BC91A02D80839183A283B383C230CF
:1086900009F044CF80E0C2DE41CF0E941A8E8823C9
:1086A00009F494CF3BCFF701E05CF84F649161117E
:1086B00007C00E94C28A8EE197E00E9452846AE05D
:1086C00070E090E080E00E9413EA9B01AC0161E061
:1086D00070E088E492E40E94A4F18B019C0185CFB4
:1086E00083E697E00E94757720E030E0A9010E94C0
:1086F0000FEA882309F417CF6D2FDD0F770B880B56
:10870000990B0E9415EA2B013C0183E697E00E9439
:1087100075774B015C0120E030E040EA50E40E94B4
:1087200090F287FF14CF812C912C90EAA92E90E42F
:10873000B92E0DCF20E030E0A901C501B4010E949F
:108740000FEA882309F45ACF00E010E0980135CFF2
:1087500080912E07882319F010922E07089540E08B
:1087600070E060E086E896E00E94618E1F920F92B2
:108770000FB60F9211240BB60F922F933F934F9386
:108780005F936F937F938F939F93AF93BF93EF9379
:10879000FF930E94B12FFF91EF91BF91AF919F91F5
:1087A0008F917F916F915F914F913F912F910F909A
:1087B0000BBE0F900FBE0F901F9018950F931F9335
:1087C00080918F07813019F50E9402D10091F20348
:1087D0001091F3032091F4033091F503601B710BAA
:1087E000820B930B28EE33E040E050E00E943DF016
:1087F0006091EE037091EF038091F0039091F1038B
:10880000620F731F841F951F1F910F910895609130
:10881000F6037091F7038091F8039091F903D6CF96
:1088200010928F071092F2031092F3031092F40348
:108830001092F5031092F6031092F7031092F803CA
:108840001092F9031092EE031092EF031092F003CE
:108850001092F103089580918F078130E1F082300A
:10886000C1F4ACDF6093EE037093EF038093F003E9
:108870009093F10381E080938F070E9402D160936F
:10888000F2037093F3038093F4039093F50381E074
:108890000895C6DFEFCF80E008950E94DBC70E94F5
:1088A000BD7B882351F08091E51482FD06C087EEE0
:1088B00091E09093ED068093EC06CDCF80918F07E9
:1088C000813079F482E080938F070E9402D1609317
:1088D000F6037093F7038093F8039093F90381E014
:1088E000089580E0089580918F078150823070F460
:1088F00010928F070E9402D16093F6037093F703E2
:108900008093F8039093F90381E0089580E008953F
:108910002091BA123091BB12263531053CF42091DA
:108920003C0730913D07263031051CF0882331F09B
:1089300092CF662319F0D7DF0C94DBC708959C0112
:1089400097FF26C0EE27FF27E81BF90B2D398FEF85
:1089500038070CF05DC08DE280939E02CF0164E683
:1089600070E00E94C7F0CB012AE030E0B9010E941C
:10897000C7F0805D80939F02CF01B9010E94C7F0CC
:10898000CB01B9010E94C7F0805D8093A0022AC08C
:10899000283E83E03807B4F1C90168EE73E00E9415
:1089A000C7F0CB01EAE0F0E0BF010E94C7F0805DB4
:1089B00080939E02C90164E670E00E94C7F0CB017B
:1089C000BF010E94C7F0805D80939F02C901BF0173
:1089D0000E94C7F0CB01BF010E94C7F0805D809369
:1089E000A002F901CF016AE070E00E94C7F0805D4B
:1089F0008093A1028EE992E008958DE237FDC5CF04
:108A000080E2C3CFF90180E2243631050CF0A4CF17
:108A100080E280939E0280939F02EA30F1056CF31E
:108A20008DE237FF80E280939F02CF016AE070E021
:108A30000E94C7F0605D6093A002D4CF9C0197FDB7
:108A40002DC080E2243631055CF0C90164E670E097
:108A50000E94C7F0CB016AE070E00E94C7F0805D21
:108A600080939F0280E22A3031055CF0EAE0F0E07A
:108A7000C901BF010E94C7F0CB01BF010E94C7F02E
:108A8000805D8093A002C9016AE070E00E94C7F097
:108A9000805D8093A1028FE992E008953195219540
:108AA00031098DE2DDCFCF92DF92EF92FF92FC0190
:108AB000C080D180E280F38020E030E0A901C701CE
:108AC000B6010E940FEA87FD26C06DEB77E386E0D2
:108AD00095E3A70196010E942DF16B017C0120E036
:108AE00030E0A9010E940FEA20E030E040E05FE3BF
:108AF00087FF04C020E030E040E05FEBC701B60133
:108B00000E942DF10E940CF2CB0198DFFF90EF90B4
:108B1000DF90CF9008956DEB77E386E095EBD9CFAA
:108B2000A4E0B0E0E6E9F5E40C9405F10E9415EA52
:108B300069837A838B839C83CE010196B4DF24966C
:108B4000E2E00C9421F1FC016081718182819381CA
:108B50000E940CF2CB0172CFA4E0B0E0E2EBF5E4AE
:108B60000C9405F10E9415EA69837A838B839C83B8
:108B7000CE010196E8DF2496E2E00C9421F10F93F8
:108B80001F930E9402D10091E1061091E20620910C
:108B9000E3063091E4060115110521053105D9F5EB
:108BA00020917B132223A1F1E0917913215020938E
:108BB0007B1321E02E0F2093791330917C13231324
:108BC00002C01092791324E0E29FF0011124E358CF
:108BD000FC4E00811181228133810093DD061093C8
:108BE000DE062093DF063093E006600F711F811DC3
:108BF000911D6093E1067093E2068093E3069093E3
:108C0000E4068091DF069091E006892B09F0149A22
:108C10001F910F910895601B710B820B930B97FDB1
:108C2000F7CF14981092E1061092E2061092E30634
:108C30001092E406EDCF0F931F93CF93DF938C0137
:108C4000EB0190917B1320917C13921304C097DF6A
:108C50000E94F029F6CF80917A1334E0839FF001CF
:108C60001124E358FC4E11830083D383C2839F5F9A
:108C700090937B138F5F281739F080937A13DF91DD
:108C8000CF911F910F91089510927A13F8CF8823F6
:108C900051F063E972E084E690E0CDDF6AEB72E0C8
:108CA00084E690E0C8CF68EB71E084E190E0FACF11
:108CB00091DA81E0ECCF8F929F92AF92BF92EF92C8
:108CC000FF920F931F93CF93DF93EC018B01E42E60
:108CD000F22E80918D1390918E138C179D07C9F100
:108CE00023E6CC33D20709F03FC08B5C9B4771F47D
:108CF0000E9402D16E517B4F8F4F9F4F6093DE03D6
:108D00007093DF038093E0039093E103D0938E137D
:108D1000C0938D1330E020E0009372071093730727
:108D20002093740730937507E0926D07F0926E07F9
:108D3000CB5CDB4721F410929A021092DD0382E0B3
:108D400080936A0181E080936F07109299021092DC
:108D5000E903DF91CF911F910F91FF90EF90BF90AA
:108D6000AF909F908F9008952BE7CB3CD20771F680
:108D70008C539346D9F40E9402D18090DE039090E8
:108D8000DF03A090E003B090E103681979098A0934
:108D90009B0997FF0BC080917F078770873031F464
:108DA0000E942723CBE0D8E58111B0CFCBECDBE7E5
:108DB000ADCF20E040E070E060E086E193E27BCF61
:108DC0000E94B8B6882339F020E040E070E060E00F
:108DD0008DE297E570CFEDCF21E020939A02FC0160
:108DE00080819181A281B3818093080190930901D0
:108DF000A0930A01B0930B0120E040E070E060E036
:108E000080915C0790915D0756CFA4E0B0E0EBE065
:108E1000F7E40C9405F18DEC9CECACECBCE389839D
:108E20009A83AB83BC83CE010196D6DF2496E2E021
:108E30000C9421F1A4E0B0E0E0E2F7E40C9405F139
:108E40008DEC9CECACECBDE389839A83AB83BC8353
:108E5000CE010196C1DF2496E2E00C9421F1A4E05A
:108E6000B0E0E5E3F7E40C9405F180E090E0A0E8E1
:108E7000BFE389839A83AB83BC83CE010196ACDFC9
:108E80002496E2E00C9421F1A4E0B0E0EAE4F7E4F7
:108E90000C9405F180E090E0A0E2B1E489839A832C
:108EA000AB83BC83CE01019697DF2496E2E00C945D
:108EB00021F181E080939A0280917F07877087304B
:108EC00051F010927F0710920D0480EF95E090937F
:108ED000ED068093EC068091B3028093EB0380E073
:108EE0000E94CA7920E040E070E060E089E797E402
:108EF000E2CE80916A01882331F041E062EA73E0BA
:108F000082E00E9470CB80910D048770873071F4ED
:108F10001092EA0320E040E070E060E08DEA97E51F
:108F2000CADE81E08093E9030C945822089520E082
:108F300040E070E060E08BEC9BE7BDCE1092AF07A5
:108F40000E94F527F4CFB0E0A0E0E9EAF7E40C9442
:108F5000FFF0CDB6DEB6E2E8F7E0DF010D900020CD
:108F6000E9F7CD018A5797402DB73EB7281B390B3B
:108F70000FB6F8943EBF0FBE2DBF0DB71EB70F5FE3
:108F80001F4FFF93EF9383E595E09F938F931F937C
:108F90000F930E94A8E9780134E0E30EF11C0F90D2
:108FA0000F900F900F900F900F90D7018D917D0132
:108FB000882349F0082E000C990B0E940EF3F7014C
:108FC00031978083F2CF6EE475E0C8010E9441E9D9
:108FD0004FE350E0B8018EEE96E00E9466F30FB6C4
:108FE000F894DEBE0FBECDBEA2DF0E94DBC7E8E074
:108FF0000C941BF18093300720E040E070E060E0CB
:109000008BEC97E558CEA2E8B0E0E9E0F8E40C94E8
:10901000F5F0ADB6BEB684E690E09093A6128093CC
:10902000A5121092CA121092C91241E064E070E0D9
:10903000CE0187589F4F0E94BFB543E050E0BE016C
:1090400067587F4F86E292E00E9458F3892BF9F02F
:10905000ED968FADED97882339F08FE3EA968FAFC9
:10906000EA97EB961FAEEB9782E0C4DF81E0809336
:109070001A0490911A0481E089270FB6F894BEBEB5
:109080000FBEADBECE57DF4FE2E10C9411F141E0CF
:1090900062E070E0CE0183589F4F0E94BFB5E99611
:1090A0001CAE1DAE1EAE1FAEE9971092CA121092F2
:1090B000C912CE018F579F4F0E942622EDB6FEB6F1
:1090C000CF57DF4FC880C158D040D12C23E0C20E0B
:1090D000D11CCC0CDD1CCC0CDD1C8DB79EB78C19C3
:1090E0009D090FB6F8949EBF0FBE8DBFEDB7FEB7BA
:1090F00031963F018C199D090FB6F8949EBF0FBEA3
:109100008DBFEDB7FEB731964F018C199D090FB693
:10911000F8949EBF0FBE8DBF0DB71EB70F5F1F4FD8
:10912000B601C3010E942B2240918C0381E04827A5
:1091300064E070E081E89DE00E94BFB5B601C40123
:109140000E942B22B601C8010E942B2290918C0311
:10915000CE57DF4F9883C258D04091114BC0CF57A4
:10916000DF4F8881C158D04090E00296A1E7BDE072
:1091700050E040E030E020E067E77AE0E7E6CE2E1E
:10918000EAE0DE2E821793070CF495C0F301E40F9A
:10919000F51F20803180428053802D923D924D9268
:1091A0005D92821793070CF48CC0F401E40FF51F55
:1091B000208031804280538050962D923D924D9276
:1091C0005C925397821793070CF481C0F801E40F67
:1091D000F51F208031804280538090962D923D92E1
:1091E0004D925C9293972F5F3F4F4C5F5F4F2430BF
:1091F000310541F685EA9DE00E94FE2189EA9DE065
:109200000E94FE218DEA9DE00E94FE2181EB9DE0FF
:109210000E94FE2185EB9DE00E94FE21CE018B582D
:109220009F4F0E94FE21CE018B589F4F0E94FE212E
:10923000CE018B589F4F0E94FE21CE018B589F4F2D
:109240000E94FE2183E997E00E94FE210FB6F89468
:10925000FEBE0FBEEDBE8E010F5F1F4FC8010E9404
:109260001E22CE0183599F4F0E940622C8010E94F0
:10927000FE218BE194E00E94FE21CE018B589F4F8E
:109280000E94FE21CE0183599F4F0E942622C801D1
:109290000E942622AE96CFACAE978981C89E60010F
:1092A0001124E1E0CE1AD108C8F0CE018B589F4FAF
:1092B0000E94FE21F6CFFB012590359045905490F9
:1092C0006CCFF601259035904590549075CFE7E529
:1092D000FAE025903590459054907FCF86E593E154
:1092E0000E941E228AE0D82EDA94CE01DD2029F0D9
:1092F0008B589F4F0E94FE21F7CF80589F4F0E94AE
:109300002622CE0181589F4F0E942622C058DF4F4F
:109310008881C058D040873009F05EC1C158DF4F06
:109320008881CF57D040873009F056C1CE57DF4FE4
:109330002881C258D040211103C080E00E94CA7920
:1093400084E893E00E9416228CE793E00E941622A4
:1093500040918C0381E0482764EC70E088EB92E058
:109360000E94BFB5C8010E940E22CE0183599F4FB3
:109370000E94062240918C03FF24F3944F2564E061
:1093800070E0C8010E94BFB58BEE96E00E940E22ED
:1093900040918C034F256CE070E08BE497E00E94D5
:1093A000BFB540918C034F2564E170E0C8010E9475
:1093B000BFB5F0908C03F11030C089819A81AB81E8
:1093C000BC818093BD129093BE12A093BF12B09344
:1093D000C0122CEA35EC47E25EE36D817E818F811D
:1093E00098850E9474EA6093C1127093C2128093B0
:1093F000C3129093C41220E030E543EC50E4698539
:109400007A858B859C850E9474EA6093C51270935F
:10941000C6128093C7129093C81241E04F2562E0B4
:1094200070E0C8010E94BFB5C8010E94F621D0902B
:109430008C03D11030C089819A81AB81BC8180932B
:109440003F0790934007A0934107B09342072CEA4F
:1094500035EC47E25EE36D817E818F8198850E94C5
:1094600074EA609343077093440780934507909391
:10947000460720E030E543EC50E469857A858B852A
:109480009C850E9474EA6093470770934807809315
:10949000490790934A07C8010E94F621C8010E941B
:1094A0000622C8010E940622C8010E94062285E009
:1094B000F80111928A95E9F7FF24F3944D2D4F2579
:1094C00065E070E0C8010E94BFB5C8010E940E228D
:1094D00040918C034F2560E270E0C8010E94BFB547
:1094E000CE0183599F4F0E940E2240918C034F253D
:1094F00069E070E0C8010E94BFB540918C034F2520
:1095000062E170E0C8010E94BFB540918C034F2515
:1095100064E270E0C8010E94BFB540918C034F2502
:1095200060E170E0C8010E94BFB540918C034F25F7
:1095300069E070E0C8010E94BFB5C8010E94FE2129
:1095400040918C034F256CE070E0C8010E94BFB5CC
:1095500040918C034F256CE670E0C8010E94BFB5B6
:1095600019821A821B821C821D821E821F8218860B
:1095700019861A861B861C86C8010E94F621409116
:109580008C034F2568E070E0C8010E94BFB5C80198
:109590000E941E22CE0181589F4F0E940622CE01BA
:1095A00083599F4F0E94FE218091A5129091A6128F
:1095B0008037934089F510921A042091C912309196
:1095C000CA12EF968EAD9FADEF972817390741F17C
:1095D000F0921A0480E023C0CE0183599F4F0E946D
:1095E0001622C8010E941622C058DF4FC880C058FA
:1095F000D040C158DF4F8881CF57D040C89E60010E
:10960000112481E0C81AD10808F4ACCECE018B58E1
:109610009F4F0E94FE21F5CFF0921A0481E0EADC10
:1096200080918C03811125CD80911A04811121CD67
:109630000E9415401ECD81E080938C03E4DC1092E3
:109640008C03882309F0DFCC0E94EA4080E0089573
:10965000F2DF1DCBCF93DF93C091DD03CC23B1F0BC
:10966000C150C093DD0389E0C89FE0011124C955B2
:10967000DC4F6A817B812F814E81888199811BDB40
:10968000888580939A02DF91CF91089550DCFBCFBB
:10969000A4E0B0E0EEE4FBE40C94F8F00E9484CC8B
:1096A000F0906D076F2C85E0782E7F0C86E0E82E19
:1096B000EF1885E0D82EDF18AA24AA94B12C84E0F4
:1096C000C82ECF1882E0982E9F1881E0882E8F1820
:1096D0005F2C5194F1105AC080917007882309F4CF
:1096E00044C080916A01882359F081E0909170070D
:1096F000911180E024E041E856E0652D0E94D0CB36
:109700008091AF078093300724E0F212F7C01092E7
:109710007C0780917007843009F4DDC080916A0174
:109720008823E1F011E080917007843009F010E0A7
:109730008091300724E6829FC001112481589F4FF9
:10974000B5010E94C7F0862F0E94DD1C00E09C013D
:1097500046E656E06C2D812F0E947375F394F71046
:10976000B9CF87E080936E070DC0809157071092A4
:109770005707882309F4B5CF6DDF80916F078823E1
:1097800009F4AFCF2496EFE00C9414F121E0F2122B
:1097900043C080917007813041F180916A01882334
:1097A000F9F011E080917007813009F010E06091CC
:1097B000100170911101072E000C880B990B0E946B
:1097C00015EA69837A838B839C83CE010196BBD98A
:1097D00000E09C014BE756E0682D812F0E947375D5
:1097E0008091AF0780933007B9CF809157071092CF
:1097F0005707882391F210E000E027EE33E04AE0BB
:1098000050E060E171E08BE796E00E9449CD8091E5
:109810006F07882311F2B6CF82E0F812D7C080918B
:109820007007823021F180916A018823C9F211E02A
:1098300080917007823009F010E06091BA12709147
:10984000BB12072E000C880B990B0E9415EA698346
:109850007A838B839C83CE01019675D900E09C01AD
:1098600044E756E0692D812F0E94737549CF80919E
:109870005707109257078823B1F20E9478CC04EF63
:1098800011E225EF30E050E040E06AEB72E184E75E
:1098900096E00E9449CD80916F07882321F272CF14
:1098A0008091570710925707882309F497C00E94A8
:1098B00078CC02E31AE623E730E050E040E06CE3C6
:1098C00077E080E796E00E9449CD80916F0788237A
:1098D00009F484C057CF8091570710925707882307
:1098E00009F41CCF0E9478CC86E696E00E94BECF99
:1098F00080916F07882309F411CF44CF85E0F812D7
:109900003DC080917007853011F180916A018823F4
:1099100009F424CF11E080917007853009F010E040
:1099200060912C0170912D01072E000C880B990B72
:109930000E9415EA69837A838B839C83CE0101960A
:1099400002D900E09C0141E656E06D2D04CF8091E4
:109950005707109257078823C1F20EEF1CE127EE3C
:1099600033E04AE050E06CE271E081E696E00E946C
:1099700049CD80916F07882341F204CF26E0F2128F
:10998000EDCE80917007863091F080916A01882336
:1099900009F4E4CE81E090917007963009F080E000
:1099A00023E042E556E06E2D0E94D0CBD7CE8091C9
:1099B000570710925707882341F38BE098E50E94E0
:1099C000DACC80916F07882301F3DCCE83E0F812B4
:1099D00097CE80917007833009F462CF80916A013D
:1099E000882309F4FDCE11E080917007833009F0DF
:1099F00010E060913C0770913D07072E000C880B2A
:109A0000990B0E9415EA69837A838B839C83CE012C
:109A1000019699D863E0661900E09C0140E756E0A2
:109A200022CFA4E0B0E0E7E1FDE40C94F6F0EE24F0
:109A3000E3948091BA129091BB12892B09F4E12C26
:109A40000E9484CCF0906D074F2C95E0592E5F0C4E
:109A500088248A94912C83E0B82EBF1882E0A82E27
:109A6000AF1881E0782E7F183F2C319486E0682E65
:109A70006F18F11015C080917007882309F4D7C0C2
:109A800080916A01882309F475C181E09091700783
:109A9000911180E024E04DE456E0632D0E94D0CB8C
:109AA0008091BA129091BB12909331078093300746
:109AB00021E0F212E8C080917007813009F4C8C03B
:109AC00080916A01882309F44DC011E080917007EC
:109AD000813009F010E06091300770913107072E56
:109AE000000C880B990B0E9415EA69837A838B839B
:109AF0009C83CE01019627D800E09C0146E456E005
:109B0000672D812F0E9473758091AF078093300776
:109B100093E0F91227C010927C0780917007833080
:109B200009F4F4C080916A018823E1F011E080918A
:109B30007007833009F010E08091300724E6829F9F
:109B4000C001112481589F4FB4010E94C7F0862F95
:109B50000E94DD1C00E09C0148E356E06B2D812F44
:109B60000E947375D12CC12C14E00F2D0419C092E2
:109B70003007F1121FC0F601EE0FFF1FEF5DF94F26
:109B80008591949190937E0780937D0780917007D3
:109B90008F1509F4CEC080916A01882359F081E0C5
:109BA00090917007911380E023E04EE256E0602F21
:109BB0000E94D0CB812F9FEFC91AD90A15E08530BA
:109BC000B1F680913C0790913D07892B19F4EE2066
:109BD00009F4CEC026E0F21221C0809170078630D1
:109BE00009F4B8C080916A018823C1F08EE997E436
:109BF0009F938F9385E296E09F938F936F9281E07E
:109C000090917007963009F080E08F930E94E222D5
:109C10000F900F900F900F900F900F9087E0EE2411
:109C2000E394F394F51025CF80936E070DC08091D7
:109C3000570710925707882309F422CF0BDD809134
:109C40006F07882309F41CCF2496E1E10C9412F1EC
:109C50008091570710925707882309F431CF0E944B
:109C600078CC02EF12E225EF30E050E040E060E314
:109C700077E086E496E00E9449CD80916F078823C3
:109C800009F41ECFE1CF82E0F8123ECF8091700739
:109C9000823019F180916A01882309F463CF11E0C1
:109CA00080917007823009F010E060913C0770915C
:109CB0003D07072E000C880B990B0E9415EA69835B
:109CC0007A838B839C83CE0101960E94A34500E09A
:109CD0009C0142E456E06A2D14CF80915707109200
:109CE00057078823B9F20E9478CC02E31AE623E7EB
:109CF00030E050E040E06CE377E082E496E00E94E0
:109D000049CD80916F07882329F29ECF8091570714
:109D100010925707882309F405CF0E9478CC88E376
:109D200096E00E94BECF80916F07882309F4FACE97
:109D30008BCF8091570710925707882309F42BCFB8
:109D400083EC9EE40E94DACC80916F07882309F4AB
:109D500022CF7ACF8091570710925707882309F4B2
:109D600041CFECD880916F07882309F43BCF6CCFAB
:109D700086E057CF8091BA129091BB129093310731
:109D800080933007C1CEB0E0A0E0E9ECFEE40C9493
:109D9000F7F0009130070E9484CCC0916D0710E06D
:109DA000000F111F0F5D194F95E0592E5C0E29EF22
:109DB000E22E25E0F22ED3E0DC1B32E0C32E33E2AC
:109DC000D32E47E0A42E46E0B42E82E0782E7C1AF3
:109DD0005EE2852E56E0952E81E0682E6C1A4C2EA0
:109DE0004194C1112AC0809170078823B1F08091FD
:109DF0006A01882359F081E090917007911180E009
:109E000024E045E156E0642D0E94D0CBCF5FC51120
:109E1000E8CF84E080936E070BC0809157071092C3
:109E20005707882321F316DC80916F078823F9F206
:109E3000CDB7DEB7E0E10C9413F1C13059F5F8016C
:109E40008591949190937E0780937D078091700710
:109E5000813081F080916A018823C1F21F929F9224
:109E60008F926F9281E090917007913009F474C0E5
:109E700080E072C08091570710925707882351F3F2
:109E800080913007682F0E944DD180916F07882301
:109E900009F3CECFC23009F042C0F8018591949108
:109EA00090937E0780937D07809170078230D1F078
:109EB00080916A01882309F4A9CFDF92CF92BF92E3
:109EC000AF927F9281E090917007923009F080E02C
:109ED0008F930E94E2220F900F900F900F900F909F
:109EE0000F9094CF8091570710925707882301F362
:109EF0000E94022380916F078823D1F299CF80912D
:109F00005707109257078823C1F0609130078FEFF1
:109F10000E944DD180916F07882379F089CFC3309B
:109F200009F074CFF8018591949190937E07809306
:109F30007D0780917007833011F380916A01882337
:109F400009F464CF1F92FF92EF92DF9381E090912A
:109F50007007933009F08CCF8F930E94E2220F900C
:109F60000F900F900F900F9051CFB0E0A0E0EBEB6F
:109F7000FFE40C94FCF00E9484CCC0916D0785E056
:109F8000E82EEC0E95EDC92E95E0D92ED4E0DC1B21
:109F900013E01C1B20EFA22E25E0B22E02E00C1BCA
:109FA00081E0F82EFC1A9C2E9194C1112AC0809158
:109FB00070078823B1F080916A01882359F081E00D
:109FC00090917007911180E024E044EF55E0692DF5
:109FD0000E94D0CBCF5FEC12E8CF85E080936E0774
:109FE0000BC08091570710925707882321F332DB6B
:109FF00080916F078823F9F2CDB7DEB7EBE00C94C0
:10A0000018F1C13011F580917007813079F080919D
:10A010006A018823F9F281E090917007913009F08C
:10A0200080E023E04AE35DE26F2DD2CF80915707B5
:10A0300010925707882359F382E990E50E94DACC01
:10A0400080916F07882319F3D7CFC23009F053C02E
:10A0500090917007923071F080916A01882309F421
:10A06000B9CF81E0923009F080E020E246EE55E081
:10A07000602FAECF8091570710925707882361F366
:10A08000B092ED06A092EC0680916F07882321F331
:10A09000B3CF80917007833081F080916A0188236B
:10A0A00009F498CF81E090917007933009F080E037
:10A0B00023E049ED55E0612F8BCF80915707109237
:10A0C0005707882351F38DE09FE50E94DACC8091F9
:10A0D0006F07882311F390CF80915707109257078D
:10A0E000882391F0D092ED06C092EC0680916F0724
:10A0F000882351F081CFC33061F2C43009F06ACFB8
:10A1000090917007943041F380916A01882309F49B
:10A1100061CF81E0943009F080E020E244EC55E02A
:10A120006D2F56CFB0E0A0E0E8E9F0E50C9400F127
:10A130000E9484CCC0916D0785E0E82EEC0ED4E03F
:10A14000DC1B13E01C1B02E00C1B81E0F82EFC1A48
:10A15000DC2ED194C1112AC0809170078823B1F000
:10A1600080916A01882359F081E0909170079111E4
:10A1700080E024E04DEB55E06D2D0E94D0CBCF5F09
:10A18000EC12E8CF85E080936E070BC080915707F3
:10A1900010925707882321F35DDA80916F07882397
:10A1A000F9F2CDB7DEB7E7E00C941CF1C13011F540
:10A1B00080917007813079F080916A018823F9F2EB
:10A1C00081E090917007913009F080E023E040E653
:10A1D0005DE26F2DD2CF80915707109257078823E9
:10A1E00059F381E193E20E94DACC80916F078823D2
:10A1F00019F3D7CFC23009F055C080917007823073
:10A2000081F080916A01882309F4B9CF81E09091AF
:10A210007007923009F080E023E049E55DE2602FAD
:10A22000ACCF8091570710925707882351F38CE0E9
:10A2300093E20E94DACC80916F07882311F3B1CFAB
:10A2400080917007833081F080916A01882309F43E
:10A2500096CF81E090917007933009F080E023E081
:10A2600042E55DE2612F89CF809157071092570731
:10A27000882351F387E093E20E94DACC80916F0744
:10A28000882311F38ECF80915707109257078823A8
:10A2900091F080EE96E40E94DACC80916F078823DB
:10A2A00051F07FCFC33061F2C43009F068CF8091A4
:10A2B0007007843041F380916A01882309F45FCFED
:10A2C00081E090917007943009F080E023E044E44D
:10A2D0005DE26D2F52CFACE0B0E0E1E7F1E50C9428
:10A2E000F6F09C878B87362E809157071092570780
:10A2F000882339F010929A02ADD92C96E1E10C94A2
:10A3000012F16091720770917307809174079091B8
:10A310007507611571058105910509F45CC02091EF
:10A320001201222309F4AEC0209113012111AAC009
:10A3300021E0321609F484C0E2E03E1609F491C02F
:10A34000C0901401D0901501E0901601F090170113
:10A3500040902001509021016090220170902301D3
:10A360000E9415EA209108013091090140910A01EB
:10A3700050910B010E9474EA6F83788789879A87CE
:10A38000F4E03F9E80011124C8018B589E4F9E83AC
:10A390008D83FC0120813181428153816F817885D9
:10A3A00089859A850E942DF14B015C01A3019201E0
:10A3B000C701B6010E940FEA811173C0F801EB5882
:10A3C000FE4F80829182A282B382832D0E941D6EF5
:10A3D00081E080936A0110927207109273071092C5
:10A3E00074071092750780916A01882309F485CF5C
:10A3F00024E0329EF0011124EB58FE4FC080D18042
:10A40000E280F380C982DA82EB82FC822DEC3CECA4
:10A410004CEC5DE3609108017091090180910A01A3
:10A4200090910B010E9490F287FD65C0CE010196CC
:10A430000E942B1BBC018B859C850E940C755DCFF7
:10A44000C0901801D0901901E0901A01F0901B0102
:10A4500040902401509025016090260170902701C2
:10A460007FCFC0901C01D0901D01E0901E01F090A4
:10A470001F01409028015090290160902A0170909E
:10A480002B016ECF412C20E5522E23EC622E27E4C7
:10A49000722EC12C30E5D32E33ECE32E37ECF32EA5
:10A4A0005FCF20E030E0A9016F81788589859A85AA
:10A4B0000E940FEA87FF0FC0A7019601C501B401F2
:10A4C0000E940FEA87FF7ACFED81FE81C082D182A0
:10A4D000E282F3827ACFA3019201C501B4010E9406
:10A4E00090F218160CF06ACFED81FE814082518205
:10A4F000628273826ACF20E030E44CE156E4C70107
:10A50000B6010E9474EA4B015C0120E030E0A90131
:10A51000C701B6010E940FEA20E030E040EA50E4B3
:10A5200087FF04C020E030E040EA50ECC501B401F0
:10A530000E942DF12DEC3CEC4CEC5DE30E9474EAA2
:10A540000E940CF26B017C01F7FC64C020EA36E843
:10A5500041E050E00E945FF0CA01B9012AE030E01A
:10A5600040E050E00E945FF0605D60939B02C70195
:10A57000B60120E137E240E050E00E945FF08AE05F
:10A58000882E912CA12CB12CCA01B901A5019401EE
:10A590000E945FF0605D60939C02C701B60128EEE7
:10A5A00033E040E050E00E945FF0CA01B901A5012C
:10A5B00094010E945FF0605D60939D028EE2809343
:10A5C0009E02C701B60124E630E040E050E00E9460
:10A5D0005FF0CA01B901A50194010E945FF0605DBE
:10A5E00060939F02C701B601A50194010E945FF02C
:10A5F0006B017C01CA01B901A50194010E945FF0C1
:10A60000605D6093A00280E3C80EC092A1028BE956
:10A6100092E010CFF094E094D094C094C11CD11C6F
:10A62000E11CF11C6DE2A1CF62E082E59DE253CE18
:10A6300061E089E59DE24FCE60E080E69DE24BCE91
:10A64000A4E0B0E0E6E2F3E50C9405F18091570751
:10A6500010925707882341F010929A020E942A4BC9
:10A660002496E2E00C9421F16091720770917307D7
:10A6700080917407909175076115710581059105A9
:10A6800061F10E9415EA2091080130910901409181
:10A690000A0150910B010E9474EA209181013091CE
:10A6A000820140918301509184010E942DF16093B9
:10A6B000810170938201809383019093840183E0F0
:10A6C0000E941D6E81E080936A01109272071092C1
:10A6D0007307109274071092750780916A0188239E
:10A6E00009F4BECF209158073091590740915A077D
:10A6F00050915B076091810170918201809183018B
:10A70000909184010E942CF169837A838B839C83CE
:10A71000CE0101960E942B1BBC0184E49DE20E94A5
:10A720000C759ECFB0E0A0E0E8E9F3E50C9400F1F1
:10A730000E942723082F0E9484CCC0916D07FC2E15
:10A7400085E0E82EEC0E11E01C1BDC2ED194C1112B
:10A7500014C0809170078823F9F080916A018823E2
:10A7600009F474C081E090917007911180E024E0B9
:10A770004CE753E06D2D0E94D0CB01113AC0D2E0DE
:10A78000C130C1F5809170078130B9F080916A01C4
:10A79000811122C0D2E044C0809157071092570720
:10A7A0008823D9F20E942A4B80916F078823A9F24F
:10A7B000CDB7DEB7E7E00C941CF1809157071092FB
:10A7C0005707882319F381E795E50E94DACC809139
:10A7D0006F078823D9F2ECCF81E090917007913018
:10A7E00009F080E023E043E753E0612F0E94D0CBE3
:10A7F000D1CFD1E0DC1314C0809170078D17B9F070
:10A8000080916A01882361F06C2F6F1981E090912B
:10A8100070079C1380E023E047E653E00E94D0CB12
:10A82000CF5FCE1194CFDF5FD0936E07C1CF809101
:10A83000570710925707882319F384E99AE50E9475
:10A84000DACC80916F078823D9F2B2CFD1E0002310
:10A8500009F4A0CFE5CFB0E0A0E0E1E3F4E50C948B
:10A86000F9F00E9484CCC0916D076C2E85E0782EA3
:10A870007C0E04E413E89AE2A92E94E0B92ED5E008
:10A88000DC1B26E1E22E23E8F22E84E0D82EDC1A2F
:10A8900083E0C82ECC1A82E0982E9C1A81E0882E84
:10A8A0008C1AC1112CC0809170078823B9F0809157
:10A8B0006A01882361F0662D619581E090917007AF
:10A8C000911180E024E04EE454E00E94D0CBCF5FB1
:10A8D000C711E7CF86E080936E070CC080915707C1
:10A8E00010925707882319F30E942A4B80916F0713
:10A8F0008823E9F2CDB7DEB7EEE00C9415F1C13054
:10A9000049F5809170078130A1F080916A01882318
:10A91000F1F28BE593E89F938F9388E494E09F9303
:10A920008F938F9281E090917007913069F180E070
:10A930002BC08091570710925707882331F38BE57E
:10A9400093E8892B11F00E945B8380916F07882325
:10A95000E1F2D0CFC23009F08FC080917007823011
:10A96000E9F080916A01882309F4B1CF8AEC92E280
:10A970009F938F938EE394E09F938F939F9281E0B8
:10A9800090917007923099F68F930E94E2220F9077
:10A990000F900F900F900F900F9099CF80915707C5
:10A9A000109257078823E9F20E94CA2280916F070C
:10A9B0008823B9F29FCF809170078330A9F08091EE
:10A9C0006A01882309F483CF8DE293E89F938F93E4
:10A9D00087E394E09F938F93CF9281E090917007EB
:10A9E000933009F0A4CFD0CF80915707109257072A
:10A9F000882329F38DE293E8892B11F00E942D839F
:10AA000080916F078823D9F275CF809170078430C9
:10AA100099F080916A01882309F459CFFF92EF924F
:10AA200082E394E09F938F93DF9281E0909170078F
:10AA3000943009F07CCFA8CF809157071092570728
:10AA4000882339F3E114F10411F00E9416838091F8
:10AA50006F078823F1F24ECF809157071092570766
:10AA60008823B1F00115110511F00E9444838091F3
:10AA70006F07882369F03ECFC33009F49CCFC43000
:10AA800021F2C53009F023CF80917007853021F382
:10AA900080916A01882309F41ACF1F930F93BF9204
:10AAA000AF92DF9381E090917007953009F03FCF2E
:10AAB0006BCF80E090E0A0E8B0E480937D019093BC
:10AAC0007E01A0937F01B09380018AE192E00E9411
:10AAD00050228091EB030E94CA7910929A020C9442
:10AAE0002A4BB0E0A0E0E7E7F5E50C94FEF00E9409
:10AAF00084CCC0916D0785E0C82ECC0ED4E0DC1B61
:10AB000013E01C1B82E0F82EFC1A81E0E82EEC1A00
:10AB1000BC2EB194C1112BC0809170078823B1F075
:10AB200080916A01882359F081E09091700791111A
:10AB300080E024E045E553E06B2D0E94D0CBCF5F51
:10AB4000CC12E8CF85E080936E070CC08091570748
:10AB500010925707882321F30E942A4B80916F0798
:10AB60008823F1F2CDB7DEB7E9E00C941AF1C130D9
:10AB700089F5809170078130C1F080916A01882346
:10AB8000F1F2DD24D39480917007813009F0D12C4B
:10AB900085E89DE00E94111E00E09C014AE453E01C
:10ABA0006E2D8D2D0E947375CACF8091570710921C
:10ABB0005707882311F30E9478CC4DEA5CE265E8E0
:10ABC0007DE08AE493E00E94E9CC80916F078823BE
:10ABD000A1F2C8CFC23009F073C0809170078230F3
:10ABE000B1F080916A01882309F4A9CFDD24D394C0
:10ABF00080917007823009F0D12C89E89DE00E9495
:10AC0000111E00E09C014FE353E06F2DCACF8091ED
:10AC1000570710925707882321F30E9478CC4CEAFB
:10AC20005CE269E87DE08FE393E00E94E9CC8091EB
:10AC30006F078823B1F296CF809170078330B1F00F
:10AC400080916A01882309F47ACFDD24D39480911E
:10AC50007007833009F0D12C8DE89DE00E94111E11
:10AC600000E09C0144E353E0612F9BCF80915707A4
:10AC700010925707882321F30E9478CC4BEA5CE2BC
:10AC80006DE87DE084E393E00E94E9CC80916F075A
:10AC90008823B1F267CF8091570710925707882316
:10ACA000C9F00E9478CC4AEA5CE261E97DE089E281
:10ACB00093E00E94E9CC80916F07882359F052CF2E
:10ACC000C33009F4B9CFC43009F039CF809170078F
:10ACD000843009F380916A01882309F430CFDD24A0
:10ACE000D39480917007843009F0D12C81E99DE0E4
:10ACF0000E94111E00E09C0149E253E06D2F51CFEC
:10AD0000A3E0B0E0E6E8F6E50C94F5F04C013B0179
:10AD10005A011901280181E080939A02409172073B
:10AD20005091730760917407709175074115510533
:10AD30006105710571F0141615060CF080E0809322
:10AD4000E903109272071092730710927407109221
:10AD500075071091E903809157078B83109257076D
:10AD6000811105C080916A01882309F46FC0C20176
:10AD70000E94C56E082F80E0C114D10419F0C601ED
:10AD80000E94C56E1A821982E114F104B1F4402FB9
:10AD900050E0282F30E0CA01820F931F46976CF4D1
:10ADA00085E190E0841B950B821B930B97FD019628
:10ADB000959587958A8381E0898301E025EC38E6C3
:10ADC000A201BE016F5F7F4FCE0102960E941D70EF
:10ADD000E114F10491F08A81882321F01A8289819B
:10ADE0008F5F898300E028EC38E6A701BE016F5F22
:10ADF0007F4FCE0102960E941D70C114D10459F0FC
:10AE000000E025EC38E6A601BE016F5F7F4FCE0162
:10AE100002960E941D7041E04127B30181E00E942B
:10AE200087D3C4010E94C56E412FB40194E1981BE1
:10AE3000892F0E9487D3EB81EE2341F0111101C0CD
:10AE40005101A114B10431F0F50109952396E2E115
:10AE50000C9411F10E942A4BF9CFCF92DF92EF921E
:10AE6000FF920F931F938EE9C82E85E0D82EF12C08
:10AE7000E12C00EA15E030E020E049ED56E460EB1B
:10AE800075E085EB95E03CDF1F910F91FF90EF900F
:10AE9000DF90CF900895B0E0A0E0E1E5F7E50C94F5
:10AEA000FDF0ADB6BEB680912B1062E877E0882346
:10AEB00011F06BE270E1FB0101900020E9F7CF0196
:10AEC000861B970B01962DB73EB7281B390B0FB683
:10AED000F8943EBF0FBE2DBF8DB79EB701967C0183
:10AEE00080E2EDB7FEB78183C70101960E9451F35E
:10AEF0008AE5C82E85E0D82E0CE515E030E020E08C
:10AF000043EA57E468E675E08FE695E0F9DE0FB6B0
:10AF1000F894BEBE0FBEADBEEAE00C9419F1CF921C
:10AF2000DF92EF92FF920F931F9388EBC82E84E07D
:10AF3000D82EF12CE12C0BE215E030E020E048E8BF
:10AF400055E66AEB74E08FEB94E0DADE1F910F9127
:10AF5000FF90EF90DF90CF900895CF92DF92EF9225
:10AF6000FF920F931F938AE8C82E83E0D82EF12C0E
:10AF7000E12C0CE813E029E535E548E552E268E903
:10AF800073E08DE993E0BCDE1F910F91FF90EF908D
:10AF9000DF90CF900895B0E0A0E0E1EDF7E50C94EC
:10AFA000FDF0ADB6BEB683E392E00E94C56E90E0C0
:10AFB00001962DB73EB7281B390B0FB6F8943EBF4C
:10AFC0000FBE2DBF8DB79EB701967C0163E372E083
:10AFD0000E9457E98091300700E012E0813031F0A3
:10AFE0000BEE11E0823011F003E112E084E2C82E92
:10AFF00082E0D82E27E937E448E053E666E272E0C3
:10B000008DE292E07DDE0FB6F894BEBE0FBEADBEFF
:10B01000EAE00C9419F18F929F92AF92BF92CF9277
:10B02000DF92EF92FF920F9380915707109257078C
:10B03000882371F010929A020E942A4B0F91FF9080
:10B04000EF90DF90CF90BF90AF909F908F9008953A
:10B0500081E080939A028091720790917307A0918A
:10B060007407B09175070097A105B10509F44AC0AE
:10B070005C01AA0CBB1CAA0CBB1C1092720710929C
:10B0800073071092740710927507B5010B2C000C12
:10B09000880B990B0E9415EA2091B8073091B907E7
:10B0A0004091BA075091BB070E9474EA20915E1349
:10B0B00030915F1340916013509161130E942DF104
:10B0C0006B017C0120E030E040EA51EC0E9490F2FC
:10B0D00087FD18C020E030E040EA51E4C701B60126
:10B0E0000E940FEA181674F0C5010E94FEC7C092B4
:10B0F0005E13D0925F13E0926013F092611382E0CE
:10B1000080936A0180916A01882309F497CFC090E7
:10B110005E13D0905F13E0906013F090611320E015
:10B1200030E44CE156E4C701B6010E9474EA4B01D9
:10B130005C0120E030E0A901C701B6010E940FEADE
:10B1400020E030E040EA50E487FF04C020E030E037
:10B1500040EA50ECC501B4010E942DF12DEC3CEC0D
:10B160004CEC5DE30E9474EA0E940CF26B017C01DE
:10B170008BE2F7FE09C0F094E094D094C094C11C17
:10B18000D11CE11CF11C8DE280939B02C701B6012A
:10B1900020E137E240E050E00E945FF06AE0862E56
:10B1A000912CA12CB12CCA01B901A50194010E94D6
:10B1B0005FF0605D60939C02C701B60128EE33E04A
:10B1C00040E050E00E945FF0CA01B901A50194017E
:10B1D0000E945FF0605D60939D028EE280939E020C
:10B1E000C701B60124E630E040E050E00E945FF085
:10B1F000CA01B901A50194010E945FF0605D6093EE
:10B200009F02C701B601A50194010E945FF06B0186
:10B21000CA01B901A50194010E945FF0605D6093CD
:10B22000A00260E36C0D6093A1026BE972E084EF11
:10B2300092E00E940C75C0905E13D0905F13E09076
:10B240006013F09061138090E5039090E603A09066
:10B25000E703B090E803A5019401C701B6010E947D
:10B260000FEA8823E9F020E030E0A901C701B60128
:10B270000E940FEA882309F479C0A5019401C7014F
:10B28000B6010E940FEA87FD73C081E08093E4035A
:10B29000C092E503D092E603E092E703F092E80360
:10B2A000D090E4038091C713813188F48091C91351
:10B2B000833068F044E04D195CEDE52E52E0F52E48
:10B2C0000CE022E062E483E993E10E94C3D4809120
:10B2D000C713853180F48091C913843160F049ED42
:10B2E000E42E42E0F42E01E023E044E16CE383E944
:10B2F00093E10E94C3D48091C7138F3308F09ECE90
:10B300008091C9138F3208F499CE40E34D198FEB29
:10B31000E82E82E0F82E0DE022E06AE583E993E171
:10B320000E94C3D441E34D1995EAE92E92E0F92E2B
:10B3300022E065E083E993E10E94C3D425E7E22E91
:10B3400022E0F22E00E123E04FE262E183E993E1A3
:10B350000E94C3D435E4E32E32E0F32E23E04FE223
:10B3600067E683E993E10E94C3D468CE80E08ECF84
:10B370008FEF8CCF0F931F93CF93DF93FC01EB01E3
:10B380008091720790917307A0917407B09175072F
:10B39000B7FF08C0109272071092730710927407DB
:10B3A000109275078091610790916207A0916307E1
:10B3B000B0916407409172075091730760917407D0
:10B3C0007091750784179507A607B70744F4809313
:10B3D000720790937307A0937407B09375078091D9
:10B3E0006A018823E1F06091720770917307809180
:10B3F0007407909175070091650710916607209179
:10B40000670730916807600F711F821F931F0995AE
:10B41000BC0180916B0790916C070E940C75809124
:10B420005707811108C080915E078823A9F1809198
:10B430006A01882389F18091690790916A070097D2
:10B44000B1F0409172075091730760917407709149
:10B450007507009165071091660720916707309185
:10B460006807400F511F621F731FFE010995E0918D
:10B470005F07F0916007309741F080915E0781117E
:10B4800003C0809157078111099580915707109249
:10B49000570781110E942A4BDF91CF911F910F9185
:10B4A000089567E17DE180E39DE164CF64E97DE19A
:10B4B00080E995E45FCF62EA7DE185EC9EE15ACFB9
:10B4C00066EB7DE18AEC9DE155CF63E07EE18CEA9D
:10B4D00095E450CFE091DD03E63028F581E08E0F52
:10B4E0008093DD0340917207509173076091740758
:10B4F0007091750720916D0790916E0780919A0267
:10B5000039E0E39FF0011124E955FC4FA0918D1320
:10B51000B0918E13B183A083428353836483758378
:10B520002683978380870895A7E0B0E0EAE9FAE5EB
:10B530000C94F5F00E9484CCF0906D072F2C85E0E0
:10B540008F0D8D833324339483E0E82E98EE892E7B
:10B5500093E0992EA12CB12C84E08F198E839E2D1F
:10B560009F199F8382E0D82EDF18C32CCF18F110CB
:10B570002CC0809170078823C1F080916A018823D4
:10B5800061F0622D619581E090917007911180E0EA
:10B5900024E045E553E00E94D0CBF3949D81F9125D
:10B5A000E6CF85E080936E070CC08091570710921C
:10B5B0005707882311F30E942A4B80916F07882335
:10B5C000E1F22796E2E10C9411F181E0F8122DC02E
:10B5D000909170079130B9F080916A018823E9F267
:10B5E00081E0913009F080E090919C032DE133E0FF
:10B5F000911102C029E133E001E040E253E06C2DFB
:10B600000E947375CACF80915707109257078823FD
:10B6100019F380919C038F2580939C03E0926A012B
:10B6200080916F078823C1F2CCCF92E0F912D1C08C
:10B6300080917007823021F180916A01882309F49A
:10B64000ACCF11E080917007823009F010E060917A
:10B65000060170910701072E000C880B990B0E94C0
:10B6600015EA69837A838B839C83CE0101960E94BD
:10B67000A34500E09C0142E153E06D2D812FC0CF36
:10B6800080915707109257078823B1F210E000E02D
:10B6900025EF30E050E040E066E071E082E193E0C9
:10B6A0000E9449CD80916F07882331F28ACF809123
:10B6B0007007833019F180916A01882309F46DCFF6
:10B6C00011E080917007833009F010E0609104016F
:10B6D00070910501072E000C880B990B0E9415EA4A
:10B6E00069837A838B839C83CE0101960E94A34554
:10B6F00000E09C014BE053E06F81C0CF8091570781
:10B70000109257078823B9F210E000E025EF30E0EF
:10B7100050E040E064E071E08BE093E00E9449CDAE
:10B7200080916F07882339F24CCF80915707109290
:10B730005707882309F459C020E030E048EC52E470
:10B7400060910001709101018091020190910301CB
:10B750000E9474EA0E9411F22B0130926F07BADE48
:10B76000E0926A0183E093E090936C0780936B070B
:10B7700080E091E090936A078093690710926507D3
:10B78000109266071092670710926807809261070F
:10B7900090926207A0926307B0926407712C612CAB
:10B7A0004092720750927307609274077092750707
:10B7B00080E69AE590938E1380938D131092600724
:10B7C00010925F0710925E0780916F07882369F0DF
:10B7D000F8CE83E0F81609F46ACF94E0F912DDCED2
:10B7E00080917007843009F4A0CF80916A0188238A
:10B7F00009F4D3CE11E080917007843009F010E095
:10B80000409000015090010160900201709003018E
:10B8100020E030E0A901C301B2010E940FEA2DEB44
:10B8200037E346E055EB87FD04C02DEB37E346E0F8
:10B8300055E3C301B2010E942DF169837A838B83A2
:10B840009C83CE0101960E94A11B00E09C0143E075
:10B8500053E06E8113CFB0E0A0E0E1E3FCE50C948F
:10B8600005F18D8190919C10891778F080939C1040
:10B870009E01285F3F4F4E815F8164E570E087E461
:10B8800090E10E94D7E910924610E2E00C9421F179
:10B890000F931F93CF93DF936F3F11F410929C107F
:10B8A00020919C1021111EC08C010E945EE9800F26
:10B8B000911FEC01C01BD10BC535D1053CF00197A0
:10B8C000FC012491207C2038D1F3F3CFDD27AE0199
:10B8D000B80187E490E10E947FE9C95BDF4E1882DE
:10B8E00010924610DF91CF911F910F910895A6E815
:10B8F000B0E0EDE7FCE50C9400F1C358DF4F18828F
:10B9000019821A821B82CD57D04080918E0290916D
:10B910008F02A0919002B0919102CF57DF4F8883A0
:10B920009983AA83BB83C158D04084E690E090936A
:10B93000A6128093A5121092CA121092C9121092E8
:10B940001A0464E070E0CE018F579F4F0E94ACD084
:10B950008091A5129091A61202969093A6128093C0
:10B96000A5121092CA121092C91281E0CA57DF4F75
:10B970008883C658D040CE018A579F4F0E943922F3
:10B9800068E470E081E79DE00E94ACD080E1E1E9ED
:10B99000F1E08E010F5F1F4FD80101900D928A9543
:10B9A000E1F760E170E0C8010E94ACD083E997E064
:10B9B0000E9441228CE0F80111928A95E9F7C801B2
:10B9C0000E943D227E01FDE6EF0EF11C8FEFF70194
:10B9D0008083C7010E94392219821A821B821C822D
:10B9E000C8010E9441228091B4029091B502A091B9
:10B9F000B602B091B70289839A83AB83BC83C80136
:10BA00000E944122C358DF4F188219821A821B827A
:10BA1000CD57D04083E0F70180838983CE018358DE
:10BA20009F4F0E944122C7010E943922C8010E94F3
:10BA300039222AE0D22EDA94DD2031F0CE0183586B
:10BA40009F4F0E944122F7CF86E593E10E943D225D
:10BA5000C358DF4F188219821A821B82CD57D040FB
:10BA60009AE0D92EDA94DD2031F0CE0183589F4F31
:10BA70000E944122F7CF87E08983F7018083C801C4
:10BA80000E943922C7010E94392268E070E084E8F0
:10BA900093E00E94ACD068E070E08CE793E00E94F5
:10BAA000ACD064EC70E088EB92E00E94ACD01982DC
:10BAB000DD24DA94F701D082C8010E943522C70143
:10BAC0000E94392264E070E082E292E00E94ACD0F1
:10BAD0008091EB068983C8010E9435226CE070E0FA
:10BAE0008BE497E00E94ACD0198A1A8A1B8A1C8AC0
:10BAF00080E090E0A0E8BFE38D879E87AF87B88B9A
:10BB00008091BD129091BE12A091BF12B091C0124F
:10BB100089839A83AB83BC8320E030E543EC50E417
:10BB20006091C1127091C2128091C3129091C4129F
:10BB30000E9474EA6D837E838F8398872CEA35ECAC
:10BB400047E25EE36091C5127091C6128091C71200
:10BB50009091C8120E9474EA69877A878B879C87C4
:10BB600064E170E0C8010E94ACD084E190E09A8367
:10BB7000898362E070E0C8010E94ACD080913F07E9
:10BB800090914007A0914107B091420789839A8321
:10BB9000AB83BC8320E030E543EC50E46091430785
:10BBA0007091440780914507909146070E9474EA7E
:10BBB0006D837E838F8398872CEA35EC47E25EE3C2
:10BBC00060914707709148078091490790914A0713
:10BBD0000E9474EA69877A878B879C87C8010E94D4
:10BBE00031228CE0E1EAF1E0D80101900D928A95D2
:10BBF000E1F7C8010E9431221982C8010E9439224E
:10BC00008FE78983C8010E943922D982C8010E9426
:10BC1000392285E0EDEAF1E0D80101900D928A9594
:10BC2000E1F765E070E0C8010E94ACD01982C8015C
:10BC30000E94352280E2E2EBF1E0D80101900D9202
:10BC40008A95E1F760E270E0C8010E94ACD0F7018C
:10BC50001082C7010E9435221982C8010E94352234
:10BC600080E090E0A0EEBFE3C358DF4F8883998364
:10BC7000AA83BB83CD57D040CE0183589F4F0E94EB
:10BC80004122C358DF4F188219821A821B82CD5776
:10BC9000D040CE0183589F4F0E94412282E1F8019B
:10BCA00011928A95E9F762E170E0C8010E94ACD078
:10BCB00084E2E2EDF1E0D80101900D928A95E1F77E
:10BCC00064E270E0C8010E94ACD080E1F8011192FA
:10BCD0008A95E9F760E170E0C8010E94ACD089E084
:10BCE000F80111928A95E9F769E070E0C8010E94B5
:10BCF000ACD0C358DF4F188219821A821B82CD57ED
:10BD0000D040CE0183589F4F0E9441228CE0D82E14
:10BD1000F8018D2D11928A95E9F76CE070E0C80169
:10BD20000E94ACD08CE6F80111928A95E9F76CE696
:10BD300070E0C8010E94ACD08EE094E00E943122F5
:10BD4000F7011082118212821382148215821682E8
:10BD5000178268E070E0C7010E94ACD0F701119231
:10BD6000DA94E9F7CB57DF4F1882C558D04080E00E
:10BD700090E0A0E4B0E4ED968CAF9DAFAEAFBFAF66
:10BD8000ED97C7010E943D22CE018B579F4F0E9425
:10BD90003922CE0187589F4F0E94412280911A0478
:10BDA000811127C00091A5121091A6128091C9128D
:10BDB0009091CA12F7019183808384E690E090937A
:10BDC000A6128093A51264E070E086E292E00E94E1
:10BDD000ACD062E070E0C7010E94ACD091E00037C7
:10BDE000F3E01F0709F490E080911A04892B8093F7
:10BDF0001A0480911A04811104C060E08BE39AE078
:10BE000047DD90911A0481E08927CA57DF4FE7E0A8
:10BE10000C941CF16CDD0C944746A7E0B0E0E3E124
:10BE2000FFE50C94F5F080917F07877089838090FF
:10BE3000840390908503A0908603B09087030E94AE
:10BE400084CC20916D072E833981373009F075C07D
:10BE500085E194E09B838A831E81312F3B5F3C8385
:10BE600033243394812F81958D83232C211A84E6EA
:10BE7000482E512C612C712C2E81222309F462C092
:10BE80003981373009F433C22E81213009F028C2BC
:10BE900090917007913009F445C180916A01811138
:10BEA00054C182E0F82E81E08F0D8F839981973005
:10BEB00009F063C020E030E0A901C501B4010E948F
:10BEC0000FEA882309F459C03F818E81381331C0AD
:10BED0009091B3029F83809170072E81821311C0CD
:10BEE0008091570710925707882359F093259F8315
:10BEF00083E080936A010E94452280916F0781113F
:10BF00000DC180916A018823A1F06E81611B81E0DF
:10BF1000909170073E81931380E09F8126EF33E07C
:10BF2000911102C022EF33E001E049EF53E00E949B
:10BF30007375F394F394FF8220C020E134E03B83D7
:10BF40002A838ACF80917007882309F4D9C0809111
:10BF50006A01882309F494CF81E0909170079111D0
:10BF600080E024E043E254E06D810E94D0CB8981DF
:10BF7000873009F41DC193E09F838091B4029091B2
:10BF8000B502A091B602B091B702809330079093AA
:10BF90003107A0933207B09333072F813E812313DB
:10BFA0001EC080917007821709F407C180916A0151
:10BFB0008823A9F0EE80E11AFF24F39480917007A2
:10BFC0003E818313F12C80E397E00E94534500E00B
:10BFD0009C0146EE53E06E2D8F2D0E9473758F816C
:10BFE0008F5F9E81891316C080917007891709F4AD
:10BFF00038C180916A01882369F06E81611B81E0FC
:10C00000909170072E81921380E023E047ED53E07A
:10C010000E94D0CB8F818E5F3E81831316C08091AA
:10C020007007831709F42EC180916A01882369F093
:10C030006E81611B81E0909170072E81921380E0E8
:10C0400023E04AEC53E00E94D0CB8F818D5F3E818C
:10C05000831323C080917007831709F424C1809152
:10C060006A018823D1F088E29BE49F938F938CEB45
:10C0700093E09F938F938E81811B8F9381E09091AA
:10C0800070073E81931380E08F930E94E2220F900D
:10C090000F900F900F900F900F908F818C5F9E816B
:10C0A000891323C080917007891709F40BC180910F
:10C0B0006A018823D1F08AE09FE59F938F938DEAF0
:10C0C00093E09F938F938E81811B8F9381E090915A
:10C0D00070072E81921380E08F930E94E2220F90CE
:10C0E0000F900F900F900F900F903E813F5F3E8317
:10C0F0008C818313C1CE9F819B5F90936E070EC08E
:10C100008091570710925707882309F420CF0E9487
:10C110002A4B80916F07882309F419CF2796E2E113
:10C120000C9411F18091570710925707882309F456
:10C13000B4CE20EF35E03093ED062093EC068091ED
:10C140006F07882309F4A9CEE9CF81E0913009F087
:10C1500080E020E249E154E0622D0E94D0CBA1CEE4
:10C16000909170073E81931731F080916A0181119F
:10C1700013C08E8197CE809157071092570788235E
:10C18000A1F32A813B813093ED062093EC06809148
:10C190006F07882351F3C2CF6E81611B81E03E811E
:10C1A000931380E020E246E054E00E94D0CBE1CF40
:10C1B00022E02F83FF24F3947DCE809157071092C5
:10C1C0005707882309F4F2CE0E9478CC609130079B
:10C1D0007091310780913207909133070E9411F2DC
:10C1E0006B0130926F0776D983E080936A0186EE07
:10C1F00093E090936C0780936B0720E337E03093D4
:10C200006A072093690710926507109266071092DB
:10C210006707109268074092610750926207609228
:10C22000630770926407F12CE12CC0927207D092E0
:10C230007307E0927407F092750786E59AE590938C
:10C240008E1380938D132BE432E23093600720939A
:10C250005F0710925E0780916F07882309F4A6CECE
:10C260005DCF8091570710925707882309F4C1CEFC
:10C270008BE098E50E94DACC80916F07882309F45F
:10C28000B8CE4CCF8091570710925707882309F4F6
:10C29000CBCE89E597E40E94DACC80916F078823A2
:10C2A00009F4C2CE3BCF80915707109257078823DD
:10C2B00009F4D5CE0E94284B80916F07882309F49A
:10C2C000CECE2CCF8091570710925707882309F4C0
:10C2D000EECEA0DD80916F07882309F4E8CE1ECF53
:10C2E0002E81223009F43CCF33E03F8346CE8E814D
:10C2F000813009F435CF92E09F835CCFA3E0B0E0BA
:10C30000E4E8F1E60C94F5F00E942723582E0E94F1
:10C3100084CC20916D072A83422E2B5F2B8383E0F0
:10C32000782E74180CE514E028E2E22E2BE4F22EAD
:10C330003DE6C32E34E0D32E4AE0A42E4FE5B42EC2
:10C340005BE7852E54E0952E82E08419898381E095
:10C35000382E3418242C21948A8181118EC080912A
:10C360007007882309F477C080916A01882359F007
:10C3700081E090917007911180E024E043EB54E05C
:10C38000622D0E94D0CB51103DC18A81833009F0CB
:10C3900029C180917007833009F4C3C080916A017C
:10C3A0008111D0C084E0682E81E0860D51104AC012
:10C3B0009A8189131FC080917007891709F4F4C00E
:10C3C00080916A018823B1F0FF92EF92DF92CF92C1
:10C3D0008A8184198F9381E0909170072A8192134A
:10C3E00080E08F930E94E2220F900F900F900F90A9
:10C3F0000F900F9082E0860D9A81891321C0809161
:10C400007007891709F4DFC080916A018823C1F0A1
:10C4100088E596E49F938F931F930F938A818419E5
:10C420008F9381E0909170072A81921380E08F931F
:10C430000E94E2220F900F900F900F900F900F909C
:10C4400083E0860D9A819F5F9A832B81291384CF85
:10C4500080936E070EC0809157071092570788236C
:10C4600009F482CF0E942A4B80916F07882309F438
:10C470007BCF2396E2E10C9411F19A81913051F532
:10C48000809170078130B9F080916A01882309F4A6
:10C490007ACF81E090917007913009F080E023E03D
:10C4A00041EA54E0632D0E94D0CB5110ABC085E02F
:10C4B00094E0692E7DCF809157071092570788230B
:10C4C00019F382E993E50E94DACC80916F07882303
:10C4D000D9F2CFCF2A81223009F055CF8091700751
:10C4E000823081F080916A01882309F44CCF81E089
:10C4F00090917007923009F080E023E042E954E027
:10C500006981D1CF8091570710925707882351F343
:10C510008BE098E50E94DACC80916F07882311F3B5
:10C52000A8CF8091570710925707882309F436CF78
:10C530008BE294E50E94DACC80916F07882309F49E
:10C540002DCF97CF81E090917007933009F080E074
:10C5500023E04AE854E0672D0E94D0CB23CF80919E
:10C56000570710925707882309F446C053DC80917F
:10C570006F07882309F440C07CCFBF92AF929F928F
:10C580008F928A8184198F9381E0909170072A811C
:10C59000921380E08F930E94E2220F900F900F90F1
:10C5A0000F900F900F902CC0809157071092570753
:10C5B000882309F405CF0E94284B80916F078823B8
:10C5C00009F4FECE56CF8091570710925707882363
:10C5D00009F41ACF0E94584680916F07882309F406
:10C5E00013CF47CF8A81843009F061CF80917007E3
:10C5F0009A81891709F4B3CF80916A018111BDCF67
:10C600008A81D1CE9A8184E0933009F01BCFEECF9E
:10C610000E94EA406CD90E9447460C949747CF93FA
:10C6200080919F03811109C08CED91E09093E30309
:10C630008093E20381E080939F030E946A5A20E086
:10C6400040E070E060E082E393E20E945B46C1E07C
:10C65000C0939A020E94AE2C0E942A4BC0939A0269
:10C6600060E08AEA9DE214D988ED91E09093ED06AE
:10C670008093EC06CF910895A6E0B0E0E2E4F3E603
:10C680000C94F5F00E94AA7B382E8091E51484FB6F
:10C69000662460F8412C84FF03C00E94BD7B482EB5
:10C6A0000E9484CC20916D072D83522E2B5F29830D
:10C6B00080E009E115E091E0792E7518952D9195AE
:10C6C0009A839FE0E92E93E6F92E26E3C22E25E019
:10C6D000D22E92E095199B8393E095199C8335EDBA
:10C6E000832E34E0932E4AEEA42E44E0B42E9D8196
:10C6F0002981921709F409C2992349F131106AC0BE
:10C700000E940082882309F47AC19D81913009F446
:10C7100044C122E02E832D818E8128135FC1809138
:10C720007007281709F46EC180916A01882309F403
:10C7300055C16D81651981E0909170072D8192132B
:10C7400080E023E042E155E00E94D0CB47C18091D8
:10C750007007882379F180916A01882379F281E05A
:10C7600090917007911180E024E042E455E06A81E5
:10C770000E94D0CB332021F224E02E839D812E8194
:10C7800092134AC080917007981709F44CC18091A8
:10C790006A01882309F440C06D81651981E0909198
:10C7A00070072D81921380E023E046E055E00E945F
:10C7B000D0CB32C08091570710925707882359F287
:10C7C0000E942A4B80916F07882329F22696E2E186
:10C7D0000C9411F18D81813009F47FC0823009F40D
:10C7E000A6C09D81933041F680917007833009F493
:10C7F000C3C080916A01882309F4BECF81E0909183
:10C800007007933009F080E023E046E255E06C8148
:10C810000E94D0CB84E08E838E818F5F9D819813A0
:10C8200016C080917007981709F40EC180916A01B3
:10C83000882369F06D81651981E0909170072D81E1
:10C84000921380E023E048EF54E00E94D0CB8E8129
:10C850008E5F662009F430C141103BC09D81981362
:10C860001BC020907007921509F4FFC080916A01E7
:10C87000882391F01F92BF92AF928D8185198F937B
:10C8800081E02D81221180E08F930E94E2220F909F
:10C890000F900F900F900F908E818D5F9D81981358
:10C8A00016C080917007981709F4F5C080916A014D
:10C8B000882369F06D81651981E0909170072D8161
:10C8C000921380E023E049ED54E00E94D0CB8E81AA
:10C8D0008C5F9D819F5F9D830ACF8091700781301F
:10C8E000D1F080916A01882309F446CFFF92EF923C
:10C8F000DF92CF927F9281E090917007913009F0A2
:10C9000080E08F930E94E2220F900F900F900F9083
:10C910000F900F9031CF80915707109257078823BF
:10C9200001F37DDE80916F078823D9F24FCF80918C
:10C930007007823091F080916A01882309F41CCF3E
:10C9400081E090917007923009F080E023E04BE2A3
:10C9500055E06B810E94D0CB0FCF8091570710928A
:10C960005707882341F38FE897E50E94DACC80913E
:10C970006F07882301F32ACF80915707109257073A
:10C98000882309F436CF88E49BE40E94DACC8091B6
:10C990006F07882309F42DCF19CF8091700781305C
:10C9A00009F180916A01882309F4B3CE8DE494E4FF
:10C9B0009F938F931F930F937F9281E090917007C5
:10C9C000913009F080E08F930E94E2220F900F9047
:10C9D0000F900F900F900F9082E08E838E818F5F6B
:10C9E0008E83CCCE80915707109257078823C9F2C7
:10C9F0000E944D4480916F07882399F2E7CE91E021
:10CA00009E8389CE8091570710925707882309F497
:10CA10008BCE85EB9FE40E94DACC80916F07882350
:10CA200009F482CED3CE80915707109257078823FE
:10CA300009F4ADCE81E19DE40E94DACC80916F07CC
:10CA4000882309F4A4CEC2CE8091570710925707CD
:10CA5000882309F4EBCE8EE791E60E94DACC809130
:10CA60006F07882309F4E2CEB1CE80915707109268
:10CA70005707882309F4FACE4FE350E064EC74E0E2
:10CA80008EEE96E00E9466F380916F07882309F48A
:10CA9000EDCE8D811ECF80915707109257078823C6
:10CAA00009F404CF86EF96E60E94DACC80916F07F6
:10CAB000882309F4FBCEEDCF9D81981314C090918B
:10CAC00070072D81291791F080916A01882359F010
:10CAD0006D81651981E02D81291380E020E248EC09
:10CAE00054E00E94D0CB8E818D5FF3CE80915707AA
:10CAF00010925707882341F39092ED068092EC063E
:10CB000080916F07882301F3C4CF80936E075ECEB8
:10CB100010929802109269010E94BD7B9091E514D9
:10CB200080FB97F99093E51460E08AEC91E00E9415
:10CB3000485C0C9497470F931F930E9402D1009179
:10CB40009402109195022091960230919702601BF9
:10CB5000710B820B930B97FD0CC089B183FB882767
:10CB600080F991E089274A9B8260309B84608093A2
:10CB700093028091930281709091930291FD826063
:10CB800090919E03981749F0813009F148F0823066
:10CB900079F0833091F080939E031F910F91089557
:10CBA000913079F09230B9F79091920291500CC087
:10CBB000992339F09330C1F3EECF9130A9F392303D
:10CBC00051F7909192029F5F90939202E4CF992344
:10CBD00059F3933001F7F5CF1F93CF93DF938091F3
:10CBE00035018F3708F475C08F579091BC12909320
:10CBF0009E04992309F46BC05D9A90913E0790932F
:10CC00009D04992309F46FC05C9A8F5F809335016E
:10CC100080919C0491E0892780939C0481118BDF93
:10CC20008091340191E0980F85300CF090E08230D3
:10CC300009F4A8C00CF059C0882309F46EC08130F3
:10CC400009F495C090933401C0918007D091810779
:10CC5000209709F42DC0F89413B1147082E00E945B
:10CC60002D2C00C000C01C161D060CF0B9C02A9A5D
:10CC700000C000C02B9A00C0000082E090E0019745
:10CC8000F0F72B9800C000C0112309F4ABC02A9A1A
:10CC900000C000C0789480918007909181071C1695
:10CCA0001D060CF0A1C00197909381078093800727
:10CCB0008091B90D9091BA0D009729F0019790934A
:10CCC000BA0D8093B90DDF91CF911F9108955D98B2
:10CCD00094CF90919E04891708F05D9890919D04DF
:10CCE000891708F492CF5C9890CF843009F461C022
:10CCF0000CF45BC0853009F0A5CF20919B04211175
:10CD000002C080939B0480919B04815080939B047C
:10CD1000882309F497CF95E095CF809133018F5FF9
:10CD200080311CF4809333018DCF109233018091B8
:10CD30009D03811113C02091B2123091B312309330
:10CD4000B5122093B41220913407309135073093F7
:10CD500037072093360781E080939D031092B3122A
:10CD60001092B21210923507109234076BCF1092C6
:10CD70007B0087E480937C0080917A0080648093BC
:10CD80007A0060CF80917A0086FD26C040917800BD
:10CD9000509179002091B2123091B312240F351FB7
:10CDA0003093B3122093B2124DCF10927B0086E4E1
:10CDB000E1CF80917A0086FD11C0409178005091BA
:10CDC00079002091340730913507240F351F3093B7
:10CDD00035072093340736CF92E034CF94E032CF3A
:10CDE0002A9846CF2A9854CF01965ECFACE3B0E0A4
:10CDF000ECEFF6E60C94F5F080917107882369F169
:10CE00008091E51410E000E084FF23C086EE92E1FB
:10CE10000E94BE248BE1E6EEF2E1DE0191960190E4
:10CE20000D928A95E1F710E000E0BE016F5F7F4F41
:10CE3000CE0181960E9416DB18163CF4CE010196B5
:10CE40000E9421D5080F111DF0CFCE0181960E94BE
:10CE50008E261093ED030093EC030E9484CC109176
:10CE60006D07312E85E0810F8CAF212E219485E551
:10CE7000A82E8DE1B82E9BE8892E95E0992E01E031
:10CE8000011B20E9622E25E0722E111113C0809142
:10CE90007007882391F180916A01882359F081E01D
:10CEA00090917007911180E024E049E955E0622DEE
:10CEB0000E94D0CB8091E51486FF3EC01130D9F49A
:10CEC00080917007813049F180916A01882309F4CB
:10CED0003EC11F927F926F920F9381E090917007F5
:10CEE000913009F080E08F930E94E2220F900F9022
:10CEF0000F900F900F9082E04FC0809157071092D3
:10CF00005707882341F20E942A4B80916F0788239C
:10CF100011F2EC96E2E10C9411F180915707109216
:10CF20005707882389F210926D070E942DD78091B0
:10CF30006F07882349F2EDCF84FF2DC01130D9F659
:10CF4000809170078130D1F080916A01882309F4C3
:10CF5000FEC0BF92AF929F928F920F9381E090910B
:10CF60007007913009F080E08F930E94E2220F90C9
:10CF70000F900F900F900F900F90BDCF809157079B
:10CF800010925707882301F30E94551D80916F0767
:10CF90008823D1F2BECF81E090916A01992309F4F0
:10CFA000D7C0582ED12CC12C412E4318852DE0908E
:10CFB000EC03F090ED03CE14DF0408F0C9C0511269
:10CFC000A5C091E0E91AF108EC18FD0886EE92E19F
:10CFD0000E94BE248BE1E6EEF2E1DE019196019023
:10CFE0000D928A95E1F7F12CBE016F5F7F4FCE0164
:10CFF00081960E9416DB18167CF4CE0101960E94E1
:10D0000021D5882389F3EF106BC0BE016F5F7F4F7E
:10D0100082E897E00E943CD5CE0181960E948E2640
:10D020008091E5149091700785FF75C0911363C0DE
:10D030008091570710925707882309F45CC0198222
:10D040001C828091E91261E073E1882311F066EEA1
:10D0500072E121E042E857E0CE0101960E9493265A
:10D06000882309F43FC08BE1FE013196A6EEB2E1C0
:10D0700001900D928A95E1F78091E5148F7B809362
:10D08000E514A091DB14AA3080F481E08A0F80932C
:10D09000DB148BE18A9FD0011124A353BC4EE6EE32
:10D0A000F2E101900D928A95E1F7CE0101960E947E
:10D0B0008E2610926D0782E090E0A0E0B0E08093B1
:10D0C000720790937307A0937407B093750781E07C
:10D0D00080936F071092990283E080936A0119CFC1
:10D0E000F39482CF0E94C28A62E877E085E795E0F8
:10D0F0000E94FCD4DACF80916A01882339F081E064
:10D10000911380E041E0642D0E940ECC8FEFC81A8D
:10D11000D80A53944BCF911759F080916A01882314
:10D12000A9F381E090917007911380E040E0EBCF8C
:10D130008091570710925707882379F38BE497E57E
:10D140000E94DACC80916F07882339F3E2CE82E027
:10D150001F5F9CAD911399CE80936E07DACEFC01D0
:10D16000A081B1811C92A281B3818C918F5F8C933D
:10D170000280F381E02D90818CE0989F800D112436
:10D18000EFE8F3E113AE84AF0895FC0184910895B4
:10D19000FC0180810895009751F0FC0180E091919D
:10D1A000992331F0907C9038D1F38F5FF8CF80E0F5
:10D1B0000895119800C087FD43C0419800C0119A9E
:10D1C00000C000C0119800C086FD46C0419800C054
:10D1D000119A00C000C0119800C085FD3BC0419865
:10D1E00000C0119A00C000C0119800C084FD30C07A
:10D1F000419800C0119A00C000C0119800C083FD82
:10D2000025C0419800C0119A00C000C0119800C00C
:10D2100082FD1AC0419800C0119A00C000C0119848
:10D2200000C081FD0FC0419800C0119A00C000C02D
:10D23000119800C0419800C0119A00C000C0089524
:10D24000419ABCCF419AF0CF419AE5CF419ADACFCB
:10D25000419ACFCF419AC4CF419AB9CF90E080E0B4
:10D260000895CF93DF93DB01F9019C919130C1F0D8
:10D27000943080F094509C938830D1F480819181D7
:10D28000009771F0019791838083480F591FEA013D
:10D29000188206C08C3539F49C5F9C93943041F41D
:10D2A000DF91CF9108958B3339F781E08C93F8CFDC
:10D2B00020813181B9016F5F7F4F71836083420F9D
:10D2C000531FEA018883808191818F3591056CF726
:10D2D000E7CF0F931F9381E00091E1141091E214C6
:10D2E0002091E3143091E4144091DD145091DE1448
:10D2F0006091DF147091E0140417150726073707B3
:10D3000008F480E01F910F91089590E080E0089567
:10D3100020910206833021F425FD0CC024FD0CC0B1
:10D3200030E0A90102C0559547958A95E2F7CA01F8
:10D330008170089581E0089580E0089580911E062F
:10D3400084FD0BC08091200687FD07C090912106C7
:10D35000937081E019F480E0089581E008952FEB47
:10D36000280F2A3108F047C0E22FF0E080911E0616
:10D3700090911F06A0912006B091210604C0B69599
:10D38000A795979587952A95D2F780FD02C0817061
:10D390000895EC5FF94FE081EE2341F18091910710
:10D3A00090919207E80FF92FF11D808190ED980F71
:10D3B0009A3030F08E3251F4818180538A3098F463
:10D3C000F093F305E093F20581E008958D3211F0BA
:10D3D0008B3249F4818190ED980F9A3088F38E3228
:10D3E00011F48281EACFF0E0E0E0EACF1092F30599
:10D3F0001092F205E9CF80E00895CF93DF9385E4A2
:10D40000AEDF882309F188E040911E0650911F0687
:10D410006091200670912106972F9170C92F90E09E
:10D42000D92FCC0FDD1F71FB222720F930E0220F0E
:10D43000331F220F331FC22B67FB442740F9C42B35
:10D440008C2BDF91CF91089580E0DECF88DF882399
:10D4500041F081E02091F2053091F305232B09F48E
:10D4600080E00895CF93DF93C0913C07D0913D07B2
:10D47000209729F1609138077091390780913A0718
:10D4800090913B070E940CF26E5F7F4F24976C17C0
:10D490007D07ACF470939703609396030E9402D1CA
:10D4A000605A75418F4F9F4F609398037093990313
:10D4B00080939A0390939B03DF91CF9108951092EC
:10D4C00098031092990310929A0310929B03F4CF41
:10D4D000B0E0A0E0EEE6FAE60C94FEF06B01E901A4
:10D4E0004A3009F4D5C0453109F081C0DB011296FC
:10D4F000ED91FC91F28096818781139A00C0000023
:10D50000E6E2F0E03197F0F7092F182FEF2CE294C4
:10D5100020EFE22230E1B32EBF0CE80188EF49DEB4
:10D5200000C0000086E290E00197F0F7BFE1BF1570
:10D5300008F49BC08F2D807780683BDE8E2D39DE0E
:10D5400000C0000086E290E00197F0F780E831DE4D
:10D5500080E02FDE00C0000086E290E00197F0F747
:10D560008AEF27DE00C0000086E290E00197F0F726
:10D57000005F1F4F8881807F1CDE89918295807FAC
:10D5800018DEC017D107B1F700C0000086E290E0B6
:10D590000197F0F7F394E0E1EE0EFB10BECF139885
:10D5A000D6011296ED91FC9180819281980F928321
:10D5B0002181921708F09FC194819F5F948393818A
:10D5C000890F821710F08FEF820F8383458150E01F
:10D5D000440F551F70E060E0868197810E942CF314
:10D5E00081E0CDB7DEB7E9E00C941AF1DEC1FB01B2
:10D5F00002811381423309F485C108F48DC1463498
:10D6000009F475C1473409F482C14B3349F7898164
:10D610002B81D80112967C91129713963C91213060
:10D6200009F4BFC1233009F0A0C148EF480F582FBB
:10D6300091E0341708F490E031E0541708F030E03E
:10D64000492F432B61E0571708F460E0462311F49B
:10D65000932331F2FA8030E0F901E25CFD4FD08093
:10D66000265C3D4FF901E08099C180EE8F0D806806
:10D67000807F9FDD8F2D8295807F9BDD00C0000025
:10D6800086E290E00197F0F780E893DD80E861CFD3
:10D690000B9A1398399A4198099A119A139A00C0D3
:10D6A000000086E290E00197F0F788E790E0CEE98D
:10D6B000DFE0FE013197F1F70197D9F788EF79DDC7
:10D6C00000C0000086E290E00197F0F780E271DD93
:10D6D00080E06FDD00C0000086E290E00197F0F787
:10D6E00080E067DD80E865DD00C0000086E290E054
:10D6F0000197F0F780E05DDD80E15BDD00C00000B8
:10D7000086E290E00197F0F7CE010197F1F7CE01A4
:10D710000197F1F7CE010197F1F7CE010197F1F7EB
:10D72000CE010197F1F7CE010197F1F7CE010197F4
:10D73000F1F7CE010197F1F7CE010197F1F7CE0194
:10D740000197F1F7CE010197F1F7CE010197F1F7BB
:10D75000CE010197F1F7CE010197F1F72197F1F78B
:10D7600080E227DD80E425DD00C0000086E290E055
:10D770000197F0F780E21DDD80E61BDD00C00000B0
:10D7800086E290E00197F0F7D0E0C0E08C2F807740
:10D7900080680FDD8D2F0DDD00C0000086E290E077
:10D7A0000197F0F780E805DD80E003DD00C00000B0
:10D7B00086E290E00197F0F78AEFFBDC00C0000002
:10D7C00086E290E00197F0F780E2119800C041985E
:10D7D00000C0119A00C000C0119800C0419800C05C
:10D7E000119A00C000C0119800C0419800C0119A61
:10D7F00000C000C0119800C0419800C0119A00C03C
:10D8000000C0119800C0419800C0119A00C000C02B
:10D81000119800C0419800C0119A00C000C0119832
:10D8200000C0419800C0119A00C000C0119800C00B
:10D83000419800C0119A00C000C0119800C04198E2
:10D8400000C0119A00C000C0119800C0419800C0EB
:10D85000119A00C000C0119800C0419800C0119AF0
:10D8600000C000C0119800C0419800C0119A00C0CB
:10D8700000C0119800C0419800C0119A00C000C0BB
:10D88000119800C0419800C0119A00C000C01198C2
:10D8900000C0419800C0119A00C000C0119800C09B
:10D8A000419800C0119A00C000C000C00000E6E22C
:10D8B000F0E03197F0F7815009F087CF88EF79DCFD
:10D8C00000C0000086E290E00197F0F7CF5FD05FE4
:10D8D000C03209F05BCF80E06CDC80EC6ADC00C019
:10D8E000000086E290E00197F0F7139879CEF801F6
:10D8F0008581888375CE80E0CDB7DEB7E9E00C94F2
:10D900001AF153C0B901C8010E9400D269CED801F2
:10D9100011968C91888364CE443191F0473109F09F
:10D920005FCE1882D80112968C9112978983159632
:10D930008C91159781508A8313968C918B8350CE4E
:10D94000D80115964C91159750E0440F551F70E083
:10D9500060E016968D919C910E942CF3F801128242
:10D9600080818150838314823BCE381708F438CEEF
:10D97000871708F435CEFA80E12CD12C243070F4CE
:10D980006ACEBE01C8010E9400D2898198819D0D96
:10D9900098838E0D8983FF0C09F422CEF7FEF6CF13
:10D9A000F0CF58E0580F482F43CEEF92FF920F93DD
:10D9B0001F93CF93DF93EC018B017A018A859B85BE
:10D9C0008617970731F0888199810E94EDD31B87D4
:10D9D0000A87B701888199810E9446CC2E813F81B8
:10D9E000820F932F911D9F838E8390E080E0CDB7AF
:10D9F000DEB7E6E00C941DF1B0E0A0E0E2E0FDE669
:10DA00000C94FDF0EC017B018A018A859B858617C9
:10DA1000970731F0888199810E94EDD3FB86EA86D1
:10DA200088859985019609F5CC80DA808E81D80E9B
:10DA3000A880B980D5015596ED91FC91C501099555
:10DA4000C80E780110E0F70121917F0121111FC05C
:10DA50008E819F81810F911D9F838E8390E080E056
:10DA6000CDB7DEB7EAE00C9419F1EE80FF80B80183
:10DA7000888199810E9446CC8E0D9F2D911D28850D
:10DA800039852817390780F681E090E0E9CF4C2DE1
:10DA90006D2DC5010E9445D4D80E180FD4CFB0E02B
:10DAA000A0E0E5E5FDE60C9400F1EC01D62E1CADFE
:10DAB0000BAD7C0184E0E80EF11CE98DFA8DC70105
:10DAC0000995412F480F2D2D602FC7010E9445D485
:10DAD0009BAD890F8BAF81E090E0CDB7DEB7E7E07B
:10DAE0000C941CF1682F70E090E080E00C9463B31C
:10DAF0008091F2059091F305009731F04AE050E0F3
:10DB000070E060E00C9430E860E070E0CB010895D4
:10DB10008091F2059091F305009731F04AE050E0D2
:10DB200070E060E00C9403E760E070E0CB010895E2
:10DB3000EFDF97FD0AC0ECDF6F3F710581059105AE
:10DB400009F02CF4E5DF862F089580E008958FEF2B
:10DB50000895CF93C62F7ADC882311F0E9DFC82F10
:10DB60008C2FCF9108958091F2059091F305892B28
:10DB700039F0DEDF91E0811101C090E0892F089536
:10DB800091E0FCCFCF93DF93C82FD62F5FDC8823A3
:10DB900021F0E9DFDF91CF9108958C2FE0DB811137
:10DBA000F9CF8D2FF7CFB4DFCB010895CF93DF935B
:10DBB000EB014CDC882311F0F6DFEC01CE01DF91A4
:10DBC000CF9108950F931F93CF938091F205909179
:10DBD000F3050097D9F0FC018F01C1912C2F2F7D07
:10DBE00081F0C53411F0C536B9F7F801108270E044
:10DBF00060E00E94ADE5F801C083CF911F910F91C5
:10DC0000089570E060E00E94ADE5F7CF60E070E05D
:10DC1000CB01F3CFCF92DF92EF92FF926A017B01AB
:10DC200015DC882319F0CEDF6B017C01C701B6013A
:10DC3000FF90EF90DF90CF900895CF92DF92EF9218
:10DC4000FF92CF93C82F0E9402D16B017C0124EA7E
:10DC500030E74DE75FE36091080170910901809121
:10DC60000A0190910B010E940FEA87FD18C08AEF0C
:10DC700090E0A0E0B0E08C0D9D1DAE1DBF1D809317
:10DC80005F0690936006A0936106B0936206C0930E
:10DC90005D01CF91FF90EF90DF90CF90089580E0ED
:10DCA00090E0DC01E8CFCF9380912E06811154C023
:10DCB0001092CA131092CB131092CC131092981397
:10DCC0001092971310929A131092991310929C131A
:10DCD00081E080939B1382E280939D131092A213A4
:10DCE0001092A113E6EBF3E124EC33E18FEF819383
:10DCF0002E173F07E1F7C1E0C093B31327E931EBDB
:10DD00003093A9132093A813C093AA131092AB13B6
:10DD10001092AC1390E49093AD131092AE1326E9D9
:10DD200031EB3093C5132093C41325E531E03093D4
:10DD30009613209395139EE19093BA1391E19093DB
:10DD4000BB139CE19093B8138093B7138093B613E1
:10DD50000E943FD2C0932E0681E080932D068DE372
:10DD600092E29093A9128093A8121092AB12109293
:10DD7000AA1253985B9A52985A9A3898409A0E94DD
:10DD80009B6510929202CF910895FC0180E030973C
:10DD900049F09491992331F0907C903809F08F5F8D
:10DDA0003196F7CF0895B0E0A0E0E9EDFEE60C94DF
:10DDB000FDF0EC015B018A01FB01099587FD10C0B4
:10DDC000C82ED12CF12CE12C2196F801C082D182F1
:10DDD000E282F382CE01CDB7DEB7EAE00C9419F10E
:10DDE000982F907E903CA9F48F7190E0B0E0A0E075
:10DDF0006C017D0156E0CC0CDD1CEE1CFF1C5A951D
:10DE0000D1F7CE010196F50109958F73C82A2296A4
:10DE1000DCCF982F907F903E11F58F7090E0B0E0AE
:10DE2000A0E06C017D0136E0CC0CDD1CEE1CFF1C7B
:10DE30003A95D1F7CE010196F50109958F73C82A5D
:10DE400046E0CC0CDD1CEE1CFF1C4A95D1F7CE0140
:10DE50000296F50109958F73C82A2396B6CF982F9D
:10DE6000987F903F79F5877090E0B0E0A0E06C017A
:10DE70007D0186E0CC0CDD1CEE1CFF1C8A95D1F7E1
:10DE8000CE010196F50109958F73C82A96E0CC0C56
:10DE9000DD1CEE1CFF1C9A95D1F7CE010296F50110
:10DEA00009958F73C82A26E0CC0CDD1CEE1CFF1CE4
:10DEB0002A95D1F7CE010396F50109958F73C82AEB
:10DEC000249683CF982F907C903841F4807C8038C2
:10DED00069F42196CE01F5010995F8CF8E7F8D3F2B
:10DEE00028F02196CE01F5010995F8CFC12CD12C4F
:10DEF00076016BCF9CE0899F802D112491E0980FD3
:10DF000090932C062CE0280F20937B0730E02E5FA7
:10DF10003F4F4091C7134217130619F014F080E0E9
:10DF200008952091C9139217D0F7662341F08E5FB0
:10DF30000E9424D380917B078E5F0E9424D380911E
:10DF40007B079091C713891750F32091C9139091C3
:10DF50002C06291720F31092CA138093CB1381E06B
:10DF6000089520912B06022E000C330B8217130606
:10DF700041F080932B0668EA73E283E993E10C9405
:10DF8000EDD30895ACE0B0E0E8ECFFE60C94FFF0D0
:10DF90006F3F71058105910509F070F48FE893E1F9
:10DFA0007EDDE0919713F09198133196849190E083
:10DFB0002C96E8E00C941BF1F090CA13E090CB1380
:10DFC00020912D0621110FC04FE052E26E2D8F2DB2
:10DFD0000E949ED490E080E0F80EF092CA13E09286
:10DFE000CB139927E5CFC0909713D090981323E9CE
:10DFF00033E13A8329832F2D30E03C832B832E2D70
:10E0000030E03E832D8318861F822FEF3FEF3A8743
:10E0100029871C861B860CEF1CE69E012F5F3F4F55
:10E02000AB01BC01C6010E94A5B2B60183E993E130
:10E030000E94EDD38F819885CFCF4F925F926F92E0
:10E040007F928F929F92BF92CF92DF92EF92FF9238
:10E050000F931F93CF93DF93CDB7DEB728970FB6FB
:10E06000F894DEBF0FBECDBF7C016A014901FB0100
:10E0700090818CE0989F800D1124982FF7012081CA
:10E08000822F880F820F880F8093CA139093CB132F
:10E090004115510559F1FA82E9827C836B830111A4
:10E0A0001EC0AE014B5F5F4FB401C6017CDE6C0148
:10E0B0006D817E818F81988561157105810591053E
:10E0C000A9F060DFF70180818F5F8083853148F39D
:10E0D000CE01019644D8E5CFB12C860129C08A0132
:10E0E000B12C26C0452846284728B1F728960FB6F8
:10E0F000F894DEBF0FBECDBFDF91CF911F910F917E
:10E10000FF90EF90DF90CF90BF909F908F907F9087
:10E110006F905F904F900895B39407C0B1102DC0D9
:10E1200001151105C9F20F5F1F4F01151105A9F265
:10E13000AE014B5F5F4FB401C60135DE6C014D800F
:10E140005E806F8078844114510461047104A9F0E9
:10E15000F0E24F1651046104710401F3D301C201CE
:10E160008D97A109B1090297A105B10530F04BE2E5
:10E17000441651046104710479F6F7018081482F37
:10E180004B0D5527551F4631510534F0853020F091
:10E19000CE0101960E94AF6881E0411451046104F0
:10E1A000710409F480E0B80EF70180818B0D808343
:10E1B000BB2009F497CFBA94AE014B5F5F4FB40117
:10E1C000C801F1DD8C016D817E818F819885DADE59
:10E1D000EFCFCF93DF93FC0125AD211104C021E0E7
:10E1E00025AF0E943FD2C0919513D0919613E09134
:10E1F000C413F091C51382E00995E091C413F09126
:10E20000C51381E0099530E020E044E1BE0183E9D7
:10E2100093E10E943AD226EC33E147E1BE0183E963
:10E2200093E10E943AD2E091C413F091C51380E0CB
:10E230000995DF91CF9108954F925F926F927F92EF
:10E240008F929F92AF92BF92CF92DF92EF92FF9206
:10E250001F93CF93DF9300D000D0CDB7DEB70E94DD
:10E2600002D16B017C0180915D018F3FC1F10E9461
:10E2700002D180905F0690906006A0906106B090F9
:10E280006206681979098A099B0997FD28C080915F
:10E290006713909168138F5F8F70891701F1E09178
:10E2A0005D01E53008F054C024E0E29FF001112444
:10E2B000EE5BFD4F80819181A281B38189839A8336
:10E2C000AB83BC8320E030E0A901BE016F5F7F4FCC
:10E2D00085E791E00E94D9C68FEF80935D010E948F
:10E2E0009B658091930282FF3CC080916E068111F4
:10E2F0003AC091E090936E068091980289278093AE
:10E3000057071092980283E080936A01109293025B
:10E310000E9402D16C507E4F8F4F9F4F60939402AA
:10E3200070939502809396029093970268E873E148
:10E3300082E090E00E941B4616E01150A1F00E947E
:10E34000BF4562E070E080E090E00E9479D0F5CFB8
:10E3500080916B0190916C01A0916D01B0916E0163
:10E36000ADCF10926E0680916A0690916B06A091D7
:10E370006C06B0916D06A7019601281B390B4A0B5C
:10E380005B0BDA01C901B7FF05C0809199028823B0
:10E3900009F4B9C1D701C6018C599F4FAF4FBF4F88
:10E3A00080936A0690936B06A0936C06B0936D06FB
:10E3B00060919202062E000C770B77FF03C07195D7
:10E3C000619571099091920280916906981365C0D8
:10E3D000633008F062C010929202809192028093A2
:10E3E0006906643008F069C0809157078111E7C061
:10E3F00080918D1390918E138B5C9B4741F480919B
:10E400005E01882309F4EDC0815080935E010E9473
:10E41000822F8090AB079090AC07A090AD07B09092
:10E42000AE0781110E948F2FD501C4013AE0B69545
:10E43000A795979587953A95D1F7009741E0A4075E
:10E44000B10520F08FEF9FEFA0E0B0E096958795A3
:10E4500020916A012111D7C030919902311180C1F8
:10E4600080918D1390918E138B5C9B4709F45FC153
:10E4700080919A0281115BC1809165069091660638
:10E48000A0916706B0916806C81AD90AEA0AFB0A81
:10E49000F7FC5BC10E94974758C1633009F09DCFDC
:10E4A0008091920287FD07C081E0880F880F8093DA
:10E4B000920264E092CF8FEFF8CF80917A0721E04B
:10E4C00030E040E050E0882309F456C080907607A1
:10E4D00090907707A0907807B09079078114910405
:10E4E000A104B104E9F170E090E080E00E9413EA39
:10E4F00020E030E040E85EE30E9474EA2B013C013A
:10E50000C701B601681979098A099B090E9413EAB3
:10E510009B01AC01C301B2010E94A4F120E030E0F4
:10E520004AE754E40E9474EA4B015C0120E030E0C9
:10E5300040EA52E40E9490F224E630E040E050E0ED
:10E5400087FF12C020E030E040EF51E4C501B40184
:10E550000E9490F22AE030E040E050E087FF04C0E3
:10E5600021E030E040E050E0C0927607D09277079B
:10E57000E0927807F0927907A09192020A2E000C9F
:10E58000BB0B0E9485F024E030E040E050E00E94A8
:10E590005FF08091720790917307A0917407B0911A
:10E5A0007507820F931FA41FB51F80937207909366
:10E5B0007307A0937407B093750710929202D70166
:10E5C000C6018856954CAF4FBF4F80936506909318
:10E5D0006606A0936706B093680681E080936A019F
:10E5E00007CF8CE080935E01809163069091640672
:10E5F000009729F00197909364068093630681E069
:10E6000080936A0104CF009741F0409163065091D6
:10E6100064064817590708F023CF809199028111A9
:10E6200011C0223038F0243008F43FC0243011F4F7
:10E6300010926A018FE893E1CCDD81E0809371074D
:10E640008093990283E08DDC81E08093B313E091A5
:10E650008D13F0918E130995109271078091990294
:10E66000811127C01092570780918D1390918E13BE
:10E670008B5C9B4709F0FCCE0E9402D1DC01CB01F0
:10E680008C199D09AE09BF098090630690906406BD
:10E69000B12CA12C88169906AA06BB0608F0E0CE7C
:10E6A0009093640680936306DBCE81E080936A01D9
:10E6B000C1CF83E993E10E94BDD391E0811101C0F4
:10E6C00090E090939902882369F280918D13909144
:10E6D0008E138B5C9B47B9F40E9402D1DC01CB0105
:10E6E0008C199D09AE09BF09C0906306D0906406DD
:10E6F000F12CE12CC816D906EA06FB0620F490930B
:10E700006406809363060F900F900F900F90DF9137
:10E71000CF911F91FF90EF90DF90CF90BF90AF907F
:10E720009F908F907F906F905F904F90089548E9F1
:10E73000C40E4AE3D41EE11CF11CC0926506D092BF
:10E740006606E0926706F092680680919902811150
:10E75000DACF80916A018130B1F610926A01D3CF8D
:10E76000009709F46FCF51CFACE0B0E0EAEBF3E7EC
:10E770000C94FFF0F090CA13E090CB1320912D067B
:10E78000211112C04FEE51E26E2D8F2D0E949ED4AA
:10E7900090E080E0F80EF092CA13E092CB13992734
:10E7A0002C96E8E00C941BF1C0909713D09098132E
:10E7B00023E933E13A8329832F2D30E03C832B83F7
:10E7C0002E2D30E03E832D8318861F827A8769873D
:10E7D0001C861B860CEF1CE69E012F5F3F4F45EC0D
:10E7E00058E6BC01C6010E943AB3B60183E993E141
:10E7F0000E94EDD38F819885CDCFA4E0B0E0E3E017
:10E80000F4E70C94FBF07C01062F5A01122F862F9F
:10E81000660F990B9C012A5C3D4F690186E0882EAA
:10E82000912C11160CF03DC0AE014F5F5F4F65ECAF
:10E8300078E6C701B8DA7C0169817A818B819C8195
:10E84000611571058105910561F16D3371058105D2
:10E85000910509F450C06E3771058105910509F4E1
:10E860004AC06A3271058105910501F507FF11C0A3
:10E8700083E392E20E3F11F08FE292E236E0130260
:10E88000B001112471DF66E070E00E94C7F0161B32
:10E8900060C065E470E080E090E074DB115069F5E1
:10E8A00010E0812F2496ECE00C9417F1643271058E
:10E8B0008105910571F4A114B104D1F0E6E01E02C6
:10E8C000B0011124C50150DFB4010E94C7F0161B2E
:10E8D000A8CF603471058105910551F41150F601FE
:10E8E0006081062E000C770B880B990B4BDB99CFC0
:10E8F00049DB115096CF07FDBBCF61E089819A813A
:10E90000AB81BC81CD97A105B10509F460E0600F32
:10E910006A30A4F01150862F6AE00E94A6F0092FF9
:10E92000682F880F770B605D7F4F072E000C880BD8
:10E93000990B28DB112309F4B3CF602F062E000CAE
:10E94000770B605D7F4F072E000C880B990B1ADB4D
:10E950001150112309F4A4CF86E01802B00111244C
:10E96000C70102DF66E070E00E94C7F0161B99CF76
:10E97000EFE8F3E183AF64AF6FEF7FEFCA01F4CE4E
:10E98000ACE0B0E0E6ECF4E70C94FFF0F090CA13D2
:10E99000E090CB1320912D06211112C04FEC51E2D3
:10E9A0006E2D8F2D0E949ED490E080E0F80EF092A4
:10E9B000CA13E092CB1399272C96E8E00C941BF134
:10E9C000C0909713D090981323E933E13A832983B9
:10E9D0002F2D30E03C832B832E2D30E03E832D8382
:10E9E00018861F827A8769871C861B860CEF1CE6B7
:10E9F0009E012F5F3F4F48EC58E6BC01C6010E94C4
:10EA00003AB3B60183E993E10E94EDD38F819885F3
:10EA1000CDCF6FEF7FEFB4CFB0E0A0E0E2E1F5E75C
:10EA20000C94FDF05C016B01B0D9E82EC6010E9488
:10EA3000CB68F12C03E110E0081B1109C5E20E15AB
:10EA40001F050CF4CFE18C2F90E09C012E5F3F4F0F
:10EA50004091C7134217130609F08CF509972091CE
:10EA6000C913281719065CF140917D0750917E0764
:10EA700060917C071092CA13C093CB1325E1C501A6
:10EA8000BCDED1E0C114D104A9F06AE370E080E0FB
:10EA900090E078DA0E151F05A4F4C45F8091C713C7
:10EAA000C81740F02091C9134C2F4950550B24171B
:10EAB00015064CF4CDB7DEB7EAE00C9419F1D0E0BE
:10EAC000E1CFDD23B9F3802F880F080F000F0093EB
:10EAD000CA13C093CB1360E270E080E090E052DA9A
:10EAE000C60197DFE7CFACE0B0E0E9E7F5E70C94CB
:10EAF000FBF0982F862F6A017901B02E692FFAD981
:10EB0000882309F487C010912D06C701002371F1F5
:10EB10003CD9A82E8090971390909813111142C061
:10EB20002FEF3FEF122F23E12A1940917D075091DB
:10EB30007E0760917C07C60160DEAA2009F46AC0E6
:10EB4000B6E08B9F600111246AE370E080E090E002
:10EB500019DA57E0C516D10408F442C060E270E04B
:10EB600080E090E00FDAC81AD90AF3CF0E94CB6890
:10EB7000A82E8090971390909813112389F2FE018C
:10EB800033968AE0DF011D928A95E9F783E993E1E4
:10EB90009A83898305ED1CE69E012F5F3F4F48EC69
:10EBA00058E612C0FE0133968AE0DF011D928A9575
:10EBB000E9F783E993E19A83898305ED1CE69E01D9
:10EBC0002F5F3F4F45EC58E6B701C4010E943AB3AE
:10EBD000B40183E993E10E94EDD32F813885A2CF60
:10EBE00040917B07212F30E0A6E0AA9EC0011124AE
:10EBF0002E5F3F4F281739070CF49C0180E8821BD9
:10EC00008093CA134093CB13BB2041F06FEF7FEF8B
:10EC1000C701AADD2C96ECE00C9417F1C701F9DED0
:10EC2000F9CFEFE8F3E183AF64AFCA01F2CE0C9401
:10EC3000C0B34F925F926F927F928F929F92BF92DA
:10EC4000CF92DF92EF92FF920F931F93CF93DF93B8
:10EC500010922306109222062FE32093260610928C
:10EC600025061092240610921E0610921F0610927E
:10EC70002006109221069C01F90190812F5F3F4FE1
:10EC80009032D1F39E34C9F4818190ED980F9A307F
:10EC900020F08D3211F08B3281F432969F012F5F7C
:10ECA0003F4F808180538A3008F46DC09F012F5FF1
:10ECB0003F4F8081803209F468C0F0939207E0935F
:10ECC00091078F010F5F1F4FC0816AE270E0C8019A
:10ECD0000E9446F3009731F0FC0131978081803229
:10ECE000E1F31182CD3421F0C43511F0C734D9F5E8
:10ECF000F80180810F5F1F4F8032D1F380538A303B
:10ED000090F5C093260690E080E06AE0AF014F5F87
:10ED10005F4F689F9001699F300D1124C901C09712
:10ED20002081820F911D27FD9A95FA0120812053A1
:10ED30002A3060F39093250680932406DF013196F4
:10ED40002C912032D9F3CD3461F58E31910539F013
:10ED5000F0F48731910519F08C31910511F5B093DC
:10ED60002306A0932206DF91CF911F910F91FF9070
:10ED7000EF90DF90CF90BF909F908F907F906F909B
:10ED80005F904F900895F90189CFF9018FCF8537B2
:10ED9000910538F08737910510F3803A13E0910719
:10EDA000F1F2809091079090920740E050E0BA0114
:10EDB00030E020E0C12CD12C7601C394FD013196C6
:10EDC000DC91DD2309F484C0D132F1F4CD34E1F4D7
:10EDD00080329105C9F440931E0650931F0660933C
:10EDE000200670932106F0932306E093220663E247
:10EDF00070E0CF010E9446F3009709F4B4CFFC0104
:10EE00001082B1CFDF01DACFD154DA3108F05BC024
:10EE1000DF011D91103291F0A0EDA10FAA30E8F0B2
:10EE20001E3271F4A181A053AA30B8F0211531052A
:10EE300019F49F0121503109B12C13C0FD01E8CF15
:10EE40001D3211F01B3291F7A181B0EDBA0FBA302B
:10EE500020F0AE3259F7A281E6CFBE2EB818309717
:10EE600059F3AD2FB0E02601370104C0440C551C06
:10EE7000661C771CDA95D2F744295529662977292B
:10EE8000AC5FB94FBC92A081A154AA3108F4BACFAB
:10EE9000DF01D191DD2309F491CF00EDB02EBD0E3D
:10EEA00019E01B15A8F713EDB12EBD0E11E01B15CF
:10EEB00078F7DB3269F3FD013196DC91D03209F04D
:10EEC0007DCFDF01F8CF21153105E9F69D01DBCFBC
:10EED000309323062093220640931E0650931F066C
:10EEE00060932006709321063ECFFC0165917591D9
:10EEF0008591949108958F929F92AF92BF92CF92F5
:10EF0000DF92EF92FF92CF93DF93EC018090B402F7
:10EF10009090B502A090B602B090B70220E030E029
:10EF2000A901C501B4010E940FEA882309F452C067
:10EF3000C880D980EA80FB80A7019601C501B40191
:10EF40000E940FEA18160CF04AC02091EE0530918D
:10EF5000EF054091F0055091F105C701B6010E94FF
:10EF60000FEA882321F1C092EE05D092EF05E092DE
:10EF7000F005F092F1052091EA053091EB05409102
:10EF8000EC055091ED05C701B6010E9474EA9B01A2
:10EF9000AC0160E070E080E89FE30E942CF1609398
:10EFA0004A0170934B0180934C0190934D01609105
:10EFB0004A0170914B0180914C0190914D01DF917C
:10EFC000CF91FF90EF90DF90CF90BF90AF909F9048
:10EFD0008F90089560E070E080E89FE3F0CF60E0FC
:10EFE00070E0CB01ECCFB0E0A0E0E9EFF7E70C94E4
:10EFF000F7F0EC0120917C0330917D0340917E037A
:10F0000050917F03688179818A819B810E942CF1D4
:10F010004B015C0120918003309181034091820378
:10F02000509183036C817D818E819F810E942CF1A0
:10F030006B017C01A5019401609142017091430133
:10F0400080914401909145010E940FEA882309F4C0
:10F0500054C08092420190924301A0924401B09228
:10F0600045012091E2053091E3054091E40550917E
:10F07000E505C501B4010E9474EA2B013C010E9420
:10F080003DF24B015C0120E030E040EA50E40E9498
:10F090000FEA181634F4812C912CC0EAAC2EC0E48F
:10F0A000BC2E20E030E0A901C501B4010E9490F21D
:10F0B00087FF03C0812C912C5401A5019401C30149
:10F0C000B2010E942CF16093DA057093DB05809306
:10F0D000DC059093DD05C501B4010E940CF260933C
:10F0E000D805062E000C770B6F5F7F4F66307105D9
:10F0F00014F066E070E06093D605D0914001109165
:10F10000D805A70196016091460170914701809151
:10F110004801909149010E940FEA811123C0D11347
:10F1200075C02091BE053091BF054091C00550913A
:10F13000C1056091DA057091DB058091DC05909145
:10F14000DD050E9474EA2091C2053091C30540910B
:10F15000C4055091C5050E942DF1CDB7DEB7E0E1A1
:10F160000C9413F1C0924601D0924701E0924801FD
:10F17000F09249012091E6053091E7054091E805BC
:10F180005091E905C701B6010E9474EA4B015C0188
:10F190000E943DF26B017C0120E030E040EA50E447
:10F1A0000E940FEA181634F4C12CD12CB0EAEB2ED1
:10F1B000B0E4FB2E20E030E0A901C701B6010E94B7
:10F1C00090F287FF03C0C12CD12C7601A7019601D4
:10F1D000C501B4010E942CF16093DE057093DF0538
:10F1E0008093E0059093E105C701B6010E940CF2FF
:10F1F0006093D905062E000C770B6F5F7F4F66304A
:10F20000710514F066E070E06093D705C091D905F0
:10F21000D11305C0809141018C1709F470C0809111
:10F22000D8059091D90590934101809340010C2E0F
:10F23000000CDD0B27E01203C0011124FC01EC0FD0
:10F24000FD1FEE0FFF1FEE0FFF1FE854FD4F208143
:10F250003181428153812093D2053093D30540936D
:10F26000D4055093D5050091D705002E000C110B45
:10F27000FC01E00FF11FEE0FFF1FEE0FFF1FE85420
:10F28000FD4F60817181828193810E942CF1609396
:10F29000CE057093CF058093D0059093D105209132
:10F2A000D60537E02303F0011124CE0FDF1FCC0F6A
:10F2B000DD1FCC0FDD1FC854DD4F288139814A8105
:10F2C0005B812093CA053093CB054093CC055093C6
:10F2D000CD05E00FF11FEE0FFF1FEE0FFF1FE854EB
:10F2E000FD4F60817181828193810E942CF1609336
:10F2F000C6057093C7058093C8059093C905809093
:10F30000DE059090DF05A090E005B090E10520912A
:10F31000CE053091CF054091D0055091D105C50162
:10F32000B4010E9474EA2091D2053091D305409136
:10F33000D4055091D5050E942DF16B017C01C0923E
:10F34000C205D092C305E092C405F092C505209194
:10F35000C6053091C7054091C8055091C905C50142
:10F36000B4010E9474EA2091CA053091CB05409106
:10F37000CC055091CD050E942DF1A70196010E9468
:10F380002CF16093BE057093BF058093C0059093E8
:10F39000C105C7CEACE0B0E0E0EDF9E70C9404F1B4
:10F3A000182F882379F020E030E0A90160918403D0
:10F3B0007091850380918603909187030E940FEAE4
:10F3C0008823F1F08091B3028117D1F00E94AE2C16
:10F3D0008CE0EAE2F2E0DE01119601900D928A954E
:10F3E000E1F7CE010196FFDD8091B302882361F041
:10F3F00085E791E00E94042D1092B3020E94A93F7C
:10F400002C96E3E00C9420F181E08093B30285E731
:10F4100091E00E94D02CF2CFCF92DF92EF92FF9238
:10F4200080E0B8DF10928003109281031092820373
:10F430001092830310927C0310927D0310927E033E
:10F4400010927F03109288031092890310928A030E
:10F4500010928B03109284031092850310928603FE
:10F460001092870348EB52E027E0C12CD12C60ECCE
:10F47000E62E6FE7F62E90E080E0FC01EE0FFF1F16
:10F48000EE0FFF1FE40FF51FC082D182E282F382EC
:10F4900001968730910589F72150445E5F4F211115
:10F4A000EACFFF90EF90DF90CF9008954F925F9258
:10F4B0006F927F928F929F92AF92BF92CF92DF9284
:10F4C000EF92FF921F93CF93DF93EC01162F2091C1
:10F4D000B4023091B5024091B6025091B7026881F2
:10F4E00079818A819B810E940FEA882309F497C061
:10F4F000B090B30280E04EDFC880D980EA80FB8004
:10F5000020E030E0A901C701B6010E9490F287FF18
:10F5100003C0C12CD12C7601C092B402D092B502A6
:10F52000E092B602F092B7022DEB37E346E855EBD6
:10F53000C701B6010E940FEA87FD0BC02DEB37E330
:10F5400046E855E3C701B6010E9490F218160CF088
:10F5500076C0A701960160E070E080E89FE30E941A
:10F56000A4F16093EA057093EB058093EC0590930A
:10F57000ED0580EF9FEFA9E7B4EC8093EE05909343
:10F58000EF05A093F005B093F105BB2009F447C047
:10F5900040907501509076016090770170907801ED
:10F5A0008090790190907A01A0907B01B0907C01CD
:10F5B000C0907D01D0907E01E0907F01F0908001AD
:10F5C00081E0E8DE112359F1A301920160917501F8
:10F5D0007091760180917701909178010E940FEAF5
:10F5E00081111BC0A50194016091790170917A018C
:10F5F00080917B0190917C010E940FEA81110DC0E6
:10F6000020917D0130917E0140917F0150918001D8
:10F61000C701B6010E940FEA81110E94F73FDF91F6
:10F62000CF911F91FF90EF90DF90CF90BF90AF9060
:10F630009F908F907F906F905F904F90089560E0C3
:10F6400070E0CB018ECF8F929F92AF92BF92CF92FC
:10F65000DF92EF92FF92C0908403D0908503E090F8
:10F660008603F090870320E030E0A901C701B601CE
:10F670000E940FEA8823E1F1A701960160E070E0A3
:10F6800080E89FE30E94A4F16B017C0180908803D5
:10F6900090908903A0908A03B0908B0320E030E023
:10F6A000A901C501B4010E940FEA882329F1A5012F
:10F6B000940160E070E080E89FE30E94A4F1C092B2
:10F6C000E205D092E305E092E405F092E50560934F
:10F6D000E6057093E7058093E8059093E905FF90B0
:10F6E000EF90DF90CF90BF90AF909F908F90089554
:10F6F000C12CD12C7601CACF60E070E0CB01DFCF06
:10F70000CF92DF92EF92FF926B017C0183E3C816E8
:10F71000D104E104F10470F082E3C81AD108E108D1
:10F72000F10862E370E080E090E00E9479D00E94EE
:10F73000F029ECCFC701B6010E9479D00E94F029D0
:10F74000FF90EF90DF90CF900895BC0190E080E0B3
:10F750000C9463B380918F07813069F09091E51428
:10F7600092FB882780F992FF07C097FB882780F9D2
:10F7700091E08927089581E008959091E51494FB24
:10F78000882780F994FF06C081E09091CE129111F4
:10F7900001C080E00895A4E0B0E0E1EDFBE70C9447
:10F7A000F7F010927A078091570710925707882335
:10F7B00061F020E040E070E060E08CE393E60E94BE
:10F7C0005B462496E0E10C9413F1209110013091F6
:10F7D00011014091720750917307CA01820F931F64
:10F7E0002436310509F01DC44730510544F0069711
:10F7F0008A3091050CF024C48AE090E02BC4069670
:10F800004A3F5F4FACF380917107882309F4C8C168
:10F810006091BA127091BB12072E000C880B990BE5
:10F820000E9415EAB1E0B9832091B6123091B71267
:10F830004091B8125091B9120E9490F218160CF033
:10F84000198260913C0770913D07072E000C880BD0
:10F85000990B0E9415EA20913807309139074091A1
:10F860003A0750913B070E9490F218161CF4E98168
:10F87000E260E983C980C0925E06C0907501D090B5
:10F880007601E0907701F090780180917901909174
:10F890007A01A0917B01B0917C0189839A83AB832B
:10F8A000BC8380907D0190907E01A0907F01B090FC
:10F8B000800120E030E04AE754E4C501B4010E9431
:10F8C00074EA2B013C0120E030E0A901C501B4013C
:10F8D0000E940FEA20E030E040EA50EC87FD04C0CF
:10F8E00020E030E040EA50E4C301B2010E942DF173
:10F8F0002DEC3CEC4CEC5DE30E9474EA0E940CF2AF
:10F900004B015C0180E2B7FE09C0B094A0949094D2
:10F910008094811C911CA11CB11C8DE280939B02E0
:10F9200060E290E1891697E29906A104B1048CF097
:10F93000C501B40120E137E240E050E00E945FF0F1
:10F94000CA01B9012AE030E040E050E00E945FF0D7
:10F95000605D60939C0260E2A8EE8A16A3E09A06BE
:10F96000A104B1048CF0C501B40128EE33E040E0FD
:10F9700050E00E945FF0CA01B9012AE030E040E0A7
:10F9800050E00E945FF0605D60939D02C501B4018C
:10F9900024E630E040E050E00E945FF06AE0462E4E
:10F9A000512C612C712CCA01B901A30192010E9452
:10F9B0005FF0605D60939E02C501B401A3019201F6
:10F9C0000E945FF04B01CA01B901A30192010E949C
:10F9D0005FF0882009F44EC32EE220939F02605D01
:10F9E0006093A002B0E38B0E8092A1026BE972E0FB
:10F9F00086E596E00E9451F320E030E0A901C701BE
:10FA0000B6010E940FEA20E030E040E05FEB87FDA6
:10FA100004C020E030E040E05FE3C701B6010E948F
:10FA20002DF10E940CF2CB010E949F44BC0181E5A4
:10FA300096E00E9451F320E030E0A90169817A81CB
:10FA40008B819C810E940FEA20E030E040E05FEB78
:10FA500087FD04C020E030E040E05FE369817A8107
:10FA60008B819C810E942DF10E940CF2CB010E949F
:10FA70009F44BC018CE496E00E9451F38091E51410
:10FA800083FD0AC37ADE882309F409C38091DD145B
:10FA90009091DE14A091DF14B091E0140097A105BD
:10FAA000B10509F4FCC2BC01CD016D597F4F8F4FE8
:10FAB0009F4F24E630E040E050E00E943DF060912E
:10FAC000E1147091E2148091E3149091E4140E9487
:10FAD0003DF029830E94DE434B015C01162F80918B
:10FAE0005C01C9808C15C1F0C0925C0128E4C29E03
:10FAF000B001112490E080E00E9413EA2AE037ED83
:10FB000043E25CE30E9474EA0E9411F260934B06A8
:10FB1000C110C7C21092460680915B01181709F404
:10FB20003FC080925B01C501B40120E13EE040E0AE
:10FB300050E00E943DF0690189019CE3492E512C5F
:10FB4000612C712CC501B401A30192010E943DF00A
:10FB50004B015C01CA01B901A30192010E943DF071
:10FB6000C114D10409F0C4C29F928F927F936F9306
:10FB700083E592E29F938F9386E396E09F938F9322
:10FB80000E94A8E90FB6F894DEBF0FBECDBF85E096
:10FB9000982F990F990F891B880F805880933506ED
:10FBA0000E9402D100913006109131062091320658
:10FBB000309133066B017C01C01AD10AE20AF30AC4
:10FBC0009701860137FD11C020912F0620952093C3
:10FBD0002F066A547C4F8F4F9F4F6093300670936F
:10FBE00031068093320690933306D0902F06D98247
:10FBF00081E00E94B16F8091C713873180F48091BA
:10FC0000C913843060F086E3E82E83E2F82E03E126
:10FC100026E044E064E083E993E10E94C3D480914C
:10FC20005E06982F927048E00CE081FD02C042E130
:10FC300002E08091C713843180F48091C913841746
:10FC400060F0992309F473C282E193E27C0123E01E
:10FC500060E583E993E10E94C3D48091C7138431A6
:10FC6000C0F48091C9138230A0F0C980CC2009F47F
:10FC700061C28091AF07882309F45CC286ED92E2ED
:10FC80007C0102E123E042E068E683E993E10E941F
:10FC9000C3D48091C7138C3108F09DC08090B612F8
:10FCA0009090B712A090B812B090B912C090BA124A
:10FCB000D090BB12843198F48091C913883078F0C9
:10FCC00080915E0680FF39C288E892E27C010CE0F8
:10FCD00022E048E069E383E993E10E94C3D4809184
:10FCE000C713883040F4D7FE2BC24CE652E267E0DF
:10FCF00087E30E94B8748091C7138C31B0F480916F
:10FD0000C913843190F020E030E040E05FE3C501AA
:10FD1000B4010E942DF10E940CF277FF34C24CE630
:10FD200052E26CE187E30E94B874C0903807D0902B
:10FD30003907E0903A07F0903B078091C71388306D
:10FD400060F480913C0790913D0797FF3FC24CE6DD
:10FD500052E267E081E50E94B8748091C7138C314C
:10FD6000B0F48091C913843190F020E030E040E09D
:10FD70005FE3C701B6010E942DF10E940CF277FFEC
:10FD800047C24CE652E26CE181E50E94B874809172
:10FD9000C7138C3100F58091C9138431E0F0809154
:10FDA000AF078823C1F024E6829FC0011124815847
:10FDB0009F4F6FEF70E00E94C7F0CB010E941E457D
:10FDC000AC016CE187E60E94117665E270E080E0AC
:10FDD00090E00E94C26FD1DC882379F18091C71333
:10FDE000843358F58091C9138A3238F107E028E04E
:10FDF0004AE26AE283E993E10E946AD305E022E0E5
:10FE00004CE262E383E993E10E946AD324E04AE092
:10FE100061E38AE20E943AD3609195137091961340
:10FE200082E38093AF138BE28093B0132FEA33E128
:10FE300042E383E993E10E943AD28091C71385336C
:10FE400050F48091C913813330F024E04AE461E337
:10FE500086E30E943AD38091C713843368F480917B
:10FE6000C913823348F002E020914B0642E367E376
:10FE700083E993E10E946AD38091C7138033D8F459
:10FE80008091C9138832B8F080914606882361F0CA
:10FE900046E456E060E387E30E94117665E270E095
:10FEA00080E090E00E94C26F46E356E060E38091FC
:10FEB00035060E9411768091C713883208F060C021
:10FEC0008091C9138D3108F45BC02BE040E86DE1EF
:10FED00080E00E943AD38091C713873208F050C067
:10FEE0008091C9138F3108F44BC083E08093CA130B
:10FEF00016E21093CB1368E570E080E090E00E947A
:10FF0000C26F8BE08093CA131093CB13C980CC20AF
:10FF100009F4A1C181E596E00E94097588E2809309
:10FF2000CA1316E21093CB1369E570E080E090E00D
:10FF30000E94C26F80E38093CA131093CB13C980D1
:10FF4000CC2009F4ABC18CE496E00E9409758DE4E5
:10FF50008093CA1316E21093CB136AE570E080E039
:10FF600090E00E94C26F85E58093CA131093CB1373
:10FF7000C980CC2009F4B5C186E596E00E940975D8
:10FF80008091C713833338F58091C9138B3218F1F0
:10FF900083E00E94B16F83E08093CA1383E3809370
:10FFA000CB1366E070E080E090E00E94C26F81E0D9
:10FFB0000E94B16F80911001909111010E941E4525
:10FFC000AC0163E38CE00E94117665E270E080E0B2
:10FFD00090E00E94C26F8091C713813408F0F1CB8A
:10FFE0008091C913863308F4ECCB1092CA138EE3C8
:10FFF0008093CB1387E490E10E94CB68182F863161
:020000021000EC
:1000000008F092C187E490E10E940975153109F466
:10001000D8CB60E270E080E090E00E94C26F1F5F8A
:10002000F5CF243631054CF48536910504F58A3038
:10003000910534F48AE090E009C084369105BCF063
:10004000883EA3E09A0714F087EE93E0281739075B
:1000500009F4D9CB9093110180931001109272078B
:10006000109273071092740710927507CCCB84E638
:1000700090E0F0CF662351F02EE220939F02605D66
:100080006093A00280E28093A102B0CC80E28093D2
:10009000A00280939F02F6CFE4E6E9831BCD19828C
:1000A00019CD498180E2443628F0842F64E60E940D
:1000B0009AF0805D80939F02698190E26A3040F0FF
:1000C0002AE0862F622F0E949AF00E949AF0905D9B
:1000D0009093A00289816AE00E949AF0905D9093CB
:1000E000A1026FE972E086E496E00E9451F314CD1C
:1000F0000436110538F47F936F93DF92CF9287E433
:1001000092E238CD7F936F93DF92CF928DE392E2AC
:100110009F938F9386E396E09F938F930E94A8E925
:100120000FB6F894DEBF0FBECDBF86E031CD8CE0B8
:1001300093E28CCD80EA92E2A3CD80E792E2C6CD35
:10014000C6010E941E45FC01808193E0803229F4A3
:10015000818192E0803209F491E043E050E0491B54
:1001600051094E0F5F1F892F880F880F981B892F09
:1001700067E0805C0E94117669E070E080E090E0CA
:100180000E94C26FB8CDCB010E941E45FC01808148
:1001900093E0803229F4818192E0803209F491E089
:1001A00043E050E0491B51094E0F5F1F892F880F14
:1001B000880F981B892F6CE1805C0E94117669E0A2
:1001C00070E080E090E00E94C26FAFCD0E941E45BB
:1001D000FC01808193E0803229F4818192E08032B9
:1001E00009F491E043E050E0491B51094E0F5F1FB5
:1001F000892F880F880F981B892F67E0865A0E94E5
:10020000117669E070E080E090E00E94C26FA5CDB9
:10021000CB010E941E45FC01808193E0803229F4CD
:10022000818192E0803209F491E043E050E0491B83
:1002300051094E0F5F1F892F880F880F981B892F38
:100240006CE1865A0E94117669E070E080E090E0EF
:100250000E94C26F9CCD87E00E94563B80FF13C076
:1002600001E516E0D8016D918D01662309F456CEA3
:100270006F320CF06FE3062E000C770B880B990B96
:100280000E94C26FEFCF80917F0780FD43CE6FEF5A
:100290007FEF87E692E20E94B47340CE87E00E942F
:1002A000563B81FF13C00CE416E0D8016D918D011F
:1002B000662309F44CCE6F320CF06FE3062E000C6F
:1002C000770B880B990B0E94C26FEFCF80917F074D
:1002D00081FD39CE6FEF7FEF87E692E20E94B47323
:1002E00036CE87E00E94563B82FF13C006E516E03B
:1002F000D8016D918D01662309F442CE6F320CF066
:100300006FE3062E000C770B880B990B0E94C26FCF
:10031000EFCF80917F0782FD2FCE6FEF7FEF8FE5CC
:1003200092E20E94B4732CCE81E0C980C11001C05A
:1003300080E0909134068917C9F0D0904610D98298
:100340008093340687E490E10E94CB68D81608F0C9
:1003500054C029812F5F2983E22FF0E0E95BFF4E33
:100360008081807C8038A9F320934610009146104C
:1003700010E0095B1F4EC8010E94CB68898360E8CA
:1003800070E0C8010E94C0744981453108F019CA63
:1003900060E270E080E090E00E94C26F69816431A9
:1003A00009F40FCA60E270E080E090E00E94C26F42
:1003B0008981833109F405CA60E270E080E090E051
:1003C0000E94C26F9981923109F4FBC9292F30E054
:1003D0002E5F3F4F4AEF4203B001439F700D11243F
:1003E00060587F4F87E490E10E94C07460E270E043
:1003F00080E090E00E94C26FE4C910924610B6CF30
:1004000080918F07823059F0B8D9882349F08091C4
:10041000E51482FB882780F991E08927089581E01F
:10042000089581E00895DC01EC918E2F90E0FC01AD
:10043000EE0FFF1FE80FF91FE25DFC4E80818F7702
:1004400080830895892B79F41092900082E0809344
:1004500091001092950010929400C19A80917100C1
:100460008260809371000895B0E0A0E0EAE3F2E8D2
:100470000C94FAF0EC017B0188818C3008F0A4C068
:1004800090E0FC01EE0FFF1FE80FF91FE25DFC4E4C
:1004900080818F770E94EBB519821A8288812CE0C7
:1004A000622F0E949AF0829FB001112430E020E078
:1004B000AB01420F531FFA01EE0FFF1FE40FF51FB0
:1004C000E25DFC4E908197FD07C02F5F3F4F2C30BF
:1004D000310571F790E0B6DF7880072D10E06801F4
:1004E000CC0CDD1CF601E00FF11FE25DFC4E8081BB
:1004F0008068808377FC68C080E2E81682E0F806B6
:100500000CF03FC08A8128E532E0281B310987FDC5
:100510003395220F331F220F331F032E000C440B81
:10052000550B898178E8872E912C881A910887FDD0
:100530009394880C991C880C991C092C000CAA080F
:10054000BB0860E070E0CB01F7FC0AC0B701653B77
:10055000710514F064EB70E0072E000C880B990B0A
:10056000281939094A095B090E942EF024EB30E072
:1005700040E050E00E945FF0820E931EA41EB51E64
:1005800074018BE08715D8F0298188E890E0821B00
:10059000910927FD9395880F991F880F991FE816D9
:1005A000F906BCF402972FB7F894E601C00FD11FEB
:1005B000C25DDC4E880F991F9A8389832FBF62E347
:1005C00070E080E090E09CD8CDB7DEB7EDE00C9411
:1005D00016F12A8188E592E0821B910927FD939507
:1005E000880F991F880F991FE816F906DCF6C701D6
:1005F000D9CFCF93DF93EB01682F70E083E593E1D0
:1006000033DF688179818A819B81643F21E07207B1
:100610008105910520F464EF71E080E090E070D8EE
:1006200086B182958170DF91CF910895A4E0B0E00A
:10063000ECE1F3E80C9405F18EEE92E0A0E0B0E07E
:1006400089839A83AB83BC83BE016F5F7F4F8AE54A
:10065000D0DF2496E2E00C9421F1A4E0B0E0E3E3E3
:10066000F3E80C9405F18EEE92E0A0E0B0E089830F
:100670009A83AB83BC83BE016F5F7F4F8AE0B9DF93
:100680002496E2E00C9421F1A4E0B0E0EAE4F3E87F
:100690000C9405F184EF91E0A0E0B0E089839A83A7
:1006A000AB83BC83BE016F5F7F4F8CE3A2DF2496D8
:1006B000E2E00C9421F1A4E0B0E0E1E6F3E80C9470
:1006C00005F184EF91E0A0E0B0E089839A83AB83E9
:1006D000BC83BE016F5F7F4F80EA8BDF2496E2E030
:1006E0000C9421F11F920F920FB60F9211240BB6AA
:1006F0000F922F933F934F935F936F937F938F93BB
:100700009F93AF93BF93EF93FF938091AF0587FFC4
:1007100027C010929500109294008091AF058F5FD2
:100720008093AF058091AF05082E000C990B2091A6
:1007300052132817190629F024F08091AF058C3048
:10074000DCF18091940090919500049680349C494E
:1007500008F47DC08091940090919500049679C032
:100760008091AF05082E000C990B20915213281789
:10077000190699F294F2E091AF058E2FEE0F990BC6
:10078000FC01EE0FFF1FE80FF91FE25DFC4E8081B8
:1007900087FFC3CFE091AF058E2FEE0F990BFC01C1
:1007A000EE0FFF1FE80FF91FE25DFC4E808160E055
:1007B0008F770E941DD0B1CF209194003091950089
:1007C000E091AF058E2FEE0F990BFC01EE0FFF1F8E
:1007D000E80FF91FE25DFC4E81819281820F931F29
:1007E0009093990080939800E091AF058E2FEE0FC3
:1007F000990BFC01EE0FFF1FE80FF91FE25DFC4EA5
:10080000808187FF11C0E091AF058E2FEE0F990B0D
:10081000FC01EE0FFF1FE80FF91FE25DFC4E808127
:1008200061E08F770E941DD0FF91EF91BF91AF9152
:100830009F918F917F916F915F914F913F912F91F8
:100840000F900BBE0F900FBE0F901F90189580E475
:100850009CE990939900809398008FEF8093AF0567
:10086000E3CF9091C00095FFFCCF8093C600089520
:10087000CF93DF93EC018991882311F0F2DFFBCF56
:10088000DF91CF910895CF93DF93EC018991882375
:1008900011F0E7DFFBCF8DE0E4DF8AE0E2DFDF91FC
:1008A000CF910895CF93DF93EC01FE0184912196BF
:1008B000882311F0D6DFF9CFDF91CF9108950F9300
:1008C0001F93CF938C01C62F81EB9FE1EBDFC80113
:1008D000E9DF8AE3C6DF80E38C0FC3DF8AE0C1DF94
:1008E000CF911F910F910895CF92DF92EF92FF92D7
:1008F0006A017B01D7DF42E0C701B6010E940AB658
:10090000FF90EF90DF90CF900895CF93DF9368EC46
:100910007FE10E9457C7C0916213D0916313488151
:1009200059816A817B818FEB9FE1DEDF4C815D81A4
:100930006E817F818DEB9DE2D7DF40915E135091F8
:100940005F1360916013709161138AEB9DE2CCDFBD
:100950008CEB9FE1A7DF86EB9FE1A4DF8AE081DFDC
:10096000DF91CF910895C0DF8AE07BCFADE5B0E0A5
:10097000ECEBF4E80C94F5F070E060E085E40E94A4
:10098000D66D7C01182F8F3FB1F1882341F08BEA9F
:1009900091E288DFC35ADF4FE2E10C9411F16EEB74
:1009A00070E083E50E94D66D5C0165E070E083E451
:1009B0000E94D66D6C0160E085E50E94C26D2C96A8
:1009C0008FAF2C9760E08EE991E20E94485C0E9414
:1009D00002D169877A878B879C871F3F09F067C49C
:1009E00034E7A316B1040CF489C183E791E25ADF1E
:1009F0000E94DBC7CFCF6CE370E0D3CF20E030E0C4
:100A000040E05EE32BAF3CAF4DAF5EAFABC12AE938
:100A100039E949E15FE323962CAF3DAF4EAF5FAFBD
:100A20002397ADC14090B6125090B7126090B812A3
:100A30007090B91251C22B96EEADFFAD2B9740834B
:100A4000A4C24BEEC42ED12CE12CF12C22C384E1A4
:100A500090E0A0E0B0E08D879E87AF87B88B34E14F
:100A6000C32ED12CE12CF12C24C3CD86DE86EF865B
:100A7000F88A1FC32B96EEADFFAD2B978083E9C399
:100A8000D501C4012EA53FA548A959A9821B930BE6
:100A9000A40BB50BB7FD47C02D968FAD2D970E94C7
:100AA0004C278AE0DEDED501C4018053984FAF4F5A
:100AB000BF4F8EA79FA7A8ABB9AB9AA991116FC0E2
:100AC0002BA93CA94DA95EA9C301B2010E9490F2D5
:100AD00018160CF050C020E030E040E050E4C301B4
:100AE000B2010E942DF16BAB7CAB8DAB9EAB2AA506
:100AF0003BA54CA55DA5280D391D4A1D5B1D2FABDF
:100B000038AF49AF5AAF6D966CAD7DAD8EAD9FAD30
:100B10006D970E9415EAA30192010E940FEA881FB7
:100B20008827881F8AAB89859A85AB85BC85898F84
:100B30009A8FAB8FBC8F29893A894B895C8928179A
:100B400039074A075B0720F4298F3A8F4B8F5C8F58
:100B5000898D9A8DAB8DBC8D881A990AAA0ABB0A19
:100B600091E889169FE4990692E1A906B10460F123
:100B700087E990E22DC2D501C4012FA938AD49AD56
:100B80005AAD821B930BA40BB50B4FEE52E16EEFE7
:100B900072E1B7FDC8CF812F0E949328C4CF699618
:100BA0006CAD7DAD8EAD9FAD69970E9415EA9B013E
:100BB000AC01C301B2010E940FEA87FFB4CF4CE23F
:100BC00053E16CE373E1E7CF2996AEADBFAD299752
:100BD000A215B3050CF08FC0B3E02B1631040CF452
:100BE0008AC08AE390E25EDE1F3F09F066C0EAE257
:100BF000F0E2FE83ED8389E190E254DE8D819E81F7
:100C000051DE49815A816B817C8186E390E2ABDEC3
:100C100089E190E247DE8D819E8144DE4D8D5E8DBF
:100C20006F8D78A182E390E29EDE89E190E23ADE68
:100C30008D819E8137DE49A15AA16BA17CA18EE2F4
:100C400090E291DE2C963FAD2C97332309F4D0CE61
:100C50002CEA35EC47E25EE36D8D7E8D8F8D98A199
:100C60000E9474EA6B017C0120E030E543EC50E423
:100C700069A17AA18BA19CA10E9474EA29813A8181
:100C80004B815C811F3FF1F420933F073093400775
:100C90004093410750934207C0924307D0924407C4
:100CA000E0924507F0924607609347077093480724
:100CB0008093490790934A079BCE21E13DE23E8312
:100CC0002D8399CF2093BD123093BE124093BF1253
:100CD0005093C012C092C112D092C212E092C312BD
:100CE000F092C4126093C5127093C6128093C7121B
:100CF0009093C8127DCE0E941C71CEC08FE591E208
:100D0000D1DD0E94F5278FE780933E072CE330E08A
:100D1000C9A6A8EEB3E00E948BF06AA77BA78CA7B8
:100D20009DA729853A854B855C85260F371F481F6F
:100D3000591F2FAB38AF49AF5AAF81E0809369019B
:100D400060E08BE491E20E94485C02E00E0D02300C
:100D500008F054CE8BEA9AEAAAEABEE38BAF9CAFC6
:100D6000ADAFBEAF023008F052CE8DEC9CECACE4DF
:100D7000BEE323968CAF9DAFAEAFBFAF23970230DB
:100D800008F4E12C2D96EFAE2D9789859A85AB85D9
:100D9000BC85898B9A8BAB8BBC8B8EA79FA7A8AB8E
:100DA000B9AB19A21AA21BA21CA21D8E1E8E1F8EE9
:100DB00018A219821A821B821C822FE730E040E0C1
:100DC00050E02D873E874F87588B80E090E4ACE160
:100DD000B6E48D839E83AF83B8871D8A1E8A1F8ADF
:100DE000188EFFE7CF2ED12CE12CF12C1AAA1BAACA
:100DF0001CAA1DAA1EAA1DA21EA21FA218A691E02F
:100E000024969FAF2497312C212C412C512C320158
:100E100095010B2C000C440B550B61962CAF3DAF8C
:100E20004EAF5FAF619749A5042E000C550B299674
:100E30005FAF4EAF299757E11502C0011124DC01C5
:100E4000A454BD4E2B96BFAFAEAF2B97C5014E96A7
:100E50009C01092E000C440B550B65962CAF3DAF41
:100E60004EAF5FAF6597CC979C01990F440B550B24
:100E700069962CAF3DAF4EAF5FAF699736E0A31ACE
:100E8000B108C5010B2C000CAA0BBB0B6D968CAFE7
:100E90009DAFAEAFBFAF6D9780916901882309F414
:100EA00098C00E9402D14B015C0190919D036E9607
:100EB0009FAF6E97992309F47BC00E9489291092F5
:100EC0009D031F3F09F0AECD409038075090390781
:100ED00060903A0770903B07A30192016D897E896B
:100EE0008F89988D0E9490F287FF04C04D8A5E8A98
:100EF0006F8A788EA30192016D817E818F819885A2
:100F00000E940FEA181624F44D825E826F82788662
:100F100061966CAD7DAD8EAD9FAD61970E9415EA77
:100F2000698F7A8F8B8F9C8F2496AFAD2497AA23DD
:100F300009F454C09B01AC01C301B2010E9490F2BC
:100F40001816B4F5D501C40129893A894B895C8901
:100F5000821B930BA40BB50BAC01BD014858534148
:100F60006109710977FD24C04D855E856F8578899B
:100F70004C195D096E097F097595679557954795D9
:100F80001F3F09F058CD40933E078DA39EA3AFA30A
:100F9000B8A7298D3A8D4B8D5C8D2D8B3E8B4F8B59
:100FA000588F89869A86AB86BC8624961FAE249776
:100FB00065966CAD7DAD8EAD9FAD65970E9415EACF
:100FC000A30192010E940FEA87FF5ACD85EB90E2C0
:100FD00069DC109269010E94F5270ACD298D3A8DAE
:100FE0004B8D5C8DC301B2010E940FEA87FFE0CFF9
:100FF000D501C40129853A854B855C85821B930BFD
:10100000A40BB50BAC01BD014858534161097109EE
:1010100077FDCECF2114310409F40AC12DA13EA1E0
:101020004FA158A5280F391F4A1F5B1F298B3A8BE8
:101030004B8B5C8B2DA13EA14FA158A5281B390BD2
:101040004A0B5B0BC701B6010E942EF029893A8931
:101050004B895C890E945FF0CD84DE84EF84F88840
:10106000C20ED31EE41EF51E34E1C316D104E10402
:10107000F1040CF4ECCC4CEEC416D104E104F10400
:101080000CF0DFCC50E8C516D104E104F1040CF4F7
:10109000ECCCCD86DE86EF86F88A8EEF90E0A0E07D
:1010A000B0E09C01AD012C193D094E095F096901B1
:1010B0007A0183E491E2F6DB6D857E858F859889E0
:1010C0000E9417768EE391E2EDDBC701B6010E9424
:1010D00017764D815E816F81788587E391E204DC2C
:1010E0004D895E896F89788D80E391E2FDDB93E025
:1010F000291631040CF49CC0C701B6010E9415EA00
:1011000020E030E040E850E40E9474EA69837A838A
:101110008B839C832D813E814F8158856D897E898B
:101120008F89988D0E942CF12BED3FE049EC5FE315
:101130000E9474EA9B01AC0169817A818B819C8158
:101140000E94A4F127966CAF7DAF8EAF9FAF27971B
:1011500069897A898B899C890E9415EA2FE632E198
:1011600043E85AE30E9474EA6D837E838F839887F5
:1011700023962CAD3DAD4EAD5FAD239727966CAD5C
:101180007DAD8EAD9FAD27970E9474EA69837A8307
:101190008B839C839B01AC010E942DF12D813E81AC
:1011A0004F8158850E94A4F16D8F7E8F8F8F98A3F9
:1011B0002BAD3CAD4DAD5EAD6D817E818F8198854F
:1011C0000E9474EA29813A814B815C810E9474EA11
:1011D00069A37AA38BA39CA327964CAD5DAD6EAD9E
:1011E0007FAD27978AE291E27FDB4D815E816F813F
:1011F000788584E291E2B7DB85E191E2023010F07C
:1012000086E091E24FDB49815A816B817C8180E0ED
:1012100091E26ADB4D8D5E8D6F8D78A18AEF90E251
:1012200063DB49A15AA16BA17CA184EF90E29BDB17
:101230008D859E85AF85B8898C0D9D1DAE1DBF1D0A
:10124000B595A795979587951F3F09F013CC809387
:101250003E072996FFAD2997FF9329A52F933F922B
:101260002F9280EE90E29F938F938BEE90E29F936C
:101270008F931F920E942B5C3FEF231A330A0FB605
:10128000F894DEBF0FBECDBF898D9A8DAB8DBC8D1E
:101290008D839E83AF83B887898A9A8AAB8ABC8AFA
:1012A0006E969FAD6E9724969FAF249781CE8E2C1D
:1012B0000E2C000C9908F40183E0EE0FFF1F8A95B5
:1012C000E1F7EF59FE4F868197810F978A159B05AD
:1012D0000CF48BCB8FE591E2E5DA0E94F52787E1EC
:1012E000889DF001899DF00D1124EE54FD4E8FE78D
:1012F000828724E130E00CCDCF93DF9362E179E186
:101300000E9457C7C4E3D7E04B855C856D857E8519
:1013100089E099E1E9DA20E030E543EC50E46F85BB
:10132000788989899A890E9474EAAB01BC0186E0B8
:1013300099E1DADA2CEA35EC47E25EE36B897C89E5
:101340008D899E890E9474EAAB01BC0183E099E11A
:101350000ADBDF91CF91089564E978E10E9457C7D5
:101360006091810D7091820D8091830D9091840D1B
:101370000E9413EAAB01BC018BE898E1B5DA409119
:10138000B10D5091B20D6091B30D7091B40D88E81C
:1013900098E1AADA4091B50D5091B60D6091B70D64
:1013A0007091B80D85E898E19FDA409193075091CC
:1013B0009407609195077091960782E898E1D3CAE7
:1013C000CF93DF9368E378E10E9457C7C1E7DDE080
:1013D0004CA95DA96EA97FA98FE298E185DA48AD95
:1013E00059AD6AAD7BAD8CE298E17EDA4CAD5DAD76
:1013F0006EAD7FAD85E898E1B6DADF91CF910895C3
:10140000CF93DF9364E178E10E9457C7C1E7DDE045
:101410004CA15DA16EA17FA18BE098E165DA48A5A2
:1014200059A56AA57BA58DEB9DE25EDA4CA55DA56D
:101430006EA57FA58AEB9DE257DA48A959A96AA94A
:101440007BA987EB9DE28FDADF91CF910895CF934F
:10145000DF936FEE77E10E9457C7C1E7DDE0688157
:1014600079818A819B810E9413EAAB01BC0186EEDF
:1014700097E13ADA6C817D818E819F810E9413EA27
:10148000AB01BC018DEB9DE22FDA688579858A85F9
:101490009B850E9413EAAB01BC018AEB9DE224DA32
:1014A0006C857D858E859F850E9413EAAB01BC010A
:1014B00087EB9DE258DADF91CF9108958F929F924A
:1014C000AF92BF92EF92FF920F931F93CF93DF9350
:1014D0008FE496E1E7D9C0E0D7E0D15019F080E27F
:1014E000C0D9FBCF8C2F0E94726DCF5FC730A1F7A0
:1014F0008AE0B7D908EB12E0C0E080E2B2D98C2FC5
:101500000E94726D7801D7E080E2ABD9F70180804C
:101510009180A280B38020E030E0A901C501B40130
:101520000E9490F287FD02C08BE29BD943E0C50187
:10153000B4010E940AB6D150FCE1EF0EF11CD111AA
:10154000E3CF8AE08ED9CF5F0C5F1F4FC730A9F67B
:101550008AE087D9DF91CF911F910F91FF90EF9093
:10156000BF90AF909F908F900895811105C088E43F
:1015700096E198D98AE075C98CE496E1FACF81E4C6
:1015800096E190C98BE396E18DC9CF9384E50E94E3
:10159000266AC0E08823D9F00E94986DC82F1816DB
:1015A000B4F4F0DF8DE45DD9809124069091250696
:1015B0000E94A57B8EED99E175D96C2FCC0F770B2E
:1015C000880B990B0E94C0B38AE04BD9CFEF8C2FC8
:1015D000CF910895CF93C82F68EF78E10E9440C75C
:1015E000C11101C0CFDF4091BD125091BE12609178
:1015F000BF127091C0128FEE98E176D920E030E5ED
:1016000043EC50E46091C1127091C2128091C312F8
:101610009091C4120E9474EAAB01BC018CEE98E177
:1016200063D92CEA35EC47E25EE36091C512709114
:10163000C6128091C7129091C8120E9474EAAB0141
:10164000BC0189EE98E150D98AE00BD9CF91089579
:10165000B0E0A0E0EEE2FBE80C94FFF061E083E58F
:101660000E94C26DC1E0C82761ED79E18C2F0E9414
:1016700040C7C11101C086DF89EC99E113D986EB1F
:101680009FE110D98AE0EDD867EB79E18C2F0E94B9
:1016900040C7C11101C076DF8AE999E103D98C2FD7
:1016A0000E9460C78C2FACDE8C2FD1DE8C2F88DEA1
:1016B0008C2F52DE6EE479E18C2F0E9457C7D091B7
:1016C000B30285E499E1EED86D2F70E090E080E000
:1016D0000E94C0B34091B4025091B5026091B6022D
:1016E0007091B7028AEB9DE2FFD888E399E1DAD8DE
:1016F0008091B3023ADF20E030E0A90160918403D9
:101700007091850380918603909187030E940FEA70
:10171000882379F188EBE82E82E0F82E10E067014B
:1017200000E0C11101C02EDF80E999E1BBD8802F14
:101730000E94726D8DE899E1B5D8812F0E94726D7B
:101740008AEB9DE2AFD8F60160817181828193813D
:1017500045E00E940AB68AE084D80F5FFCE1CF0E14
:10176000D11C0730F1F61F5F84E0E80EF11C173042
:10177000B1F662E779E18C2F0E9440C70BE417E0D5
:10178000D0E0C11101C0FEDE89E699E18BD88D2F32
:101790000E94726DF80160817181072E000C880B28
:1017A000990B0E9415EAAB01BC0186E699E19CD831
:1017B000F80162817381072E000C880B990B0E943F
:1017C00015EAAB01BC0183E699E18ED8F801E4800B
:1017D000F58080E699E166D8C7010E94A57B8AE082
:1017E00040D80A5F1F4FD13059F48C2FF3DE8C2F75
:1017F00083DD8C2F8AD8CDB7DEB7E8E00C941BF1DF
:10180000D1E0BFCFACE1B0E0E8E0FCE80C94F5F04B
:1018100083E50E94AF69182F882309F41CC10E9438
:10182000B36D8D838091750190917601A0917701C0
:10183000B0917801898F9A8FAB8FBC8F20917901FD
:1018400030917A0140917B0150917C012D8B3E8B30
:101850004F8B588F80917D0190917E01A0917F01E7
:10186000B09180018D879E87AF87B88B112331F0AF
:101870009D81911103C080E00E94CA7980911E066B
:1018800090911F06A0912006B091210635E1B695F2
:10189000A795979587953A95D1F79C01AD01217051
:1018A00033274427552729873A874B875C8720E0D1
:1018B00030E0A901609184037091850380918603D3
:1018C000909187030E940FEA882309F4C8C083E43B
:1018D0000E94AF69882309F493C00E94E26D698B6E
:1018E0007A8B8B8B9C8B48EB52E05F834E838A0113
:1018F00057E05887412C512C98EC692E92EC792EA8
:10190000812C912C28ECA22E22E4B22E312C212CF9
:10191000F101EE0FFF1FEE0FFF1FE00FF11FC08060
:10192000D180E280F380A7019601C501B4010E9435
:101930000FEA181614F446015701A7019601C301D6
:10194000B2010E9490F287FF02C0260137018FEF9B
:10195000281A380A97E029163104D1F6A885A15033
:10196000A887045E1F4FA111D1CFA3019201C50129
:10197000B4010E942DF120E030E040E05FE30E94DE
:1019800074EA29893A894B895C890E942DF14B01BF
:101990005C012DEB37E346E855EB0E940FEA87FD2B
:1019A0000AC02DEB37E346E855E3C501B4010E94B8
:1019B00090F218162CF580E00E94CA7917E0EE80AC
:1019C000FF8007E0F70161917191819191917F0111
:1019D0006F01F4E0CF1AD108A50194010E942CF107
:1019E000D6016D937D938D939C931397015051F77E
:1019F0001150EE81FF817C96FF83EE831111DFCFC2
:101A000089859A85AB85BC85892B8A2B8B2B79F0B0
:101A100020E030E0A90160918403709185038091FA
:101A20008603909187030E940FEA811147DD8AE5C2
:101A30000E94AF69882359F00E94E26D69837A831E
:101A40008B839C8360E0CE0101960E94567A8D8143
:101A50000E94CA7914C02091B3022D83E3CEFD8188
:101A6000F11108C029853A854B855C85232B242BF1
:101A7000252BE9F287DD81E297E10E9452849D8166
:101A8000992349F08091B302811105C078DD82E08D
:101A900097E10E94528476DD84EF96E10E945284A1
:101AA0008091B30262DD6EDD87EE96E10E94528482
:101AB000C090B402D090B502E090B602F090B702A8
:101AC00020E030E0A901C701B6010E9490F218168B
:101AD0000CF040C042E0C701B6010E940AB68DE09A
:101AE0000E9431848AE00E943184298D3A8D4B8D89
:101AF0005C8D609175017091760180917701909174
:101B000078010E940FEA81111FC02D893E894F89FB
:101B1000588D6091790170917A0180917B0190914B
:101B20007C010E940FEA81110FC020917D0130914C
:101B30007E0140917F01509180016D857E858F856A
:101B400098890E940FEA81110E94F73F6C96E2E1AA
:101B50000C9411F182EE96E10E945284C6CFCF938D
:101B6000DF93EB010E945284BE01DD0F880B990BBD
:101B70000E94C0B3DF91CF9108950E94F5270E9483
:101B8000734480912F07813099F0F9DC84EC95E162
:101B90000E94528460E08AEB95E10E94485C6EE509
:101BA00071E080E090E00E94807B81E080932F07CD
:101BB0000895CF92DF92EF92FF921F93CF93DF931E
:101BC00000D000D0CDB7DEB78EEEC82E82E0D82E82
:101BD000E12CF12CC982DA82EB82FC82BE016F5FBC
:101BE0007F4F8AE50E94F98281110EC010E0812F9B
:101BF0000F900F900F900F90DF91CF911F91FF905A
:101C0000EF90DF90CF9008950E945B83C982DA82C3
